:020000040000FA
:100000006005002089150000392B00001D14000038
:100010001D1400001D1400001D1400001D1400001C
:100020001D1400001D1400001D140000750F0000B9
:100030001D1400001D1400001D0F0000CF2A000039
:100040004915000049150000491500004915000038
:100050004915000049150000491500004915000028
:100060004915000049150000491500004915000018
:100070004915000049150000491500004915000008
:1000800049150000491500004915000049150000F8
:1000900049150000491500004915000049150000E8
:1000A00049150000491500004915000049150000D8
:1000B00049150000491500004915000049150000C8
:1000C00049150000491500004915000049150000B8
:1000D00049150000491500004915000049150000A8
:1000E0004915000049150000491500004915000098
:1000F0004915000049150000491500004915000088
:100100004915000049150000491500004915000077
:100110004915000049150000491500004915000067
:100120004915000049150000491500004915000057
:100130004915000049150000491500004915000047
:10014000491500007BB972B90029BEBF00204FF0ED
:10015000004106E008BF00281CBF6FF000414FF0CF
:10016000FF3000F0AFB9ADF1080C6DE904CE002905
:1001700009DB002B1ADB00F035F8DDF804E0DDE9DF
:10018000022304B07047404261EB4101002B1BDBAE
:1001900000F028F8DDF804E0DDE9022304B0404275
:1001A00061EB4101524263EB43037047524263EB00
:1001B000430300F017F8DDF804E0DDE9022304B0A2
:1001C000404261EB41017047524263EB430300F050
:1001D00009F8DDF804E0DDE9022304B0524263EBE4
:1001E000430370472DE9F0478C46089D04468A4634
:1001F000002B4AD18A42174662D9B2FA82F64EB132
:10020000C6F1200E01FA06F3B740B44020FA0EFE04
:100210004EEA030A4FEA1748230C1FFA87F9BAFB84
:10022000F8FE08FB1EAA0EFB09F243EA0A439A42B3
:100230000BD9FB180EF1FF312CBF012000209A4290
:1002400002D9002800F02A818E469A1AA3B2B2FB86
:10025000F8F008FB102200FB09F943EA0244A1452B
:1002600007D93C1900F1FF3302D2A14500F21081F9
:100270001846A4EB090440EA0E4000211DB1F440E9
:100280000023C5E90043BDE8F0878B4208D9002D63
:1002900000F0F2800021C5E9000C0846BDE8F087B7
:1002A000B3FA83F100294ED16345C0F0E880824261
:1002B00040F2E5800846002DE5D0C5E9004AE2E7B6
:1002C00002B9FFDEB2FA82F6002E40F099808B1A56
:1002D0004FEA124E1FFA82F801214FEA144CB3FB89
:1002E000FEF20EFB123008FB02F94CEA004CE1452D
:1002F00008D917EB0C0C02F1FF3302D2E14500F2F2
:10030000CA801A46ACEB090CA3B2BCFBFEF00EFB94
:1003100010CC08FB00F843EA0C44A0450ED93C1968
:1003200000F1FF332CBF4FF0010C4FF0000CA04543
:1003300003D9BCF1000F00F0A8801846A4EB080414
:1003400040EA02409AE7C1F120048B4002FA01FE24
:100350000CFA01F6E24020FA04F72CFA04FC00FA49
:1003600001F813433E431F0C320C1FFA83F9BCFB08
:10037000F7F007FB10CC00FB09FA42EA0C4CE2450F
:1003800008D913EB0C0C00F1FF3202D2E24500F267
:1003900089801046ACEB0A0CB6B2BCFBF7FA07FB3F
:1003A0001ACC0AFB09F946EA0C42914506D99A187B
:1003B0000AF1FF3601D291457AD8B2464AEA0040A6
:1003C000A2EB0902A0FB0E67BA42B446B94602D3BB
:1003D00007D1B04505D2B6EB0E0C67EB030301382D
:1003E0009946002D6BD0B8EB0C0362EB090202FAC0
:1003F00004F4CB40CA4000211C43C5E9004242E757
:10040000B740C6F1200201FA06F3B44021FA02FC1B
:100410004FEA174E20FA02F21FFA87F8BCFBFEF1F2
:100420001A430EFB11CC01FB08F0130C43EA0C4CF1
:10043000604507D917EB0C0C01F1FF3301D2604581
:1004400033D81946ACEB000C92B2BCFBFEF00EFBAD
:1004500010CC00FB08F342EA0C4C634507D917EBBC
:100460000C0C00F1FF3201D2634525D81046ACEBED
:10047000030340EA014130E72946284603E7841A8E
:100480006CEB030301209A4615E702383C4455E71C
:1004900002383C44EDE6023ABC4433E7AEF1020ECA
:1004A0003B44D2E602389C4474E70239BC44C9E7B5
:1004B000AAF1020A1A4481E70238BC44D7E7294668
:1004C000E1E600BF704700BF2DE9E04F2746A04698
:1004D000A146A246A346A4462DED108B4FF0000581
:1004E00045EC185B45EC195A45EC1A5A45EC1B5A79
:1004F00045EC1C5A45EC1D5A45EC1E5A45EC1F5A5A
:10050000F1EE105A4FF66076C0F6FF763540E1EE18
:10051000105A84F3008825462646A447BDEC108B6C
:10052000BDE8E08F82680C4B9A60036883F388888B
:10053000436883F38988027B02F00101EFF394831F
:1005400023F00303920748BF43F0020309B143F0CD
:10055000010383F39488704700ED02E0084AD368F2
:1005600048B123F400531B041B0C43F0BF6343F456
:100570000033D36070479BB243F40053F5E700BFEC
:1005800000ED00E0084AD36840B19BB243F48043D9
:1005900043F0BF6343F40033D360704723F48043D8
:1005A0001B041B0CF4E700BF00ED00E0084AD36811
:1005B00040B19BB243F0080343F0BF6343F4003300
:1005C000D360704723F008031B041B0CF4E700BF43
:1005D00000ED00E0034AD2F88C3043F44063C2F8E7
:1005E0008C30704700ED00E0084B1A6818B142F0FB
:1005F00001021A60704722F001021A601A6811B1F4
:1006000042F00202F5E722F00202F2E7D0ED00E04C
:100610000B6801330B60014B1B681847A00E0020CC
:100620002DE9F04F85B00E9C9B46012CB8BF0124EC
:10063000012B0CBF30232023154680468946012616
:100640000A270022DFF870A0019402930AF1010446
:100650000AB9AA451ED2B5FBF4F049463030C0476E
:1006600001220136B5FBF4F10A23013F012F04FBFF
:100670001155BAFBF3FAE9D1494605F13000C047FC
:10068000BBF1030F03D1019B9C1B002C0FDC05B0B9
:10069000BDE8F08F019BBB42E4DBBBF1020FE1D868
:1006A0004946029803920136C047039ADAE7494661
:1006B0002020C047013CE8E7FFC99A3B002313B55F
:1006C00002AC44F8043D02460B460348214602F0C2
:1006D00052F802B010BD00BF1106000010B54FF077
:1006E0002003EFF3118483F31188BFF36F8F00F0C1
:1006F00013F80122064BC3F840254FF0FF32054B9B
:100700009A62DA6284F31188BFF36F8F002010BD04
:100710000090035000ED00E0524A136843F00203DA
:1007200013600022D30003F57F03D3F800130131D7
:1007300008D0D3F800130132D3F80433B2F5807F28
:100740000B60EFD1484AD36913F001033BD0474B0C
:100750001946D3F80024012AFBD1C3F80425D1F8A7
:100760000034012BFBD1404BDA69D20708D5DA6996
:100770003E4922F00102DA61D1F80024012AFBD1BE
:100780001A6A01320AD11A6A22F0FF0242F02002EC
:100790001A62364AD2F80034012BFBD10022334BC7
:1007A000C3F80425D3F80024012AFBD1BFF34F8FEF
:1007B0002F49304BCA6802F4E0621343CB60BFF3A9
:1007C0004F8F00BFFDE7126A0132C0D02A4A11687C
:1007D00009290AD129490968013901299EBF4FF029
:1007E0005021C1F81431C1F818311368092B09D10F
:1007F000224B1B68012B01BF214A1360A2F638224D
:10080000C2F878351C4B1A68092A0BD11B4A1268AA
:10081000022A07D100211A4A11600121A2F63822CA
:10082000C2F878151B68092B06D1144B1B68022BE4
:1008300002BF0C22134B1A600D4BD3F88C2042F4EC
:100840004062C3F88C20D3F8882042F47002C3F8C9
:100850008820BFF34F8FBFF36F8F0B4B0B4A1A608B
:10086000704700BFD0ED00E00080FF000090035013
:1008700000ED00E00400FA053001FF003401FF0044
:10088000384A0050E4AE0350A40E00200090D0037C
:1008900010B54FF02003EFF3118283F31188BFF3FB
:1008A0006F8F154C237833B982F31188BFF36F8FA4
:1008B0006FF0440010BD013BDBB2237033B182F313
:1008C0001188BFF36F8F6FF00F00F3E70B4B01211F
:1008D000187838B1217082F31188BFF36F8F6FF0F1
:1008E0000A00E7E7197082F31188BFF36F8F044A9B
:1008F00011601870DEE700BF5A0100205901002086
:100900000450005010B54FF02002EFF3118382F332
:100910001188BFF36F8F144C207898B183F311883E
:10092000BFF36F8F4FF05022D2F81C34D2F8182446
:1009300003F0030343F48033934314BF6FF0430089
:10094000002010BD0122227083F31188BFF36F8F46
:100950004FF05023C3F80401C3F818150221C3F85F
:1009600004139A60DEE700BF58010020F8B54FF08D
:100970002002EFF3118382F31188BFF36F8F294AAE
:100980001078441C147080B183F31188BFF36F8F0B
:100990004FF05023D3F80C3403F00113B3F1011FCF
:1009A0000CBF00206FF0430009E01F4D2F783FB1CE
:1009B000107083F31188BFF36F8F6FF00A00F8BDDA
:1009C00001262E7083F31188BFF36F8F4FF05024F0
:1009D00021B3052000F0C0FCC4F80071D4F8043342
:1009E000C4F804632660D4F800219AB10022DB0722
:1009F00058BF0123C4F800214FF0200258BFC4F8AB
:100A000008330A4B0520C3F8802100F095FC002331
:100A10002B70BDE720BF40BF20BFE4E7C4F8001142
:100A20002660F4E75A0100205901002000E100E0AF
:100A30000022114B10B4C3F840214FF02002EFF315
:100A4000118482F31188BFF36F8FD3F8040540F24D
:100A500047130A4A1168401A20F07F40B0FBF3F0B8
:100A600003FB0013136084F31188BFF36F8F5DF8ED
:100A7000044B01F07DBD00BF005001500800002074
:100A800038B51B4801F086F970B3436802211B6832
:100A90009847002440F24713164D4FF40012C5F852
:100AA0000845C5F840354FF48033C5F84433C5F8E0
:100AB0000433114B01211C60104B1520C3F8802119
:100AC000224600F05DFC152000F036FC0123204694
:100AD0000B4A13602B60D5F8043503F2471323F05B
:100AE0007F43C5F8403538BD4FF0FF30FBE700BF0E
:100AF000B3330000005001504051015000E100E0CC
:100B0000085001504CF6690270B5B0F1FF3F08BFC4
:100B100010464FF02003EFF3118483F31188BFF3E5
:100B20006F8F01389042124DA8BF10462E6840F2D8
:100B30004715104920EAE070D1F804359A1B22F0DD
:100B40007F4202F5A37205FB0020B0FBF5F005FB28
:100B50000060C31A23F07F431F2B98BF401920F079
:100B60007F40C1F8400584F31188BFF36F8F70BDDB
:100B700008000020005001504FF02002EFF31183D5
:100B800082F31188BFF36F8F084AD2F80405084A30
:100B90001268801A40F2471220F07F40B0FBF2F05A
:100BA00083F31188BFF36F8F704700BF005001506F
:100BB0000800002008B543B2002B0CDB012200F036
:100BC0001F018A405B091049203341F82320BFF3FD
:100BD0004F8FBFF36F8F830003F1A04303F54053A2
:100BE0003128D3F8002806D0002A07DA02F00302E1
:100BF000023A012A02D8054AC3F80028002101F070
:100C00006AFF002008BD00BF00E100E00001008095
:100C100030B54FF4004448F2040585B04FF400416C
:100C20002C4801F004FF21682B4801F000FF2968DF
:100C30002A4801F0FCFE10220021684601F0C5FFA1
:100C40002368684600930294FFF76CFC0120FFF7CD
:100C500099FC0020FFF782FC0020FFF7A7FC012190
:100C60000020FFF7C1FCFFF7B5FC2C681C4801F021
:100C7000DEFE0820FFF79EFF24F00104BFF34F8F34
:100C8000BFF36F8F64086400204621462246234646
:100C90009FED140ADFED130A9FED121ADFED111A12
:100CA0009FED102ADFED0F2A9FED0E3ADFED0D3A92
:100CB0009FED0C4ADFED0B4A9FED0A5ADFED095A12
:100CC0009FED086ADFED076A9FED067ADFED057A92
:100CD000FFF7FAFB9E340000B5340000CA34000070
:100CE000E8340000000000002DE9F8435D4801F001
:100CF0009EFE0021DFF8AC815B4F5C4D58F821402F
:100D0000CA0301F5C07347F82340594802F5004370
:100D10004E1C01F08CFE574B14F0100F56495748EB
:100D200008BF194601F083FE14F0040F14BF7221AE
:100D30002D21284601F07BFE14F0020F14BF77210D
:100D40002D21284601F073FE14F0010F14BF782105
:100D50002D21284601F06BFE14F4807F14BF6C2116
:100D60002D21284601F063FE454801F060FE202E4B
:100D70003146C3D1424801F05AFE424801F057FEC5
:100D80000021DFF82481384F384D58F821404A03BC
:100D900001F5E07347F823403B4802F500534E1C31
:100DA00001F045FE334B14F0100F3349334808BFB0
:100DB000194601F03CFE14F0040F14BF72212D21DE
:100DC000284601F034FE14F0020F14BF77212D21C4
:100DD000284601F02CFE14F0010F14BF78212D21BC
:100DE000284601F024FE14F4807F14BF6C212D21CD
:100DF000284601F01CFE224801F019FE202E314643
:100E0000C3D100241E4801F012FE204801F00FFE5D
:100E1000154B1F4DDFF89480DFF89490C3F8C04461
:100E200005EBC406777955F83420002F14BF4346EC
:100E30004B462146174801F0FAFD57B916480134D0
:100E400001F0F5FD122CEBD10D48BDE8F84301F09F
:100E5000EEBD3079FFF7AEFE08B11048EFE710485D
:100E6000EDE700BFF13300000030005029340000EE
:100E700014340000DA330000D1330000873400005E
:100E80007F3800002C3400004E3400006234000033
:100E9000543200007E3400008A3400009134000097
:100EA00099340000D4310000E4320000E633000041
:100EB000DE33000004488168406A884203D0034959
:100EC0004FF080520A6070471801002004ED00E0E6
:100ED000002320210348C2180133412B82F800135C
:100EE000F9D1704700E100E0094A0A4993680968AE
:100EF0005866996608494B6843F080534B6000235D
:100F000083F31188BFF36F8F9368986E704700BFAB
:100F1000180100209C33000000ED00E0202080F349
:100F20001188BFF36F8F11498A684FF02800104471
:100F3000EFF3098C80E8F01F0D4F4FF000664A6A0E
:100F40008A603E60506E0023536680F3118804B5BA
:100F50000648806801F0F7FDBDE8044002F1280072
:100F600090E8F01F8CF309887047000018010020FA
:100F700004ED00E01EF0040F0CBFEFF30880EFF368
:100F80000980816931F8021C11F0FF010229FFD0AC
:100F900001B501F0C9FD01BD38B51B4C05461B4824
:100FA00001F045FDA36AD90602D5194801F03FFDBD
:100FB000A36A1A0702D5174801F039FDA36A9B07F7
:100FC0000ED5154801F033FD616BA36A180607D5ED
:100FD000124801F02CFD1DB1A36A23F08003A36227
:100FE000094CA36ADA0702D50D4801F020FDA36A77
:100FF0009B0602D50B4801F01AFDA36AA36A0020E4
:1010000043F0FF03A36238BD00ED00E04F3600005F
:10101000663600009A360000AE360000C736000083
:10102000DE360000FE36000038B51E4C05461E4870
:1010300001F0FDFCA36AD90402D51C4801F0F7FCBD
:10104000A36A1A0502D51A4801F0F1FCA36A9B05B0
:101050000ED5184801F0EBFCA16BA36A180407D564
:10106000154801F0E4FC1DB1A36A23F40043A36218
:101070000C4CA36A590502D5104801F0D8FCA36AAC
:10108000DA0509D50E4801F0D2FC064A0020936A21
:1010900043F47F43936238BDA36A9B04F5D50948A6
:1010A000F1E700BF00ED00E0C1350000D8350000D9
:1010B0009A360000EA350000043600001A360000B7
:1010C00036360000FE36000010B51C4C1C4801F0FE
:1010D000AEFCA36A9A0102D51A4801F0A8FCA36AE3
:1010E000DB0102D5184801F0A2FCA36ADC0202D59C
:1010F000164801F09CFC114CA36A180302D5144851
:1011000001F095FCA36A590302D5124801F08FFC47
:10111000A36A9A0302D5104801F089FC074CA36A20
:10112000DB0302D50D4801F082FCA36A00206FEAC0
:1011300003436FEA1343A36210BD00BF00ED00E05C
:101140000E380000273800003B38000056380000F9
:1011500081380000A0380000C6380000E1380000E7
:1011600010B51A4C1A4801F062FCA169636958066F
:1011700002D5184801F05BFC6369D90707D516480A
:1011800001F055FC636943F0FF03636110BD6369BF
:101190009A0701D51148F3E763695B0701D5104849
:1011A000EEE76369180701D50E48E9E76369D906D8
:1011B00001D50D48E4E763699A0601D50B48DFE7DE
:1011C00063691B06DED50A48DAE700BFD0ED00E010
:1011D0002E370000483700005937000070370000F4
:1011E0008F370000AB370000C9370000DF37000041
:1011F000FA3700003D4B70B55E6801F07F43B3F1F4
:101200007F4F05460C465DD111F0010041D04806E4
:101210001BD42968364B37480B44012B98BF296CE7
:1012200001F005FC14F00804304B09D0EFF3898578
:101230005C6814F4006408D12F4801F0F8FB41E029
:10124000EFF388855B681905F6D4C6F30806F21E2D
:10125000092A3FD8DFE802F005383A2D343E3E3EF9
:101260003E3C264801F0E3FB204BDA6A920701D5A9
:101270002348E2E7D86A10F080400AD0214801F004
:10128000D6FB214B1B784BB10120FFF785FE0628CA
:101290002BD02946BDE8704000F0D2B81B4B1B781C
:1012A0001BB10120FFF7C0FEF1E7194B188884B28B
:1012B00014B1FFF709FFEAE7164B58690028E8D098
:1012C000FFF74EFF0020E4E70020DEE70020E9E71B
:1012D0001148B2E711481249A6F110020F2ED8BFEB
:1012E0000146104801F0A3FBECE770BD00ED00E003
:1012F000A6ED05013B3900005B3900008039000094
:1013000098390000BA39000028ED00E029ED00E02E
:101310002AED00E0D0ED00E0DA3900000D390000E0
:1013200022390000113A0000024A536943F01003C9
:101330005361704700ED00E043B2002B08DB01224F
:1013400000F01F0002FA00F0024A5B0942F8230095
:10135000704700BF00E100E043B2002B0DDB01222B
:1013600000F01F0002FA00F05B09044A203342F843
:101370002300BFF34F8FBFF36F8F704700E100E092
:1013800043B2002B01F10101A8BF03F160434FEA12
:101390004111B8BF054BC9B2ABBF03F5614300F0C3
:1013A0000F0083F800131954704700BF14ED00E0DC
:1013B0002DE9F0418C18884617461E4604220A9BE8
:1013C0000999054601F06BFD00220D49A4F12003A7
:1013D00023F0070321F00101C5E91322C5E91687AF
:1013E000996106991E605960079999600899D960BA
:1013F0004FF08071D961AB646A66BDE8F08100BFCF
:1014000043270000014910220A60704710ED00E0F8
:10141000404080F3118830BF704700BF404080F3E8
:1014200011884FF004007146014202D0EFF30980A9
:1014300001D1EFF30880714601B5FFF7DBFE01BD76
:1014400038B504460D4605281AD8DFE800F0031920
:10145000191315170D4801F0EAFA00F045FFAA69C3
:1014600001460B4801F0E3FA29462046BDE8384022
:1014700000F018B80748EEE70748ECE70748EAE746
:101480000146074801F0D3FAE7E700BF253A00001C
:10149000C33A0000453A00006B3A0000853A00006C
:1014A000A03A0000052810B50CD000F023FF60B171
:1014B00000F020FF0C490D4B002808BF19460C48CE
:1014C00001F0B5FAFFF7A4FFFCE700F023FF0028C6
:1014D000EED1084C0848A16801F0A9FAA068BDE85F
:1014E000104000F00BB800BFFF3A0000033B0000C3
:1014F000143B000018010020343B000038B50546BD
:101500004FF02003EFF3118483F31188BFF36F8F43
:1015100001F0A6FC0A4B9B68AB420BD1094B5A6801
:10152000C2F3080212B92046FFF7DEFC5A6842F007
:1015300080525A602046BDE8384001F038BC00BFF8
:101540001801002000ED00E001B572B60B4A106AE8
:1015500000281EBF0021116201F0F7FB62B6EFF315
:101560000580A0F110004FEAC0000549014409C9F7
:101570009847BDE8014003480047000018010020DB
:10158000382F0000B50E000001F0D2FA00F004F888
:1015900030BFFFF7FDBF00BF08B50E4B83F30988CE
:1015A000EFF3148343F0020383F31488BFF36F8FC8
:1015B000094B0A4A23F07F039360BFF34F8FBFF3B9
:1015C0006F8F00F027FC00F02FFCFFF781FC00F08C
:1015D00059FC00BFA00E00200000000000ED00E05C
:1015E00010B50E4B88B002930D4B0E4C03930E4B6F
:1015F00008A8049302AB40F81C3D0C4A2346012185
:1016000000F044F900230793094B0121E41A05A8CF
:101610000593069400F044F908B010BD00000020C6
:101620000000000000000120060001000000002072
:101630000000002010B50B680C7A23F01F0304F0A3
:101640001F021A43CB68640923F01F03044943F0C7
:10165000010343EA44038860CA600B6110BD00BF08
:1016600090ED00E030B585B09DF808200D890B683D
:101670004C68498965F3040261F3471200938DF8C1
:10168000082023F01F03621E134423F01F0303935B
:10169000084B04461B68C3F30723013B984205DC53
:1016A0006946FFF7C7FF204605B030BD6FF015044F
:1016B000F9E700BF90ED00E02DE9F04F06460F4638
:1016C00014460025DFF8488185B0BD420BDA56F894
:1016D0002530D3F80490B9F1000F3CD0B9F11F0FB9
:1016E00005D86FF01504204605B0BDE8F08F19F05D
:1016F0001F0FF6D1D3F800A01AF01F0FF1D15046FA
:1017000000F0A7FF834609EB0A00013800F0A1FFB3
:101710008345E6D11BF1160FE3D0631E5B45E0DB8A
:10172000C8F808B0D8F80C00C8F808B0D8F81030DD
:1017300056F8251020F01F0043F01F09D1E90032B0
:101740001A44984202F1FF3A1AD1D14505D15FFA05
:101750008BF0FFF787FF0135B7E7C8F808B0D8F876
:101760000C3022F01F0203F01F031A43C8F80C20AC
:10177000E0B2FFF777FF10F1160FB2D0441CEAE792
:10178000C8F808B0D8F81020013B23F01F0302F07E
:101790001F021343D145E0B2C8F81030E9D0FFF77B
:1017A00061FF10F1160F9CD0C8F808B0D8F80C20D3
:1017B0009DF80830441C62F304038DF80830D8F813
:1017C00010309DF808205B0863F3471256F8253067
:1017D0008DF80820D3E900231A44009209F1FF3361
:1017E00022F01F021344A3EB0A0323F01F03039309
:1017F000D8F80030E4B2C3F30723013BA342FFF65D
:1018000070AF20466946FFF715FF0134A3E700BF1C
:1018100090ED00E00522034B5A60BFF34F8FBFF3FA
:101820006F8F704790ED00E0BFF35F8F0022014B98
:101830005A60704790ED00E0104970B5104D0A688D
:101840002E68C2F30722964214D8FFF7EDFF00245A
:101850000C4B0B63A64205D10B4B1E70FFF7DAFF52
:10186000002070BD6968204601EB0411FFF7E2FE1D
:101870000134EFE74FF0FF30F3E700BF90ED00E0F9
:1018800094310000AAFF44005B01002010B5034C16
:101890002278FFF711FF207010BD00BF5B01002010
:1018A0002DE9F74F894607460026DFF89080DFF8DC
:1018B00090A0214C4E4519DAD7F804B0BBF1000FC7
:1018C00036D03B681846019300F0C3FE019B0546E5
:1018D0000BEB0300013800F0BCFE1423854203FB30
:1018E00006F306D06FF0150248F8032003B0BDE8F8
:1018F000F08F15F1160F48F80350F7D09AF8002032
:10190000AA42F3DDA5604344A560E068197B60F35B
:10191000040119732169187B490861F34710187392
:10192000E26822F01F025A60226922F01F021A6147
:1019300001360C37BEE700BF90ED00E00C00002040
:101940005B01002070B50E4B0E461C78002223462A
:1019500005460C480168C1F307218B420BDB0A4B9B
:10196000191D1868FFF766FE224631462846BDE875
:101970007040FFF7A1BE836002610133EAE700BF58
:101980005B01002090ED00E00C000020074B03EB12
:101990008000D0F8003223F44033C0F80032D0F891
:1019A000003243EA0141C0F800127047002584501C
:1019B000F8B5036801F01F049B680D461B7949497F
:1019C00044EA43140023D1F804238668D2B203F515
:1019D000A27051F82000C0F30420844267D122FA9B
:1019E00003F0C00763D59A0002F1A04202F550420D
:1019F000D2F8100520F00100C2F81005012202FA09
:101A000003F3C1F8083320460021FFF7BFFFB06899
:101A1000E84010F0010049D0F068E84010F0010003
:101A200044D07069E84010F001024CD0B369EB403B
:101A3000DB0740D4336923FA05F2F36923FA05F58D
:101A400005F0010502F00103AB420CBF02250125A0
:101A50000021244E01F5A27356F8230010F0030074
:101A60002BD18B0003F1A04303F55047D7F8102585
:101A7000240222F4473222F44072C7F81025D7F826
:101A8000102504F4F85444EA054503F55143154381
:101A9000C7F810551860D7F8103543F00103C7F8A0
:101AA0001035012303FA01F1C6F80413F8BD013320
:101AB000082B8CD1A7E70325CAE701310829C9D132
:101AC0006FF01200F2E7F169336920464B4023FAC8
:101AD00005F515F0010F0CBF03210221FFF756FF9A
:101AE0001046E3E700D0005008B5094B1A786AB9F0
:101AF00001210D2019700521FFF742FC0D20FFF791
:101B00001BFC4FF00042034BC3F80423002008BD28
:101B10005C01002000D000502DE9F74F8046856819
:101B200003F47040B0F5804F1E4649D02CDCB0F570
:101B3000805F3DD0B0F5405F3ED060BB06F440779B
:101B4000B7F5807F3ED0A7F5007463426341012959
:101B500019BFD4B2A1464FF01F0900244FF0010B6A
:101B600006F0010C4FEA4C0747EA0C0747EA002051
:101B7000DFF8C8A040EA830706F00203A14523D29C
:101B8000002003B0BDE8F08FB0F5E04F16D005DCC3
:101B9000B0F5A04F0ED06FF01500F2E7B0F5404F52
:101BA00004D0B0F5504FF6D10720C7E70620C5E7AF
:101BB0000120C3E70320C1E70420BFE70520BDE7FC
:101BC0000220BBE70323C2E7D8F80020926811790E
:101BD00004F01F0242EA411280324AF82270A968DA
:101BE0000BFA04F2002B25D01143A9606969B006F5
:101BF0004CBF114391436961A96970064CBF114301
:101C00009143A961296970074CBF11439143296130
:101C1000E96930064CBF0A4321EA0202EA61214623
:101C200040460193FFF7C4FE0028AAD10134E4B274
:101C3000019BA3E721EA0201D7E700BF00258450FA
:101C40002DE9F843454E3568012D5BD12F464FF005
:101C50000009434A93681268DC69D2F80880D3E926
:101C600002120A40D3E90510014322EA0102D8F822
:101C700000101B6909695C404C4022EA040482BBE5
:101C80003260002301279C46364ED6F8042307FA1B
:101C900003F1114211D003F1A05202F5515292000A
:101CA0001168012909D103F5A27056F82000C2F885
:101CB00000C0C0F3042081400C430133082BE4D161
:101CC00014B3274FBB681968F1B10E688B681C42CA
:101CD00003D04B68224638469847AEB13146366845
:101CE000F4E73A420AD098F8043009F01F000021C6
:101CF00040EA4310FFF74AFE22EA070209F1010910
:101D00007F00BCE70024BCE7012D0DD10026144B59
:101D10009C681B689F68D4E902321A40D4E90531F7
:101D20000B4322EA03020AB9BDE8F883154212D038
:101D3000E169236997F804C04B40F34013F0010FA9
:101D400006F01F000CBF0321022140EA4C10FFF7F0
:101D50001DFE22EA050201366D00E4E77CD1005049
:101D6000F80E002000D0005070B50026084B53F844
:101D70002040013053F82050A54200D870BD2368A0
:101D800020465B68984700B166600C34F4E700BFFA
:101D900088330000104B70B505461E460F4C9C4220
:101DA00004D10E4CB44209D1002412E062681AB189
:101DB00022681268AA420CD00C34F0E763680BB9B1
:101DC0000C34EFE723682846196800F0C4FE0028A9
:101DD000F6D1204670BD00BF040F0020B00E0020D9
:101DE00008B50B4D4FF02002EFF3118382F31188F9
:101DF000BFF36F8F01F071F8012104460228D8BFAC
:101E0000084601F07AF82C62FFF702FBEAE700BF10
:101E1000180100200248034A0021121A00F0D5BE22
:101E2000000000206001002008B50648064A074966
:101E3000121A00F09DFEBDE80840054A0549064813
:101E400000F096BEA00E0020180F00206C3B000092
:101E5000000000006C3B00000000002008B50220DC
:101E6000FFF782FF0320FFF77FFF00F099FA00F0F1
:101E7000E9FB034A137B23F00103137308BD00BF82
:101E8000AC00002080B5414BA2B083F30888002449
:101E9000E0223F4B012783F82220DC771C765C761A
:101EA0009C76DC765A6A3B4E42F4E0225A625A6AC9
:101EB000394D42F400225A629C63DA6892B242F0D1
:101EC000BF6242F40832DA60FFF72EFAFFF79AFA9F
:101ED00007AB21466C22184600F077FEB060204622
:101EE0008DF82970FFF740FF3846FFF73DFF00F0FF
:101EF000EFF92A4B75624FF48062CDE90473CDE9A6
:101F00000244CDE90044264B2649284600F02EFA2B
:101F10006B7B344623F0040213F01B0F6A7304D169
:101F2000AB6913B9284600F001F91F4B0122059354
:101F30000F23CDE9033200231C4E4FF4A0721C493D
:101F40003046CDE9013300931A4B00F00FFA737B52
:101F5000E66023F004037373174BC4E90633FFF7FD
:101F60003FFB0D48A56000F0EEFD0D4B134A1846EF
:101F700082F3098863B64FF0000181F31188BFF343
:101F80006F8F00210022002300F0DBFBA00E002059
:101F900000ED00E018010020AC000020603B0000D4
:101FA0005D1E000060010020653B00004000002035
:101FB00060050020E11D00003001002060050020C8
:101FC000EFF305800D2809D828B1054B586880F437
:101FD0000060C0F3C02080F0010070470120FAE7E4
:101FE00000ED00E008B5FEF7C7FD054B054A1B688C
:101FF0000021184410611846BDE8084000F07DBF7C
:102000005001002018010020F8B50D464FF02003C4
:10201000EFF3118483F31188BFF36F8F4FF4004106
:10202000002700220B4E0C4BC1FB00671A613046A3
:102030004FF4A02200233946FEF784F8074B1860BE
:10204000074B1D60FFF7CEFF84F31188BFF36F8F3E
:10205000F8BD00BFFFFF0400180100205001002060
:102060004C0100204FF02003EFF3118183F311881E
:10207000BFF36F8F044B9A68D37B013BD37381F31B
:102080001188BFF36F8F704718010020094B03F1CF
:102090002802824205D19B688B4202D14B7BDB0632
:1020A00007D1D1E900231A600A6853600023C1E90F
:1020B000003370471801002038B50D4C024604F17A
:1020C000280000F08DFE054600B9E568A3684AB90E
:1020D0005A7BD20606D1AA6922B9DA897F2A01D9A8
:1020E000636238BD9D4201D0FFF77CFF6562F8E76F
:1020F0001801002010B54FF02003EFF3118483F393
:102100001188BFF36F8F084B01209A68D37B01338E
:10211000D373FFF7D1FF84F31188BFF36F8FBDE84E
:10212000104000F053BE00BF18010020F8B54FF07A
:102130002003EFF3118483F31188BFF36F8F164AE6
:10214000114651F8283F8B420CD05BB1D66A90F90A
:102150000E5093F90E70AF420BDCB34202D01B68F5
:10216000002BF6D1D36A01604360D36A1860D06255
:1021700005E05A68C0E900325A6810605860437B35
:1021800043F0400343730020FFF796FF84F3118868
:10219000BFF36F8FF8BD00BF18010020F8B50446EB
:1021A0004FF02003EFF3118683F31188BFF36F8F95
:1021B000194F014607F128052846FFF767FFBB6A5C
:1021C0003A46AB420CD05BB1F86A94F90E1093F921
:1021D0000E708F420BDC834202D01B68002BF6D1BD
:1021E000D36A25606360D36A1C60D46205E05968D5
:1021F000C4E9003159680C605C60637B906843F00F
:1022000040036373031B58425841FFF755FF86F3A1
:102210001188BFF36F8FF8BD180100201449154ACB
:1022200010B58B681468A34203D1BDE81040FFF7D6
:10223000D9BE00241460104A1268BAB1DA897F2A24
:1022400014D80E4A93F90E40126894420EDB0C4AE1
:10225000126893420AD09A6942B90A69824203DC41
:102260001846FFF79BFFE0E7121A0A6110BD00BF96
:102270001801002048010020500100204C010020DE
:10228000A033000038B504464FF02003EFF311856A
:1022900083F31188BFF36F8F437B5A0607D501463E
:1022A0000948FFF7F3FE637B23F040036373074B9A
:1022B0009868031B58425841FFF7FEFE85F31188CA
:1022C000BFF36F8F38BD00BF400100201801002010
:1022D0000021044B084603F12802C3E90A22FFF754
:1022E00093BE00BF18010020014B9868704700BFE3
:1022F00018010020EFF305800D2807D838B1044BF2
:10230000586880F40060C0F3C02070470120704717
:1023100000ED00E0024B9B68187B00F00100704765
:102320001801002010B502464FF02003EFF311848E
:1023300083F31188BFF36F8F437B590704D484F371
:102340001188BFF36F8F10BD23F00403437300F0B7
:102350007EFD10B11046FFF7E9FE2146BDE81040B2
:10236000014800F016BD00BF5D01002030B587B008
:102370000E9D044604950D9D03950C9D02950B9DA5
:1023800001950A9D0095FFF713F8044B9B6813B95C
:10239000236607B030BD1B6EFAE700BF18010020AE
:1023A0002DE9F04F284E294DB04687B0B54205F1D2
:1023B00030040FD3FFF756FE4FF400490027234C9B
:1023C000234EDFF890A0444521D307B0BDE8F04F7D
:1023D000FFF790BE54F8043C059354F8103C049366
:1023E00054F8143C039354F8183C029354F81C3CE2
:1023F000019354F8203C009354E90A2354E90C015A
:10240000FFF7B4FF54F8303CDD642546CEE7616A3F
:102410004B1C04D0256821B92846FFF783FF3034D0
:10242000D1E7B346BC46C9FB01BC4FF4A022002350
:1024300058466146FDF786FE5146421C05F11800DC
:1024400000F052F8EBE700BF040F0020040F00205B
:10245000FFFF0400ED2D0000034B1B680BB9FEF7D6
:102460008BBB0020704700BF54010020036840B1BF
:10247000084A5268904204D01BB19A6881680A44A5
:102480009A604268136003685A600023C0E9003311
:10249000704700BFA80E002038B5104B1B78002BEA
:1024A0000F4B18BF4FF0FF301C6808BF6FF00040A3
:1024B0009C420AD04CB1A568FFF7CEFF281A00282D
:1024C0000ADBA468FFF7C8FF201A064B1B6913B18B
:1024D0009842A8BF184638BD0020F6E75D010020ED
:1024E000A80E00201801002070B504461646C160F1
:1024F0004FF02003EFF3118583F31188BFF36F8F43
:10250000FFF7AAFF012EACBF80190130174BA06066
:102510001A689A4201D05E6832B95A6823606260D4
:102520005A6814605C600BE09068A168884216DD10
:10253000411A91605168C4E9002151680C605460EF
:102540001A689A4206D0944204D1FFF7A5FF0021F1
:10255000FEF7D8FA85F31188BFF36F8F70BD091AA3
:102560009642A160D9D01268D6E700BFA80E00201D
:102570002DE9F04B0446FFF751FE4FF02003EFF337
:10258000118583F31188BFF36F8F214F214EB84619
:10259000DFF884903460D9F8004032684C45D7E9C0
:1025A00000BC05D024B1A368934214DD9B1AA3603C
:1025B00000241BEB02004CEBE271C8E9000134601F
:1025C000FFF76AFF2146FEF79DFA85F31188BFF3F6
:1025D0006F8FBDE8F08B1BEB03004CEBE371D31A5C
:1025E00033600023C7E90001A3602046FFF73EFFE8
:1025F00085F31188BFF36F8FE36898474FF020038E
:10260000EFF3118583F31188BFF36F8FC3E700BF2A
:102610000000002054010020A80E002038B5074C0F
:10262000074DAC4201D3002038BD04F1140320460D
:10263000C4E9053300F03AF81C34F2E7040F002037
:10264000040F002008B5FEF74FFBBDE80840FEF779
:10265000DFBA40E800F313F4803FD8B208BF6FF050
:102660001500704770B50C254D43C66890F90B00F6
:1026700074198842A8BF21464FF0200492FBF4F45D
:10268000B8BF715902F01F0001EB8401196070BDE1
:1026900007B501ABFFF7E6FF0123019A03FA00F04B
:1026A00013680343136003B05DF804FB2DE9F8439E
:1026B0000446FF2200214FF00C0E43680589006894
:1026C0005D4394F80AC02844E2728C4505DC00257D
:1026D0002389AB4222DCBDE8F883B5FBF3F20EFBA5
:1026E00001F7D4F80C801F2A08EB0706C8BF1F3279
:1026F0004FEA930306F10409C8BF520903F103032B
:10270000C6E9019923F00303D4BFE17248F807003A
:1027100001F10101C8BF00EB8200D6E76268E368FF
:102720006A4320681E1D811886509A6820464A60B8
:102730009A68116099602A460021FFF7A9FF0135C8
:10274000C6E708B50446084611461A46A047FFF7F3
:10275000CBFDFEF7D3FE0020704770B50D46044652
:102760004520A04729465220A04729462346BDE8D8
:102770007040522018472DE9F04F4FF0000A0646EE
:102780000F464FF0FF39D04689B01C46531E0393C5
:10279000002505E06DB9252800F03D813946B04798
:1027A000039B13F8010F03930028F3D109B0BDE890
:1027B000F08F642862D019D839280AD8312851D22C
:1027C0002D283DD030283ED0252808D13946B047A5
:1027D000DEE7582800F0A880632800F0168139460B
:1027E0002520B047039B39461878F0E7702800F0A1
:1027F000918006D8692841D06C283CD06828CFD079
:10280000EDE775286DD017D87328E8D1256804F155
:10281000040B2B461C4614F8010B002840F0EC80FA
:10282000B8F1030F40F000815C1BA9EB0404002CFD
:1028300000F3E6805C46ABE7782875D07A28DEE7BF
:102840004FF00308ACE7B9F1000F0EDAB8F1000F52
:1028500000F0E780A0F13009B8F1000F08BF4FF099
:1028600002089DE7B9F1000FF4DB0A2303FB090915
:10287000A9F13009F0E70AF1010A91E7BAF1000F76
:1028800012D125680434002D05DA39462D20B047D1
:102890006D4209F1FF3943462A46CDF8009039468A
:1028A0003046FDF7BDFE73E7BAF1010FE9D04FF0F6
:1028B000000C4FF0FF3B073424F0070303F108043A
:1028C000D3E9002312F1004043F100018C4508BF19
:1028D000834504D239463046FFF73FFF58E7154697
:1028E000D1E7BAF1000F05D122680434CDF8009089
:1028F0004346D4E7BAF1010FF6D0073424F00703BA
:1029000003F10804D3E90023002B08BFB2F1004F04
:10291000ECD3DFE739463020B04739467820B0475E
:102920004FF008094FF00108BAF1010F27DC2368C6
:102930000434079300230493102200239346029348
:102940000693079B0BF1FF3B4FEA8B00C0F1200C75
:10295000A0F1200123FA00F0049B03FA0CFC40EAEA
:102960000C0023FA01F1084310F00F0013D1069B6D
:1029700013B9BBF1000F2ED14FF0300C11E007342A
:1029800024F007031A6803F108045B6807920493B4
:10299000D2E7059AD5E709288CBF4FF0570C4FF0C6
:1029A000300C394660440592B047029B06950133CE
:1029B0000293BBF1000FECD1B8F1030F7FF4E8AE46
:1029C000029BC3EB4905002D7FF7E2AE394620207C
:1029D000B047013DF7E7531E91450593E9DBB8F198
:1029E000010F03D139463020B047E2E7B8F1020FBA
:1029F000DFD139462020F7E73946B047234609E7BB
:102A000039462020B047013C11E72068251D394692
:102A1000B0472C46BCE6AA46A8464FF0FF39012530
:102A2000BEE64FF00108BBE65C460546B8E60FB4CB
:102A300007B504A951F8040B0191FDF73FFE03B05F
:102A40005DF804EB04B0704770474FF0502330B589
:102A5000D3F80851D3F80423D3F8004102F001025F
:102A6000D3F80413D3F8040115B10025C3F80851B5
:102A7000B4B14FF050230024C3F8004122B14FF00D
:102A800050230122C3F8082348B100224FF05023FD
:102A9000C3F804218A0702D50222C3F8082330BDF7
:102AA000002AF1D04FF05023D3F80C3403F0011377
:102AB000B3F1011FE8D1E2E708B5002201210520AA
:102AC000FEF75EFC0520FEF737FC002008BD7047CE
:102AD0007047FEF7A3BC43B2A9B1002B12DB012162
:102AE0005B099B0003F1604303F56143D3F8802247
:102AF00000F01F0001FA00F022EA0000C3F8800293
:102B0000D3F880327047002BFCDB01225B099B006D
:102B100003F1604303F56143D3F8801200F01F0016
:102B200002FA00F00843E9E701460068FEF788BCB6
:102B3000202383F31188704708B5FEF729FDBDE80F
:102B40000840FEF7B7B907B5002101A8FEF7FAFE65
:102B500003B05DF804FB0138013910F8013F11F8AA
:102B6000012F934202D1002BF7D11A46981A7047D1
:102B7000F0B581EA0004A50703460BD0013B0A44E7
:102B800091421DD1F0BD002AFCD011F8014B013A51
:102B900003F8014B9C07F6D10C461D1F8F183E1BF6
:102BA000032E08D86FF00305940805FB0422A40047
:102BB00023442144E2E754F8046B45F8046FEEE740
:102BC00011F8014B03F8014FDAE70346F0B5C9B23B
:102BD0009C070FD11D4641EA012444EA04449F1892
:102BE0007E1B032E0CD8940803EB840413449C42F0
:102BF00009D1F0BD002AFCD003F8011B013AE7E738
:102C000045F8044BECE704F8011BF0E710B5046845
:102C10008068A46801292468C06903D158406060B5
:102C2000002010BD00334FF0010118BF0123D04038
:102C300000F001009140834214BFA160E160EFE722
:102C400070B504688068A468C069256801296E6948
:102C50002C696D6880EA040084EA050404EA06042D
:102C600080EA04001CBFD04000F001001860002082
:102C700070BD836830B5186858B10024814213D103
:102C800008685CB95C681860A14200D158600020F7
:102C9000086072B9002030BD2846EFE72060586810
:102CA000814208BF5C60F2E705680446002DF3D15D
:102CB0003AB11A680A60586819600028EAD1596068
:102CC000E9E76FF01500E6E701292DE9F04118BFAB
:102CD000D4B2064612BF25461F2500244FF0010836
:102CE0008768AC4202D90020BDE8F081FB6808FA91
:102CF00004F223EA0203FB6021463046FEF758FE49
:102D00000028F1D10134E4B2EBE701292DE9F041CB
:102D100018BFD4B2064612BF25461F2500244FF027
:102D200001088768AC4202D90020BDE8F081FB6849
:102D300008FA04F21343FB6021463046FEF738FEE2
:102D40000028F2D10134E4B2ECE7FFF7C1BE437BC7
:102D5000DB0603BF8069B0FA80F0400900207047AD
:102D600038B504464FF02003EFF3118583F3118843
:102D7000BFF36F8F01468068FFF788F9637B23F00C
:102D80000203637385F31188BFF36F8F0023A36081
:102D900038BD08B5FFF714F920B1BDE80840084672
:102DA000FEF7A2B881F31188BFF36F8F08BD08B595
:102DB0000246FFF705F920B1BDE808401046FEF7CE
:102DC00093B882F31188BFF36F8F08BD4FF02003D3
:102DD000EFF3118083F31188BFF36F8FFFF7E7BF25
:102DE0000368984214BF18460020704750F8103C02
:102DF00070B50446A0F11805CBB14FF02003EFF3F6
:102E0000118683F31188BFF36F8F294650F8100C99
:102E1000FFF73CF914F80B3C23F0020304F80B3CD9
:102E200086F31188BFF36F8F002344F8103C14F829
:102E30000B3C284623F0140304F80B3CFFF787FFF4
:102E400020B12846BDE87040FFF770B970BD437BE4
:102E5000DB0603BF8069B0FA80F0400900207047AC
:102E6000036D10B5044603B198472046FFF7EFFF06
:102E700038B12046FFF706FA637B43F0080363731B
:102E800010BD637B9B0702D52046FFF769FFA3694E
:102E9000002BF1D004F1180000F009F8ECE70373FF
:102EA000002342738173C373C0E90633704710B5C2
:102EB0004FF02002EFF3118482F31188BFF36F8F7C
:102EC00003683BB1FFF7D2FA002084F31188BFF307
:102ED0006F8F10BD6FF01500F7E710B54FF02003AE
:102EE000EFF3118483F31188BFF36F8FFFF7D4FAE8
:102EF00084F31188BFF36F8F10BD70B504460E4682
:102F00004FF02003EFF3118583F31188BFF36F8F28
:102F1000FFF7C2FAA04205DD012803DD3146204655
:102F2000FDF7F0FD85F31188BFF36F8F70BD70471B
:102F3000B4D2FF7F0100000000000000D32A00008F
:102F400000000000D32A000000000000D32A000087
:102F500000000000D32A000000000000D32A000077
:102F6000000000004B2A000000000000D32A0000EF
:102F700000000000D32A000000000000D32A000057
:102F800000000000D32A000000000000D32A000047
:102F900000000000D32A000000000000D32A000037
:102FA00000000000411C000000000000D32A0000C7
:102FB00000000000D32A000000000000D32A000017
:102FC00000000000D32A000000000000D32A000007
:102FD00000000000D32A000000000000D32A0000F7
:102FE00000000000310A000000000000D32A0000A9
:102FF00000000000D32A000000000000D32A0000D7
:1030000000000000D32A000000000000D32A0000C6
:1030100000000000D32A000000000000D32A0000B6
:1030200000000000D32A000000000000D32A0000A6
:1030300000000000D32A000000000000D32A000096
:1030400000000000D32A000000000000D32A000086
:1030500000000000D32A000000000000D32A000076
:1030600000000000D32A000000000000D32A000066
:1030700000000000D32A000000000000D32A000056
:1030800000000000D32A000000000000D32A000046
:1030900000000000D32A000000000000D32A000036
:1030A00000000000D32A000000000000D32A000026
:1030B00000000000D32A000000000000D32A000016
:1030C00000000000D32A000000000000D32A000006
:1030D00000000000D32A000000000000D32A0000F6
:1030E00000000000D32A000000000000D32A0000E6
:1030F00000000000D32A000000000000D32A0000D6
:1031000000000000D32A000000000000D32A0000C5
:1031100000000000D32A000000000000D32A0000B5
:1031200000000000D32A000000000000D32A0000A5
:1031300000000000D32A000000000000D32A000095
:10314000D9330000DD06000000000000B3330000AA
:10315000B92A000000000000BD330000B92A0000B9
:1031600000000000C7330000810A000000000000DA
:10317000D93300003918000000000000593B00005E
:10318000E91A000080330000D93300001D2600003A
:1031900000000000020000009C3100000000000060
:1031A000A433000006000000E0FF0F000000002034
:1031B000AC33000021000000E0FF00200509000002
:1031C00000000000000000006D09000091080000F0
:1031D00000000000170100000701000007010000C7
:1031E00007010000070100000701000007010000BF
:1031F00007010000070100000701000007010000AF
:10320000070100000701000007010000070100009E
:10321000070100000701000007010000070100008E
:10322000070100000701000007010000070100007E
:10323000070100000701000007010000070100006E
:10324000070100000701000007010000070100005E
:103250000701000013350000420100001A3500008C
:103260000501000024350000150100002D35000087
:103270003901000036350000090100004135000029
:103280000A0000004C3500002A01000054350000FF
:103290003A0100005C3500002C010000643500009C
:1032A0001C0100006D3500001D0100007635000096
:1032B0000A010000803500000B0100008A35000083
:1032C0000F0100009535000010010000A03500003E
:1032D00011010000AB3500000E010000B535000003
:1032E0003101000017010000170100001701000064
:1032F000170100001701000017010000170100006E
:10330000170100000701000007010000070100008D
:10331000070100000701000007010000070100008D
:10332000070100000701000007010000070100007D
:10333000070100000701000007010000070100006D
:10334000070100000701000007010000070100005D
:10335000070100000701000007010000070100004D
:1033600007010000191B00000D2C0000412C00007B
:10337000732C00000B2D0000C92C00000000000081
:103380000025845000000000B00E0020EC0E00204C
:10339000F80E0020040F0020040F0020F5FFFFFFAF
:1033A00040000020464C4153485F30005352414D8D
:1033B0005F3000434C4F434B5F33324B00434C4F25
:1033C000434B5F31364D007379735F636C6F636B92
:1033D000005365637572650909004E6F6E2D536564
:1033E0006375726509004E6F6E2D53656375726566
:1033F00000466C61736820726567696F6E090944E5
:103400006F6D61696E09095065726D697373696FDB
:103410006E730A00253032752030782530357820DB
:103420003078253035782009002563005352414D0E
:1034300020726567696F6E0909446F6D61696E0975
:10344000095065726D697373696F6E730A00253078
:103450003275203078253035782030782530357831
:1034600009005065726970686572616C0909446F82
:103470006D61696E09095374617475730A002530B2
:103480003275202573090925730009534B49500AE9
:1034900000094552524F520A00094F4B0A0053503F
:1034A0004D3A204E5320696D61676520617420306C
:1034B0007825780A0053504D3A204E53204D5350F2
:1034C00020617420307825780A0053504D3A204E00
:1034D0005320726573657420766563746F72206122
:1034E0007420307825780A0053504D3A2070726568
:1034F0007061726520746F206A756D7020746F2022
:103500004E6F6E2D53656375726520696D616765D9
:103510002E0A004E52465F5030004E52465F434CDA
:103520004F434B004E52465F52544331004E524679
:103530005F4E564D43004E52465F55415254453101
:10354000004E52465F554152544532004E52465F3E
:10355000495043004E52465F564D43004E52465F1F
:10356000465055004E52465F45475531004E524633
:103570005F45475532004E52465F5457494D320021
:103580004E52465F5350494D33004E52465F5449A8
:103590004D455230004E52465F54494D4552310020
:1035A0004E52465F54494D455232004E52465F538B
:1035B00041414443004E52465F4750494F544531C4
:1035C000002A2A2A2A2A20425553204641554C5483
:1035D000202A2A2A2A2A0A002020537461636B6950
:1035E0006E67206572726F720A00202050726563E8
:1035F00069736520646174612062757320657272FD
:103600006F720A0020204246415220416464726574
:1036100073733A20307825780A002020496D707243
:1036200065636973652064617461206275732065E8
:1036300072726F720A002020496E7374727563741F
:10364000696F6E20627573206572726F720A002A4C
:103650002A2A2A2A204D5055204641554C54202ACA
:103660002A2A2A2A0A002020537461636B696E6734
:10367000206572726F722028636F6E746578742093
:1036800061726561206D69676874206265206E6F84
:10369000742076616C6964290A002020556E737469
:1036A00061636B696E67206572726F720A00202019
:1036B00044617461204163636573732056696F6C64
:1036C0006174696F6E0A0020204D4D4641522041C1
:1036D0006464726573733A20307825780A0020207C
:1036E000496E737472756374696F6E2041636365AC
:1036F00073732056696F6C6174696F6E0A002020C5
:10370000466C6F6174696E672D706F696E74206CA2
:10371000617A792073746174652070726573657263
:10372000766174696F6E206572726F720A002A2A60
:103730002A2A2A20534543555245204641554C5488
:10374000202A2A2A2A2A0A002020416464726573EA
:10375000733A20307825780A002020496E76616C13
:10376000696420656E74727920706F696E740A00E6
:103770002020496E76616C696420696E7465677299
:10378000697479207369676E61747572650A0020C7
:1037900020496E76616C6964206578636570746930
:1037A0006F6E2072657475726E0A00202041747409
:1037B0007269627574696F6E20756E6974207669BE
:1037C0006F6C6174696F6E0A002020496E76616CBF
:1037D0006964207472616E736974696F6E0A002087
:1037E000204C617A792073746174652070726573FE
:1037F0006572766174696F6E0A0020204C617A7977
:10380000207374617465206572726F720A002A2ACF
:103810002A2A2A205553414745204641554C5420D9
:103820002A2A2A2A2A0A0020204469766973696FA5
:103830006E206279207A65726F0A002020556E61D1
:103840006C69676E6564206D656D6F727920616368
:10385000636573730A002020537461636B206F7675
:103860006572666C6F772028636F6E74657874205C
:1038700061726561206E6F742076616C6964290ADB
:103880000020204E6F20636F70726F636573736FDB
:103890007220696E737472756374696F6E730A0057
:1038A0002020496C6C6567616C206C6F6164206FCF
:1038B00066204558435F52455455524E20696E74F8
:1038C0006F2050430A002020496C6C6567616C20B2
:1038D000757365206F662074686520455053520AE1
:1038E000002020417474656D707420746F206578B9
:1038F000656375746520756E646566696E656420C0
:10390000696E737472756374696F6E0A00526573C1
:10391000657276656420457863657074696F6E20A2
:10392000280053707572696F757320696E746572C3
:10393000727570742028495251200020205320694C
:103940006E737472756374696F6E206164647265FE
:1039500073733A2020307825780A00524554544F2A
:103960004241534520646F6573206E6F74206D6112
:10397000746368204558435F52455455524E0A00BF
:103980002A2A2A2A2A2048415244204641554C548A
:10399000202A2A2A2A2A0A002020427573206661DA
:1039A000756C74206F6E20766563746F722074611D
:1039B000626C6520726561640A0020204661756C46
:1039C0007420657363616C6174696F6E2028736520
:1039D000652062656C6F77290A002A2A2A2A2A2024
:1039E0004465627567206D6F6E69746F72206578CB
:1039F00063657074696F6E20286E6F7420696D70D6
:103A00006C656D656E74656429202A2A2A2A2A0A43
:103A1000002A2A2A2A2A20257320256429202A2AD6
:103A20002A2A2A0A002A2A2A2A2A20486172647726
:103A300061726520657863657074696F6E202A2AEB
:103A40002A2A2A0A002A2A2A2A204B65726E656CC5
:103A500020416C6C6F636174696F6E204661696CA4
:103A600075726521202A2A2A2A0A002A2A2A2A2A45
:103A7000204B65726E656C204F4F505321202A2ACF
:103A80002A2A2A0A002A2A2A2A2A204B65726E65C7
:103A90006C2050616E696321202A2A2A2A2A0A0092
:103AA0002A2A2A2A20556E6B6E6F776E2046617423
:103AB000616C204572726F7220256421202A2A2AA7
:103AC0002A0A0043757272656E74207468726561AB
:103AD00064204944203D2025700A4661756C746954
:103AE0006E6720696E737472756374696F6E20619E
:103AF000646472657373203D20307825780A00492C
:103B0000535200657373656E7469616C20746872DA
:103B100065616400466174616C206661756C742037
:103B2000696E20257321205370696E6E696E672E51
:103B30002E2E0A00466174616C206661756C7420DB
:103B4000696E20746872656164202570212041626D
:103B50006F7274696E672E0A004750494F5F3000DC
:103B60006D61696E0069646C650000005727000094
:103B70000090D003A80E0020A80E002040310000C5
:103B8000000000000000000088310000000000007C
:103B90000000000070310000000000000000000084
:103BA0004C310000BC310000000000005831000022
:103BB000C831000000000000643100000000000077
:103BC000000000007C310000643300002000002071
:103BD000040F0020040F002000000000000000007F
:043BE0000F000000D2
:10800000F031022021A00000EBA50100B59E000088
:10801000B59E0000B59E0000B59E0000B59E000014
:10802000B59E0000B59E0000B59E0000D19A0000EC
:10803000B59E0000B59E0000799A0000D1A5010010
:10804000E19F0000E19F0000E19F0000E19F000030
:10805000E19F0000E19F0000E19F0000E19F000020
:10806000E19F0000E19F0000E19F0000E19F000010
:10807000E19F0000E19F0000E19F0000E19F000000
:10808000E19F0000E19F0000E19F0000E19F0000F0
:10809000E19F0000E19F0000E19F0000E19F0000E0
:1080A000E19F0000E19F0000E19F0000E19F0000D0
:1080B000C9AC0000FFA90100E19F0000E19F0000A2
:1080C000E19F0000E19F0000E19F0000E19F0000B0
:1080D000E19F0000E19F0000E19F0000E19F0000A0
:1080E000E19F0000E19F000021AA0100E19F000044
:1080F000E19F0000E19F0000E19F0000E19F000080
:10810000E19F0000E19F0000E19F0000E19F00006F
:10811000E19F0000E19F0000E19F0000E19F00005F
:10812000E19F0000E19F0000E19F0000E19F00004F
:10813000E19F0000E19F0000E19F0000E19F00003F
:10814000E19F00007BB972B90029BEBF00204FF04B
:10815000004106E008BF00281CBF6FF000414FF04F
:10816000FF3000F0C7B9ADF1080C6DE904CE00296D
:1081700009DB002B1ADB00F04DF8DDF804E0DDE947
:10818000022304B07047404261EB4101002B1BDB2E
:1081900000F040F8DDF804E0DDE9022304B04042DD
:1081A00061EB4101524263EB43037047524263EB80
:1081B000430300F02FF8DDF804E0DDE9022304B00A
:1081C000404261EB41017047524263EB430300F0D0
:1081D00021F8DDF804E0DDE9022304B0524263EB4C
:1081E0004303704753B94AB9002908BF00281CBF90
:1081F0004FF0FF314FF0FF3000F07CB9ADF1080CCB
:108200006DE904CE00F006F8DDF804E0DDE90223B4
:1082100004B070472DE9F0478C46089D04468A4615
:10822000002B4AD18A42174662D9B2FA82F64EB181
:10823000C6F1200E01FA06F3B740B44020FA0EFE54
:108240004EEA030A4FEA1748230C1FFA87F9BAFBD4
:10825000F8FE08FB1EAA0EFB09F243EA0A439A4203
:108260000BD9FB180EF1FF312CBF012000209A42E0
:1082700002D9002800F02A818E469A1AA3B2B2FBD6
:10828000F8F008FB102200FB09F943EA0244A1457B
:1082900007D93C1900F1FF3302D2A14500F2108149
:1082A0001846A4EB090440EA0E4000211DB1F44039
:1082B0000023C5E90043BDE8F0878B4208D9002DB3
:1082C00000F0F2800021C5E9000C0846BDE8F08707
:1082D000B3FA83F100294ED16345C0F0E8808242B1
:1082E00040F2E5800846002DE5D0C5E9004AE2E706
:1082F00002B9FFDEB2FA82F6002E40F099808B1AA6
:108300004FEA124E1FFA82F801214FEA144CB3FBD8
:10831000FEF20EFB123008FB02F94CEA004CE1457C
:1083200008D917EB0C0C02F1FF3302D2E14500F241
:10833000CA801A46ACEB090CA3B2BCFBFEF00EFBE4
:1083400010CC08FB00F843EA0C44A0450ED93C19B8
:1083500000F1FF332CBF4FF0010C4FF0000CA04593
:1083600003D9BCF1000F00F0A8801846A4EB080464
:1083700040EA02409AE7C1F120048B4002FA01FE74
:108380000CFA01F6E24020FA04F72CFA04FC00FA99
:1083900001F813433E431F0C320C1FFA83F9BCFB58
:1083A000F7F007FB10CC00FB09FA42EA0C4CE2455F
:1083B00008D913EB0C0C00F1FF3202D2E24500F2B7
:1083C00089801046ACEB0A0CB6B2BCFBF7FA07FB8F
:1083D0001ACC0AFB09F946EA0C42914506D99A18CB
:1083E0000AF1FF3601D291457AD8B2464AEA0040F6
:1083F000A2EB0902A0FB0E67BA42B446B94602D30B
:1084000007D1B04505D2B6EB0E0C67EB030301387C
:108410009946002D6BD0B8EB0C0362EB090202FA0F
:1084200004F4CB40CA4000211C43C5E9004242E7A6
:10843000B740C6F1200201FA06F3B44021FA02FC6B
:108440004FEA174E20FA02F21FFA87F8BCFBFEF142
:108450001A430EFB11CC01FB08F0130C43EA0C4C41
:10846000604507D917EB0C0C01F1FF3301D26045D1
:1084700033D81946ACEB000C92B2BCFBFEF00EFBFD
:1084800010CC00FB08F342EA0C4C634507D917EB0C
:108490000C0C00F1FF3201D2634525D81046ACEB3D
:1084A000030340EA014130E72946284603E7841ADE
:1084B0006CEB030301209A4615E702383C4455E76C
:1084C00002383C44EDE6023ABC4433E7AEF1020E1A
:1084D0003B44D2E602389C4474E70239BC44C9E705
:1084E000AAF1020A1A4481E70238BC44D7E72946B8
:1084F000E1E600BF704700BF70B491E87800B2E8D1
:1085000002105B1854EB0C04B2E802104D4156EB1C
:108510000C0680E878008041013070BC704770B470
:1085200091E87800B2E802105B1A74EB0C04B2E830
:1085300002108D4176EB0C0680E8780080414042C5
:1085400070BC70472DE9F00791E8F807B2E8021017
:108550005B1854EB0C04B2E802104D4156EB0C06CC
:10856000B2E802104F4158EB0C08B2E8021059EB88
:1085700001095AEB0C0A80E8F80780410130BDE898
:10858000F00770472DE9F00791E8F807B2E802100C
:108590005B1A74EB0C04B2E802108D4176EB0C060A
:1085A000B2E802108F4178EB0C08B2E8021079EBC8
:1085B00001097AEB0C0A80E8F80780414042BDE8E7
:1085C000F00770472DE9F007524290E87800B1E8D3
:1085D00080071740DB1918EA020854EB080419EA6F
:1085E000020955EB09051AEA020A56EB0A0678C099
:1085F00090E87800B1E8800717407B4118EA02084C
:1086000054EB080419EA020955EB09051AEA020AB3
:1086100056EB0A0678C080410130BDE8F00770478C
:108620002DE9F007524290E87800B1E88007174042
:10863000DB1B18EA020874EB080419EA020975EB5F
:1086400009051AEA020A76EB0A0678C090E8780073
:10865000B1E880071740BB4118EA020874EB080430
:1086600019EA020975EB09051AEA020A76EB0A060D
:1086700078C080414042BDE8F007704790E8300084
:1086800091E8C000A31B1340E41AF618EB1B13403B
:10869000ED1AFF1830C0C0C17047F0B55242FFF765
:1086A000EDFFFFF7EBFFFFF7E9FFFFF7E7FFF0BD97
:1086B0002DE9F0073AC91668A1FB069A4FF0000CA5
:1086C000E3FB06AC4FF00007E4FB06C74FF00008E1
:1086D000E5FB067840F8049B56684FF00009E1FB83
:1086E00006A91CEB090C4FF0000949EB0909E3FB53
:1086F00006C917EB09074FF0000949EB0909E4FB2C
:10870000067918EB09084FF0000949EB0909E5FB68
:10871000068940F804AB96684FF0000AE1FB06CAF0
:1087200017EB0A074FF0000A4AEB0A0AE3FB067A46
:1087300018EB0A084FF0000A4AEB0A0AE4FB068A23
:1087400019EB0A094FF0000A4AEB0A0AE5FB069A00
:1087500040F804CBD6684FF0000CE1FB067C18EB28
:108760000C084FF0000C4CEB0C0CE3FB068C19EBE7
:108770000C094FF0000C4CEB0C0CE4FB069C1AEBC4
:108780000C0A4FF0000C4CEB0C0CE5FB06AC80E83F
:108790008017BDE8F00770470A462DE9F04F41EC1D
:1087A000140A92EC080A1EC910EE100AA1FB007808
:1087B0004FF00009E2FB00894FF0000AE3FB009A4A
:1087C0004FF0000BE4FB00AB12EE100A4FF0000C70
:1087D000E1FB00BC4FF0000EE2FB00CE4FF00005C5
:1087E000E3FB00E54FF00006E4FB005605EE107ACF
:1087F00010EE900A4FF00007E1FB008719EB070924
:108800004FF0000747EB0707E2FB00971AEB070A58
:108810004FF0000747EB0707E3FB00A71BEB070B35
:108820004FF0000747EB0707E4FB00B712EE900A92
:108830001CEB070C4FF0000747EB0707E1FB00C7F5
:108840001EEB070E4FF0000747EB0707E2FB00E7C0
:10885000ED194FF0000747EB0707E3FB0057F61948
:108860004FF0000747EB0707E4FB006705EE908A2F
:1088700011EE100A4FF00008E1FB00981AEB080A0D
:108880004FF0000848EB0808E2FB00A81BEB080BC0
:108890004FF0000848EB0808E3FB00B81CEB080C9D
:1088A0004FF0000848EB0808E4FB00C813EE100A7C
:1088B0001EEB080E4FF0000848EB0808E1FB00E84B
:1088C00015EB08054FF0000848EB0808E2FB0058DC
:1088D00016EB08064FF0000848EB0808E3FB0068B9
:1088E00017EB08074FF0000848EB0808E4FB007896
:1088F00006EE109A11EE900A4FF00009E1FB00A974
:108900001BEB090B4FF0000949EB0909E2FB00B929
:108910001CEB090C4FF0000949EB0909E3FB00C906
:108920001EEB090E4FF0000949EB0909E4FB00E9D1
:1089300013EE900A15EB09054FF0000949EB090900
:10894000E1FB005916EB09064FF0000949EB090954
:10895000E2FB006917EB09074FF0000949EB090931
:10896000E3FB007918EB09084FF0000949EB09090E
:10897000E4FB008906EE90AA14EE901A01F11001B2
:108980001EC910EE100A4FF0000AE1FB00BA1CEB02
:108990000A0C4FF0000A4AEB0A0AE2FB00CA1EEB7F
:1089A0000A0E4FF0000A4AEB0A0AE3FB00EA15EB55
:1089B0000A054FF0000A4AEB0A0AE4FB005A12EEDD
:1089C000100A16EB0A064FF0000A4AEB0A0AE1FB0E
:1089D000006A17EB0A074FF0000A4AEB0A0AE2FBAB
:1089E000007A18EB0A084FF0000A4AEB0A0AE3FB88
:1089F000008A19EB0A094FF0000A4AEB0A0AE4FB65
:108A0000009A07EE10BA10EE900A4FF0000BE1FB4F
:108A100000CB1EEB0B0E4FF0000B4BEB0B0BE2FBF6
:108A200000EB15EB0B054FF0000B4BEB0B0BE3FBD7
:108A3000005B16EB0B064FF0000B4BEB0B0BE4FB54
:108A4000006B12EE900A17EB0B074FF0000B4BEB8D
:108A50000B0BE1FB007B18EB0B084FF0000B4BEB13
:108A60000B0BE2FB008B19EB0B094FF0000B4BEBF0
:108A70000B0BE3FB009B1AEB0B0A4FF0000B4BEBCD
:108A80000B0BE4FB00AB07EE90CA11EE100A4FF09F
:108A9000000CE1FB00EC15EB0C054FF0000C4CEB6F
:108AA0000C0CE2FB005C16EB0C064FF0000C4CEBE0
:108AB0000C0CE3FB006C17EB0C074FF0000C4CEBBD
:108AC0000C0CE4FB007C13EE100A18EB0C084FF0C2
:108AD000000C4CEB0C0CE1FB008C19EB0C094FF07B
:108AE000000C4CEB0C0CE2FB009C1AEB0C0A4FF058
:108AF000000C4CEB0C0CE3FB00AC1BEB0C0B4FF035
:108B0000000C4CEB0C0CE4FB00BC08EE10EA11EE80
:108B1000900A4FF0000EE1FB005E16EB0E064FF0E0
:108B2000000E4EEB0E0EE2FB006E17EB0E074FF041
:108B3000000E4EEB0E0EE3FB007E18EB0E084FF01E
:108B4000000E4EEB0E0EE4FB008E13EE900A19EBB6
:108B50000E094FF0000E4EEB0E0EE1FB009E1AEBDD
:108B60000E0A4FF0000E4EEB0E0EE2FB00AE1BEBBA
:108B70000E0B4FF0000E4EEB0E0EE3FB00BE1CEB97
:108B80000E0C4FF0000E4EEB0E0EE4FB00CE14EE7A
:108B9000100AA0EC075A80E8E05FBDE8F08F00BF44
:108BA00030B44FF0000310F8014B11F8015B013AAB
:108BB00084EA050443EA0403F5D1A3F101034FEA73
:108BC000D37030BC70474FF0000310F8012B01390F
:108BD00043EA0203F9D1A3F101034FEAD3707047CE
:108BE00011F8013B00F8013B013AF9D1704700222E
:108BF00000F8012B0139FBD1704700BF2DE9F007C8
:108C000091E8F807B2E802105B1854EB0C04B2E8E4
:108C100002104D4156EB0C06B2E802104F4158EBE2
:108C20000C08B2E8021059EB01095AEB0C0A894111
:108C3000B3F1FF3374F1FF3475F1FF3576F10006BF
:108C400077F1000778F1000879F101097AF1FF3A2C
:108C500051F100014A425B184C414D4156F100066A
:108C600057F1000758F1000859EB02095AEB010AC5
:108C700080E8F807BDE8F00770472DE9F00791E8B4
:108C8000F807B2E802105B1A74EB0C04B2E80210A9
:108C90008D4176EB0C06B2E802108F4178EB0C08A0
:108CA000B2E8021079EB01097AEB0C0A89414A42D9
:108CB0005B184C414D4156F1000657F1000758F141
:108CC000000859EB02095AEB010A80E8F807BDE8F1
:108CD000F00770470A462DE9F04F41EC140A92EC78
:108CE000080A1EC910EE100AA1FB00784FF0000917
:108CF000E2FB00894FF0000AE3FB009A4FF0000B03
:108D0000E4FB00AB12EE100A4FF0000CE1FB00BCDC
:108D10004FF0000EE2FB00CE4FF00005E3FB00E554
:108D20004FF00006E4FB005605EE107A10EE900AB4
:108D30004FF00007E1FB008719EB07094FF0000730
:108D400047EB0707E2FB00971AEB070A4FF0000713
:108D500047EB0707E3FB00A71BEB070B4FF00007F0
:108D600047EB0707E4FB00B712EE900A1CEB070C79
:108D70004FF0000747EB0707E1FB00C71EEB070EAC
:108D80004FF0000747EB0707E2FB00E7ED194FF054
:108D9000000747EB0707E3FB0057F6194FF0000702
:108DA00047EB0707E4FB006705EE908A11EE100A17
:108DB0004FF00008E1FB00981AEB080A4FF000089A
:108DC00048EB0808E2FB00A81BEB080B4FF000087B
:108DD00048EB0808E3FB00B81CEB080C4FF0000858
:108DE00048EB0808E4FB00C813EE100A1EEB080E5F
:108DF0004FF0000848EB0808E1FB00E815EB080518
:108E00004FF0000848EB0808E2FB005816EB080694
:108E10004FF0000848EB0808E3FB006817EB080771
:108E20004FF0000848EB0808E4FB007806EE109AC3
:108E300011EE900A4FF00009E1FB00A91BEB090BB2
:108E40004FF0000949EB0909E2FB00B91CEB090CE2
:108E50004FF0000949EB0909E3FB00C91EEB090EBD
:108E60004FF0000949EB0909E4FB00E913EE900A11
:108E700015EB09054FF0000949EB0909E1FB005921
:108E800016EB09064FF0000949EB0909E2FB0069FE
:108E900017EB09074FF0000949EB0909E3FB0079DB
:108EA00018EB09084FF0000949EB0909E4FB0089B8
:108EB00006EE90AA14EE901A01F110011EC910EEF0
:108EC000100A4FF0000AE1FB00BA1CEB0A0C4FF04D
:108ED000000A4AEB0A0AE2FB00CA1EEB0A0E4FF038
:108EE000000A4AEB0A0AE3FB00EA15EB0A054FF019
:108EF000000A4AEB0A0AE4FB005A12EE100A16EBCB
:108F00000A064FF0000A4AEB0A0AE1FB006A17EB77
:108F10000A074FF0000A4AEB0A0AE2FB007A18EB54
:108F20000A084FF0000A4AEB0A0AE3FB008A19EB31
:108F30000A094FF0000A4AEB0A0AE4FB009A07EE1E
:108F400010BA10EE900A4FF0000BE1FB00CB1EEBC5
:108F50000B0E4FF0000B4BEB0B0BE2FB00EB15EB9A
:108F60000B054FF0000B4BEB0B0BE3FB005B16EB21
:108F70000B064FF0000B4BEB0B0BE4FB006B12EE00
:108F8000900A17EB0B074FF0000B4BEB0B0BE1FBC1
:108F9000007B18EB0B084FF0000B4BEB0B0BE2FBCD
:108FA000008B19EB0B094FF0000B4BEB0B0BE3FBAA
:108FB000009B1AEB0B0A4FF0000B4BEB0B0BE4FB87
:108FC00000AB07EE90CA11EE100A4FF0000CE1FB67
:108FD00000EC15EB0C054FF0000C4CEB0C0CE2FB1D
:108FE000005C16EB0C064FF0000C4CEB0C0CE3FB9A
:108FF000006C17EB0C074FF0000C4CEB0C0CE4FB77
:10900000007C13EE100A18EB0C084FF0000C4CEB30
:109010000C0CE1FB008C19EB0C094FF0000C4CEB35
:109020000C0CE2FB009C1AEB0C0A4FF0000C4CEB12
:109030000C0CE3FB00AC1BEB0C0B4FF0000C4CEBEF
:109040000C0CE4FB00BC08EE10EA11EE900A4FF0A5
:10905000000EE1FB005E16EB0E064FF0000E4EEB2D
:109060000E0EE2FB006E17EB0E074FF0000E4EEBFC
:109070000E0EE3FB007E18EB0E084FF0000E4EEBD9
:109080000E0EE4FB008E13EE900A19EB0E094FF062
:10909000000E4EEB0E0EE1FB009E1AEB0E0A4FF097
:1090A000000E4EEB0E0EE2FB00AE1BEB0E0B4FF074
:1090B000000E4EEB0E0EE3FB00BE1CEB0E0C4FF051
:1090C000000E4EEB0E0EE4FB00CE53EC172A18EE0A
:1090D000104A12EB0A0253EB0B0354EB0C0455EB52
:1090E0000E05002040F1000012EB0B0253EB0C03C5
:1090F00054EB0E0455EB0E0546410020474158EB5A
:10910000000859EB0A0940F10000B2EB0E0273F1BE
:10911000000374F1000475EB0A0576EB0B0677EBA0
:109120000C0778EB0A0879EB0C0960F10000B5EB4D
:109130000B0576EB0C0677EB0E0778EB0B0879EB5B
:109140000E0960F100005FEAE07C7FEA0C0CDCF1C4
:10915000000EB2EB0C0273EB0C0374EB0C0475F114
:10916000000576F1000677F1000778EB0E0879EB41
:109170000C0960F100005FEAE07CDCF1000E12EB0C
:109180000C0253EB0C0354EB0C0455F1000556F1A3
:10919000000657F1000758EB0E0859EB0C0940F197
:1091A00000005FEAE07CDCF1000E12EB0C0253EBF6
:1091B0000C0354EB0C0455F1000556F1000657F171
:1091C000000758EB0E0859EB0C095BEC15AA51ECA3
:1091D000160A1AEB060A5BEB070B50EB080051EB83
:1091E00009015FF0000C4CF1000C1AEB070A5BEB75
:1091F000080B50EB090051EB090152EB0C025FF038
:10920000000C53EB0C0354EB0C0475414CF1000CB7
:10921000BAEB090A7BF1000B70F10000B141BA41D1
:1092200073EB0803B44175EB08056CF1000CC91B26
:1092300072EB080273EB0903BC4175EB09056CF195
:10924000000C5FEAEC787FEA0808D8F10009BAEB75
:10925000080A7BEB080B70EB080071F1000172F15A
:10926000000273F1000374EB090475EB08056CF15F
:10927000000C5FEAEC78D8F100091AEB080A5BEB06
:10928000080B50EB080051F1000152F1000253F1BC
:10929000000354EB090455EB08054CF1000C5FEAA0
:1092A000EC78D8F100091AEB080A5BEB080B50EBDD
:1092B000080051F1000152F1000253F1000354EB98
:1092C000090455EB080514EE107AA7E8000C87E8AE
:1092D0003F00BDE8F08F00BF0A22074B196801313B
:1092E0001960B1FBF2F302FB131313B90122034B14
:1092F0001A70034811F053B908000220C22002205E
:109300008CE201002DE9F347054688460B9F0D4E80
:109310000FFA83F90FFA82FA0A9A336800920197DA
:109320009C6A52464B4641462846A047041E04DA32
:1093300001F0F2FE03680B2BEED0204602B0BDE830
:10934000F08700BF0C000220312313B530221946EC
:109350000D4811F024F9302331221946CDE90023BC
:109360000A4811F01CF9012001F07CFE041E09DA04
:1093700001F0D2FE21460268054802B0BDE8104067
:1093800011F00DB902B010BD88E301009AE30100AD
:10939000B4E30100182300222DE9F043474D93B0B8
:1093A00003932B6811465C6B454802ABA047011E36
:1093B00005DA444811F0F3F813B0BDE8F0834FF438
:1093C000F64201200024029B02215B695A80CDE90C
:1093D00004042B6822461B689847071E0BDA39469F
:1093E000394811F0DCF8394811F0D9F82B683846C3
:1093F0005B689847E0E72B680822DB6804A9984778
:10940000061E07DA01F088FE31460268304811F086
:10941000C6F8E8E72B6802995B6908224969384673
:109420009847061E05DA01F077FE314602682948A2
:10943000EDE73022214606A811F022FAE3238DF849
:1094400018302B683022DE6A06A923463846B0471A
:1094500006460146204811F0A2F8002E05DA01F078
:109460005BFE314602681D48D1E703AB0193029BC6
:109470004FF480625B691A49009338462346FFF730
:1094800041FF061E05DA01F047FE31460268154825
:10949000BDE7154811F083F8DFF84480DFF85090FD
:1094A000B44203D1114811F07AF89CE718F804107F
:1094B000484611F074F80134F2E700BF0C000220B6
:1094C0009EE20100AAE20100C0E2010062E30100A5
:1094D000D0E20100E9E2010005E3010016E301002A
:1094E000C21C022031E301004EE30100E0E501006F
:1094F0005EE301004EF660220148114602F096BC80
:10950000FC50022008B50D4811F049F8FFF742FF62
:10951000FFF71AFFFFF7EEFF094C0A4D41F28830C2
:1095200002F00AFA2378002BF8D0284611F037F819
:1095300000232370FFF72EFFF0E700BF6CE301006C
:10954000C22002207FE301000B6801330B60014B56
:109550001B681847505002202DE9F04F85B00E9C33
:109560009B46012CB8BF0124012B0CBF30232023C4
:1095700015468046894601260A270022DFF870A09A
:10958000019402930AF101040AB9AA451ED2B5FB5F
:10959000F4F049463030C04701220136B5FBF4F102
:1095A0000A23013F012F04FB1155BAFBF3FAE9D15D
:1095B000494605F13000C047BBF1030F03D1019BC1
:1095C0009C1B002C0FDC05B0BDE8F08F019BBB425B
:1095D000E4DBBBF1020FE1D8494602980392013661
:1095E000C047039ADAE749462020C047013CE8E734
:1095F000FFC99A3B002313B502AC44F8043D024670
:109600000B460348214610F06EFE02B010BD00BFAD
:109610004995000010B54FF02003EFF3118483F358
:109620001188BFF36F8F00F013F80122064BC3F8C7
:1096300040254FF0FF32054B9A62DA6284F31188BD
:10964000BFF36F8F002010BD0090034000ED00E0DD
:10965000074AD2F8883043F47003C2F88830BFF369
:109660004F8FBFF36F8F034B034A1A60704700BFE1
:1096700000ED00E0545002200090D003014B186030
:10968000704700BF0C00022010B54FF02003EFF32D
:10969000118283F31188BFF36F8F154C237833B990
:1096A00082F31188BFF36F8F6FF0440010BD013B50
:1096B000DBB2237033B182F31188BFF36F8F6FF089
:1096C0000F00F3E70B4B0121187838B1217082F3BA
:1096D0001188BFF36F8F6FF00A00E7E7197082F30C
:1096E0001188BFF36F8F044A11601870DEE700BF66
:1096F000C5200220C42002200450004010B54FF0C5
:109700002002EFF3118382F31188BFF36F8F134CA4
:10971000207890B183F31188BFF36F8F104AD2F88D
:109720001C34D2F8182403F0030343F4803393432A
:1097300014BF6FF04300002010BD0122227083F39C
:109740001188BFF36F8F064BC3F80401C3F81815D7
:109750000221C3F804139A60E0E700BFC32002208F
:1097600000500040174B30B5D3F80851D3F804230C
:10977000D3F8004102F00102D3F80413D3F8040136
:1097800015B10025C3F8085194B10024C3F8004175
:109790001AB101220B4BC3F8082340B10022094B38
:1097A000C3F804218A0702D50222C3F8082330BD7A
:1097B000002AF2D0D3F80C3403F00113B3F1011FE7
:1097C000EBD1E6E700500040F8B54FF02002EFF390
:1097D000118382F31188BFF36F8F284A1078441CDD
:1097E000147078B183F31188BFF36F8F244BD3F8D3
:1097F0000C3403F00113B3F1011F0CBF00206FF014
:10980000430009E01F4D2F783FB1107083F311889A
:10981000BFF36F8F6FF00A00F8BD01262E7083F33F
:109820001188BFF36F8F164C21B3052000F0D2FAD8
:10983000C4F80071D4F80433C4F804632660D4F883
:1098400000219AB10022DB0758BF0123C4F8002190
:109850004FF0200258BFC4F808330B4B0520C3F863
:10986000802100F0A7FA00232B70BFE720BF40BF84
:1098700020BFE4E7C4F800112660F4E7C520022009
:1098800000500040C420022000E100E00022114B03
:1098900010B4C3F840214FF02002EFF3118482F39B
:1098A0001188BFF36F8FD3F8040540F247130A4ABB
:1098B0001168401A20F07F40B0FBF3F003FB001367
:1098C000136084F31188BFF36F8F5DF8044B02F0CF
:1098D00015BA00BF005001401000022038B51B48E7
:1098E00001F0F4FB70B3436802211B689847002421
:1098F00040F24713164D4FF40012C5F80845C5F85D
:1099000040354FF48033C5F84433C5F80433114B68
:1099100001211C60104B1520C3F88021224600F065
:109920006DFA152000F046FA012320460B4A136019
:109930002B60D5F8043503F2471323F07F43C5F8B5
:10994000403538BD4FF0FF30FBE700BFE4E30100D6
:10995000005001404051014000E100E0085001404A
:109960004CF6690270B5B0F1FF3F08BF10464FF0EA
:109970002003EFF3118483F31188BFF36F8F013855
:109980009042124DA8BF10462E6840F2471510496C
:1099900020EAE070D1F804359A1B22F07F4202F5EC
:1099A000A37205FB0020B0FBF5F005FB0060C31AB5
:1099B00023F07F431F2B98BF401920F07F40C1F850
:1099C000400584F31188BFF36F8F70BD1000022033
:1099D000005001404FF02002EFF3118382F3118811
:1099E000BFF36F8F084AD2F80405084A1268801A3C
:1099F00040F2471220F07F40B0FBF2F083F3118871
:109A0000BFF36F8F704700BF00500140100002206D
:109A100004488168406A884203D003494FF080526D
:109A20000A6070470806022004ED00E000232021B0
:109A30000348C2180133412B82F80013F9D1704753
:109A400000E100E0094A0A49936809685866996686
:109A500008494B6843F080534B60002383F311881F
:109A6000BFF36F8F9368986E704700BF080602209F
:109A70000CB9010000ED00E0202080F31188BFF355
:109A80006F8F11498A684FF028001044EFF3098C5A
:109A900080E8F01F0D4F4FF000664A6A8A603E6012
:109AA000506E0023536680F3118804B50648806821
:109AB00010F0A2FDBDE8044002F1280090E8F01F7C
:109AC0008CF30988704700000806022004ED00E0CE
:109AD0001EF0040F0CBFEFF30880EFF309808169DB
:109AE00031F8021C11F0FF010229FFD001B510F07E
:109AF00074FD01BD38B51B4C05461B4810F04FFDE9
:109B0000A36AD90602D5194810F049FDA36A1A07BD
:109B100002D5174810F043FDA36A9B070ED51548E0
:109B200010F03DFD616BA36A180607D5124810F0CE
:109B300036FD1DB1A36A23F08003A362094CA36A1A
:109B4000DA0702D50D4810F02AFDA36A9B0602D55C
:109B50000B4810F024FDA36AA36A002043F0FF0322
:109B6000A36238BD00ED00E090E40100A7E401002D
:109B7000DBE40100EFE4010008E501001FE501005E
:109B80003FE5010038B51E4C05461E4810F007FDA4
:109B9000A36AD90402D51C4810F001FDA36A1A0576
:109BA00002D51A4810F0FBFCA36A9B050ED5184895
:109BB00010F0F5FCA16BA36A180407D5154810F046
:109BC000EEFC1DB1A36A23F40043A3620C4CA36A0C
:109BD000590502D5104810F0E2FCA36ADA0509D550
:109BE0000E4810F0DCFC064A0020936A43F47F43E1
:109BF000936238BDA36A9B04F5D50948F1E700BF1D
:109C000000ED00E002E4010019E40100DBE40100E2
:109C10002BE4010045E401005BE4010077E401006E
:109C20003FE5010010B51C4C1C4810F0B8FCA36ABD
:109C30009A0102D51A4810F0B2FCA36ADB0102D5E2
:109C4000184810F0ACFCA36ADC0202D5164810F0EC
:109C5000A6FC114CA36A180302D5144810F09FFC0F
:109C6000A36A590302D5124810F099FCA36A9A031B
:109C700002D5104810F093FC074CA36ADB0302D511
:109C80000D4810F08CFCA36A00206FEA03436FEAD2
:109C90001343A36210BD00BF00ED00E06FE50100BB
:109CA00088E501009CE50100B7E50100E2E501005F
:109CB00001E6010027E6010042E6010038B52D4B20
:109CC00005465C6801F07F43B3F17F4F05D000206B
:109CD0002946BDE8384000F0FFB8C807F7D4490668
:109CE00002D5254810F05BFCC4F30804E21E092AE3
:109CF00035D8DFE802F0052E302B343434343432DA
:109D00001E4810F04CFC1B4BDA6A920703D51C4826
:109D100010F045FCDBE7DB6A5B00D8D5194810F092
:109D20003EFC194B1B782BB10120FFF7E3FE062800
:109D3000CED138BD154B1B781BB10120FFF722FF98
:109D4000F5E7134B1B889BB2002BC0D0FFF76AFFCF
:109D5000EDE70020E9E70020F0E70E48D8E70E48DD
:109D60000E49A4F110020F2CD8BF01460C4810F088
:109D700016FCACE700ED00E09CE60100C0E6010047
:109D8000D8E60100FAE6010028ED00E029ED00E048
:109D90002AED00E01AE701006EE6010083E601000B
:109DA00051E70100024A536943F0100353617047C1
:109DB00000ED00E043B2002B08DB012200F01F00A1
:109DC00002FA00F0024A5B0942F82300704700BF24
:109DD00000E100E043B2002B0DDB012200F01F0088
:109DE00002FA00F05B09044A203342F82300BFF373
:109DF0004F8FBFF36F8F704700E100E043B2002B3D
:109E000001F10101A8BF03F160434FEA4111B8BF5E
:109E1000054BC9B2ABBF03F5614300F00F0083F8F7
:109E200000131954704700BF14ED00E008B572B676
:109E3000044B186A18B100221A6211F0FDF962B6DB
:109E400008BD00BF080602202DE9F0418C188846A5
:109E500017461E4604220A9B0999054611F019FB74
:109E600000220D49A4F1680323F0070321F001014A
:109E7000C5E91322C5E91687996106991E605960E4
:109E800007991A6699600899D9604FF08071D96175
:109E9000AB646A66BDE8F081B3A2010001491022FB
:109EA0000A60704710ED00E0404080F3118830BF39
:109EB000704700BF404080F311884FF004007146A6
:109EC000014202D0EFF3098001D1EFF3088071461F
:109ED00001B5FFF7F3FE01BD38B504460D46052870
:109EE0001AD8DFE800F00319191315170D4810F000
:109EF00056FB01F06DFDAA6901460B4810F04FFBBF
:109F000029462046BDE8384000F018B80748EEE77B
:109F10000748ECE70748EAE70146074810F03FFB2F
:109F2000E7E700BF65E7010003E8010085E70100FE
:109F3000ABE70100C5E70100E0E70100052810B527
:109F40000CD001F09DFD60B101F09AFD0C490D4B64
:109F5000002808BF19460C4810F021FBFFF7A4FFAA
:109F6000FCE701F09DFD0028EED1084C0848A168EF
:109F700010F015FBA068BDE8104000F00BB800BF62
:109F80003FE8010043E8010054E801000806022010
:109F900074E8010038B505464FF02003EFF3118453
:109FA00083F31188BFF36F8F11F054FA0A4B9B684B
:109FB000AB420BD1094B5A68C2F3080212B92046D2
:109FC000FFF740FD5A6842F080525A602046BDE8D3
:109FD000384011F07CB900BF0806022000ED00E017
:109FE00001B572B60B4A106A00281EBF002111622B
:109FF00011F022F962B6EFF30580A0F110004FEAEC
:10A00000C0000549014409C99847BDE8014003481B
:10A010000047000008060220CCB50100119A00009C
:10A0200010F0DFFA00F004F830BFFFF7FDBF00BF0B
:10A0300008B5164B83F30988EFF3148343F002034A
:10A0400083F31488BFF36F8F114A124B22F07F0203
:10A050009A60BFF34F8FBFF36F8FD3F8882042F41D
:10A060007002C3F888204FF00042C3F83422BFF3D7
:10A070006F8FB0EE400ABFF36F8F01F06DF801F003
:10A0800075F8FFF7D3FC01F09FF800BF303B0220CA
:10A090000080000000ED00E010B50E4B88B0029388
:10A0A0000D4B0E4C03930E4B08A8049302AB40F8E3
:10A0B0001C3D0C4A2346012100F044F9002307937C
:10A0C000094B0121E41A05A80593069400F044F910
:10A0D00008B010BD000002200000000000000420B5
:10A0E00006000100000002200000022010B50B68ED
:10A0F0000C7A23F01F0304F01F021A43CB68640993
:10A1000023F01F03044943F0010343EA440388603A
:10A11000CA600B6110BD00BF90ED00E030B585B0A6
:10A120009DF808200D890B684C68498965F3040285
:10A1300061F3471200938DF8082023F01F03621E7D
:10A14000134423F01F030393084B04461B68C3F317
:10A150000723013B984205DC6946FFF7C7FF20460D
:10A1600005B030BD6FF01504F9E700BF90ED00E0D9
:10A170002DE9F04F06460F4614460025DFF84881CA
:10A1800085B0BD420BDA56F82530D3F80490B9F10A
:10A19000000F3CD0B9F11F0F05D86FF01504204611
:10A1A00005B0BDE8F08F19F01F0FF6D1D3F800A06D
:10A1B0001AF01F0FF1D150460FF078FE834609EBDD
:10A1C0000A0001380FF072FE8345E6D11BF1160F2D
:10A1D000E3D0631E5B45E0DBC8F808B0D8F80C009C
:10A1E000C8F808B0D8F8103056F8251020F01F0035
:10A1F00043F01F09D1E900321A44984202F1FF3AB4
:10A200001AD1D14505D15FFA8BF0FFF787FF0135F1
:10A21000B7E7C8F808B0D8F80C3022F01F0203F0F6
:10A220001F031A43C8F80C20E0B2FFF777FF10F1C4
:10A23000160FB2D0441CEAE7C8F808B0D8F81020CE
:10A24000013B23F01F0302F01F021343D145E0B28C
:10A25000C8F81030E9D0FFF761FF10F1160F9CD05D
:10A26000C8F808B0D8F80C209DF80830441C62F3F8
:10A2700004038DF80830D8F810309DF808205B08EA
:10A2800063F3471256F825308DF80820D3E90023F0
:10A290001A44009209F1FF3322F01F021344A3EB8A
:10A2A0000A0323F01F030393D8F80030E4B2C3F38A
:10A2B0000723013BA342FFF670AF20466946FFF734
:10A2C00015FF0134A3E700BF90ED00E00522034B2A
:10A2D0005A60BFF34F8FBFF36F8F704790ED00E070
:10A2E000BFF35F8F0022014B5A60704790ED00E092
:10A2F000104970B5104D0A682E68C2F307229642C5
:10A3000014D8FFF7EDFF00240C4B0B63A64205D1D8
:10A310000B4B1E70FFF7DAFF002070BD6968204606
:10A3200001EB0411FFF7E2FE0134EFE74FF0FF30DD
:10A33000F3E700BF90ED00E04CB80100AAFF440035
:10A34000C620022010B5034C2278FFF711FF2070C1
:10A3500010BD00BFC62002202DE9F74F89460746F1
:10A360000026DFF89080DFF890A0214C4E4519DAE6
:10A37000D7F804B0BBF1000F36D03B681846019304
:10A380000FF094FD019B05460BEB030001380FF025
:10A390008DFD1423854203FB06F306D06FF01502F2
:10A3A00048F8032003B0BDE8F08F15F1160F48F808
:10A3B0000350F7D09AF80020AA42F3DDA560434489
:10A3C000A560E068197B60F3040119732169187BAB
:10A3D000490861F347101873E26822F01F025A60BF
:10A3E000226922F01F021A6101360C37BEE700BF56
:10A3F00090ED00E014000220C620022070B50E4B44
:10A400000E461C780022234605460C480168C1F31D
:10A4100007218B420BDB0A4B191D1868FFF766FEFC
:10A42000224631462846BDE87040FFF7A1BE836052
:10A4300002610133EAE700BFC620022090ED00E090
:10A44000140002202DE9F04F1F4600239346C9B0A7
:10A45000CDE90C0104939BF800000BF1010548B114
:10A46000252879D0DDE90C319847013006D14FF02D
:10A47000FF330493049849B0BDE8F08FAB46049BCA
:10A480000133CDE90437059FE5E7232C5DD052D891
:10A49000002CEFD0202C08BF4FF001095D46AB46E1
:10A4A0001BF8014BBD48214610F064F90028ECD19F
:10A4B0002A2C59D13A683B1D002A0392BEBF524252
:10A4C000039201221F466C78B8BF069205F1020B79
:10A4D000039BC92B28BFC82303932E2C69D19BF85B
:10A4E00000302A2B62D13D680BF1010B0437C92DD6
:10A4F000A8BF4FF0FF359BF800400BF1010B214640
:10A50000A74810F037F918B19BF800400BF1010B88
:10A51000672C7CDC652C80F2E080472C4CDC452CE1
:10A5200080F2DB80002CA5D0252C00F03583C82CD0
:10A5300040F33C839BE72D2C0BD0302C07D02B2CE9
:10A54000079B08BF01230793A8E70126A6E702940B
:10A55000A4E701230693A1E74FF000092023CDE9EA
:10A56000069902934E469AE7A4F13003092B039013
:10A57000B3D80A22AB461BF8010BA0F13003092B1C
:10A580000446A5D8039B5D4602FB0300A0F13003FF
:10A590000393EFE7934600FB0535303D5A4612F82A
:10A5A000013BA3F130010929F4D9A0E700250A20D5
:10A5B000F4E74FF0FF35A2E7632C6FD032DC582C64
:10A5C000B5D13B1D05933968002E00F0DC8247F6BB
:10A5D00030030DF15607ADF854302B4610223846A3
:10A5E00010F06FF9582C06D10DF1530212F8013F0B
:10A5F000002B40F0CA820DF15408002EA7EB08088A
:10A60000404414BF4FF002094FF0000929E0702CBC
:10A6100000F094822BDC6E2C00F0538200F3578202
:10A62000692C84D13C683B1D002C059342DA2D2314
:10A63000B4F1004F8DF8543041D061420DF155080E
:10A640002B4640460A2210F03CF9079B804415A88F
:10A65000A8EB0000002B3DD1B9F1000F01D14FEA6A
:10A66000D4790135029B18BF2023029380E0752C1A
:10A6700000F08082782CA4D0732C7FF458AF002691
:10A680003B1D396805938B5D002B00F06682013617
:10A69000C82EF8D1002D80F2628266E23B1D059340
:10A6A0003B6801268DF8543000238DF855304FF06B
:10A6B00000091CE2079B23B12B238DF8543021465F
:10A6C000BCE7B9F1000F01D02023F6E721460DF1D8
:10A6D0005408B5E7DDF81C90C3E7073727F00707F4
:10A6E00007F108030593D7E900C7FB0243EA5C536F
:10A6F00023F000410B464FEACC22CDE9102340F273
:10A70000FF731046C7F30A589845CDE9000160462B
:10A7100048D1DDE90012002877F10003B8BF2D23EE
:10A7200015A8AEBF03468DF854300DF155030A430A
:10A73000A4F1410403F1030825D1192C1DD84922A5
:10A740001A704E225A7046229A700022DA70079BC5
:10A75000A8EB0000002B40F05582B9F1000F07D1A3
:10A760009DF85410A1F12D03D3F1000949EB030921
:10A77000C8283FF77CAE0646B9E169221A706E22FE
:10A780005A706622E0E7192C99BF4E2241216E22B1
:10A79000612194BF1A701A705970D5E799E80100C9
:10A7A0009FE80100462CDDE9002342EA080243EA63
:10A7B000E87308BF6624134343D0DDE90023002873
:10A7C00043F00043CDE9102377F10003A8F2FE38EF
:10A7D00039DA2D238DF854300DF1550A00230093FA
:10A7E00018F1020F3EDBB8F1000F79DC10A808F178
:10A7F000010810F08EF8B8F1040FF7D1002D24F005
:10A800002003B8BF0625472B40F09780002E40F06C
:10A8100092802B1C18BF01230893009B033304DB99
:10A82000009A6B1C9A4240F38D80672C0CBF652404
:10A83000452405F10108102398450F93A8BF9846B9
:10A8400089E04FF00008079B0BB12B23C2E7B9F159
:10A85000000F01D02023BDE70DF1540ABEE710A878
:10A8600010F057F8DDE9107C00230B930023CDF89E
:10A8700028C0A94ADDE90A018B4208BF824208F1DB
:10A880000108ECD30522A7FB0201CDE90801099BD1
:10A8900002FB0C334FF0000C0993DDE90823CDE9EE
:10A8A0001023009B013B0093002300216FF0004028
:10A8B000099A994208BF904207D2BCF1000F8FD08D
:10A8C000DDE90823CDE910238AE7DDE908239218A2
:10A8D0005B41CDE9082308F1FF384FF0010CE3E7B5
:10A8E00010A810F029F84FF0000C009B08F1FF3879
:10A8F00001330093DDE91023CDE908230023002173
:10A900006FF00040099A994208BF904208D2BCF10A
:10A91000000F3FF468AFDDE90823CDE9102362E7BB
:10A92000DDE9082392185B41CDE9082308F1FF38DF
:10A930004FF0010CE2E700236EE70023662C08933A
:10A940007FF477AF009B13EB05084BD510236624EB
:10A950004FF000080F9300224FF0006348A961E90F
:10A96000362318F1FF383FD2DDE91023DDE912016B
:10A97000171843EB01083A464346CDE9102300235C
:10A9800008F07042134308D010A80FF0D5FF10A8AC
:10A990000FF0BFFF009B01330093662C0AF1010802
:10A9A00040D1009B002B29DD534498460FA910A8E5
:10A9B0000FF0F2FF0AF8010BC245F7D10023009314
:10A9C00006B95DB12E2346464FF0300A88F80030B4
:10A9D00008EB0503B34215D10135A844089B002BB1
:10A9E00039D160E0662426E708460A910FF0A4FFFB
:10A9F0000A9908460FF08DFF0A99B2E730238AF8CA
:10AA00000030DDE7009A2AB1013286F801A00092F9
:10AA10000136DFE70FA910A80A930FF0BDFF0A9BCC
:10AA20007070F5E70FA910A80FF0B6FF302818BF17
:10AA3000009B8AF800001CBF03F1FF33009306B9A6
:10AA40003DB12E230AF102088AF8013045444545FC
:10AA50002ED1089B43B118F8012C08F1FF33302A9E
:10AA60002DD02E2A08BF984624F02003452B1AD15A
:10AA7000009B0A22002BBBBF5B4200932B232D239C
:10AA800088F80130009B88F8004093FBF2F303F153
:10AA9000300188F80210009908F1040802FB13172E
:10AAA000303708F8017C002315A888F800304EE6FE
:10AAB0000FA910A80FF070FF08F8010BC7E7984620
:10AAC000C9E73B1D0593049A3B681A60DBE43B1D14
:10AAD0000593396816B330238DF8543059BB0135CE
:10AAE000029B18BF202389468DF855100293039BC3
:10AAF000B34240F38580069B15AD002B58D0202330
:10AB0000039AAB550136B242FAD1DDE9033215ACF6
:10AB100013441D46A41A6FE03233333315A80DF1E8
:10AB200054082B460822A0EB08080FF0CAFE404448
:10AB30004FF0000995E50DF15500F0E73B1D059339
:10AB400047F630033968ADF85430102208230DF170
:10AB500056000FF0B6FE0230EAE7002D02DBAE42EF
:10AB6000A8BF2E46002E3FF48EAC324615A80FF03B
:10AB70005AFE9CE53B1D05930A222B46396815A811
:10AB80000FF09FFED4E715AF27E5A3F16101192966
:10AB90009CBF203B137029E50D9920460C9B9847DC
:10ABA00001303FF464AC049B0133049305976AE4DD
:10ABB000039B721C9C1B281929460FF01DFE069B47
:10ABC000029A202A18BF4B4606931C44069BA342B8
:10ABD0009BDA069B1A46029BAB541346013306933D
:10ABE000F4E7049B0D99E05C0C9B984701303FF41F
:10ABF0003EAC049B01330493049BAB42F1D142E48D
:10AC0000039682E7DDF81C90B2E500BF0CB41FB5D7
:10AC100009B90DF10300CDE9020107AB069A02A9BB
:10AC200005480193FFF70EFC0022029B1A7005B045
:10AC30005DF804EB02B07047CFA901008279044BA4
:10AC400003EB4213DB69C01A024BC0105843704734
:10AC500090510220ABAAAAAA10B5094B827903EB46
:10AC600042139B690A685C6823689A4294BF0A6031
:10AC70000B60FFF7E3FFD4E9002302FB003010BDB7
:10AC80009051022000220E4BF0B51C680D4B164669
:10AC90001F46BD58B91885420DD075B14D680832B0
:10ACA000651BB542C4BF2E460B46502AF1D119464A
:10ACB000013C18605C600846F0BD0B46F7E700BF3A
:10ACC0002800022034000220684620F007018D464B
:10ACD00019B50FF081FC0D4BD3E8EF2F0132C3E81B
:10ACE000E12F0029F8D104F0FDFD094B1C6824B1C7
:10ACF000201D00F073FE2468F9E7FFF797F8FEF7D0
:10AD000087FEBDE819408546704700BF2800022035
:10AD10002C0002202DE9F0430D4689B010F005FC0F
:10AD20002B680646002B0F4603D100F0BBFD3C20EC
:10AD30006CE0B8BF4FF0FF334FF00102B8BF2B609B
:10AD4000002102A810F074FB0DF104084FF020035D
:10AD5000EFF3118983F31188BFF36F8F00F038FE92
:10AD6000FFF790FF324C4368226893424FF0000394
:10AD700008D101932F4B5A68002A4AD1C3E90088B1
:10AD8000012300E0426089F31188BFF36F8F002B2D
:10AD90003BD0296802A800F04DFE4FF02003EFF3EE
:10ADA000118983F31188BFF36F8F0021214B1A683B
:10ADB0005AB1424538D1019800292FD159681860FD
:10ADC000914200D158600023019300F001FEFFF78B
:10ADD00059FF2368436089F31188BFF36F8F2C6894
:10ADE000631C12D010F0A1FB861B61EB0707E31771
:10ADF000A21B63EB07031946002A71F100031046FA
:10AE0000B8BF00202860002891D0002009B0BDE81C
:10AE1000F083C2F80080C3F80480B1E70860586886
:10AE2000904208BF5960CEE711461268C0E700BFE4
:10AE3000280002202C0002204FF08052014BC3F862
:10AE40000021704700E100E04FF08052014BC3F851
:10AE50008021704700E100E04FF00052014BC3F841
:10AE60000021704700E100E04FF00052014BC3F8B1
:10AE70008021704700E100E008B50023074AC2E9DD
:10AE80000033074AD2E8EF1FC2E8E03F0028F9D1BB
:10AE90000FF060FEBDE808400FF051BE2C0002200C
:10AEA0002800022008B50248FEF7E8FB002008BD94
:10AEB000B8B80100B0F58D7F0DD040F20223984262
:10AEC0002AD001282AD1142924D0192922D00429D2
:10AED00024D1042313E0013905291FD801A353F815
:10AEE00021F000BFFDAE000005AF000009AF00007B
:10AEF0000DAF0000D3AE000011AF000002231360BD
:10AF0000002070470523FAE70623F8E70723F6E752
:10AF10000123F4E71160F3E70129F9D04FF0FF3086
:10AF2000704700BF014B1B685B6818470C0002208C
:10AF3000F0B50E4CA1B023681646DF6A0023054623
:10AF4000B84786420ED1236880225C6A6946002396
:10AF50002846A047012805D90222694604480FF077
:10AF60003BFC08B16FF0040021B0F0BD0C000220E2
:10AF70003FE90100034B40F201221B6800211B68DE
:10AF8000662018470C0002202DE9F043A1B0FFF71E
:10AF9000F1FF431C04464FD00A222949FFF7C8FF9E
:10AFA000054630B12046FFF7BDFF284621B0BDE879
:10AFB000F0830A2223492046FFF7BAFF05460028FE
:10AFC000F0D1162220492046FFF7B2FF054600289F
:10AFD000E8D109221D492046FFF7AAFF05460028AF
:10AFE000E0D11B4E1B4FDFF8788033688022D3F806
:10AFF0002490694600232046C8470028F5D009223E
:10B00000694638460FF0E8FB0028CBD00822694695
:10B0100040460FF0E1FB0028C4D0092269460E48E3
:10B020000FF0DAFB0028BDD0082269460B480FF06C
:10B03000D3FB0028D9D1B5E76FF00D05B5E700BF08
:10B0400034E90100A4E80100AFE80100C6E801000E
:10B050000C000220FDE8010010E901001AE90100DE
:10B0600007E9010038B50446FFF784FF431C054695
:10B070000ED0094B002C094912BF22220922194681
:10B08000FFF756FF04462846FFF74CFF204638BD21
:10B090006FF00D04FAE700BFD0E80100DAE8010024
:10B0A00070B50026084B53F82040013053F820506B
:10B0B000A54200D870BD236820465B68984700B160
:10B0C00066600C34F4E700BFF8B80100104B70B5AF
:10B0D00005461E460F4C9C4204D10E4CB44209D189
:10B0E000002412E062681AB122681268AA420CD0E9
:10B0F0000C34F0E763680BB90C34EFE7236828469B
:10B1000019680FF04DFB0028F6D1204670BD00BF36
:10B11000FC50022084500220014B98685430704744
:10B120000806022008B50B4D4FF02002EFF3118303
:10B1300082F31188BFF36F8F10F0C9F90121044623
:10B140000228D8BF084610F0D2F92C62FEF7ACFEF8
:10B15000EAE700BF080602200248034A0021121A4B
:10B160000FF08EBB00000220EC21022008B506483B
:10B17000064A0749121A0FF056FBBDE80840054A77
:10B18000054906480FF04FBB50500220D051022015
:10B190004CE90100000000004CE901000000022021
:10B1A00008B50220FFF77CFF0320FFF779FF00F0CE
:10B1B000BDFCFEF7A7F9034A137B23F001031373C9
:10B1C00008BD00BF3001022080B53B4BB2B083F315
:10B1D00008880024E022394B012783F82220DC77FD
:10B1E0001C765C769C765A6A354E42F4E0225A62AE
:10B1F000FEF7D8FDFEF752FE07AB2146AC221846FB
:10B200000FF03EFBB06020468DF82970FFF748FF35
:10B210003846FFF745FF2B4D00F038FB2A4B75628F
:10B22000CDE904730723CDE90044CDE902434FF48F
:10B230008052264B2649284600F05EFC6B7B344644
:10B2400023F0040213F01B0F6A7304D1AB6913B926
:10B25000284600F0CDF91F4B012205930F23CDE9BD
:10B26000033200231C4E4FF4A0721C493046CDE936
:10B27000013300931A4B00F03FFC737BE66023F030
:10B2800004037373174BC4E90633FEF705FF0D483B
:10B29000A5600FF0B1F90D4B134A184682F30988E7
:10B2A00063B64FF0000181F31188BFF36F8F002167
:10B2B000002200230EF0FDFF303B022000ED00E0F5
:10B2C000080602203001022042E90100A1B100007D
:10B2D000F021022047E9010084000220F031022021
:10B2E00025B1000020060220F031022070B50024B4
:10B2F0000A4B0B48834201D3002070BD00211A691C
:10B300009D685C61A94201D11C33F3E75E6901319C
:10B310001660DE685A613244F4E700BF285102200B
:10B320006051022038B5074C074DAC4201D30020D4
:10B3300038BD04F114032046C4E905330EF002FEC3
:10B340001C34F2E7605102207C5102202DE9F04FBD
:10B350001D1E85B006460C46174659DD00F024FD3B
:10B360004FF4004C002180462A484FF4A0220023CD
:10B37000CCFB0501FCF7E6FE18EB0002264B9046DD
:10B38000F31A264A9B1002FB03FA06F1140B5FFA2C
:10B390008AFA009403AB02AA394630460EF01DFE2D
:10B3A00010F10B0F0BD1009403AB02AA39463046C3
:10B3B0000EF013FE10F10B0F08BF6FF00B00637956
:10B3C000029A84F804A062F3030363716368039A2A
:10B3D00062F31F336360C0B1BDB110F10C0F14D123
:10B3E0004FF02003EFF3118083F31188BFF36F8FC9
:10B3F0002A46594600F012FA6B1CCAD000F0D4FC61
:10B40000B8EB0005C5D56FF00A0005B0BDE8F08FB8
:10B410000022B3E7FFFF040060510220B76DDBB6E6
:10B4200070B5047802684178114EC4EBC404A400DE
:10B43000120B01F00F0130190EF096FE4FF02003B1
:10B44000EFF3118583F31188BFF36F8F04F11400BC
:10B4500030440FF0D7FF28B12946BDE870400548B9
:10B460000FF027BF85F31188BFF36F8F70BD00BF4A
:10B4700060510220C7200220014601480FF0DEBEC5
:10B4800060510220EFF305800D2809D828B1054B43
:10B49000586880F40060C0F3C02080F0010070475D
:10B4A0000120FAE700ED00E008B5FEF793FA054B3E
:10B4B000054A1B680021184410611846BDE8084081
:10B4C00010F015B84006022008060220F8B50D4617
:10B4D0004FF02003EFF3118483F31188BFF36F8FD4
:10B4E0004FF40041002700220B4E0C4BC1FB0067BC
:10B4F0001A6130464FF4A02200233946FCF722FEA1
:10B50000074B1860074B1D60FFF7CEFF84F31188CF
:10B51000BFF36F8FF8BD00BFFFFF040008060220D5
:10B52000400602203C0602204FF02003EFF3118179
:10B5300083F31188BFF36F8F044B9A68D37B013B71
:10B54000D37381F31188BFF36F8F70470806022011
:10B55000094B03F12802824205D19B688B4202D13C
:10B560004B7BDB0607D1D1E900231A600A685360E0
:10B570000023C1E9003370470806022038B50D4C9E
:10B58000024604F128000FF0D9FE054600B9E5682F
:10B59000A3684AB95A7BD20606D1AA6922B9DA89C8
:10B5A0007F2A01D9636238BD9D4201D0FFF77CFF3D
:10B5B0006562F8E70806022010B54FF02003EFF3AC
:10B5C000118483F31188BFF36F8F084B01209A68B1
:10B5D000D37B0133D373FFF7D1FF84F31188BFF31B
:10B5E0006F8FBDE810400FF081BE00BF080602203B
:10B5F000F8B54FF02003EFF3118483F31188BFF304
:10B600006F8F164A114651F8283F8B420CD05BB120
:10B61000D66A90F90E5093F90E70AF420BDCB3422C
:10B6200002D01B68002BF6D1D36A01604360D36A55
:10B630001860D06205E05A68C0E900325A681060AC
:10B640005860437B43F0400343730020FFF796FFAD
:10B6500084F31188BFF36F8FF8BD00BF0806022086
:10B66000F8B504464FF02003EFF3118683F31188F9
:10B67000BFF36F8F194F014607F128052846FFF7E2
:10B6800067FFBB6A3A46AB420CD05BB1F86A94F9EB
:10B690000E1093F90E708F420BDC834202D01B68B0
:10B6A000002BF6D1D36A25606360D36A1C60D46234
:10B6B00005E05968C4E9003159680C605C60637B3F
:10B6C000906843F040036373031B58425841FFF7EF
:10B6D00055FF86F31188BFF36F8FF8BD080602206F
:10B6E0001449154A10B58B681468A34203D1BDE80C
:10B6F0001040FFF7D9BE00241460104A1268BAB196
:10B70000DA897F2A14D80E4A93F90E4012689442BF
:10B710000EDB0C4A126893420AD09A6942B90A6950
:10B72000824203DC1846FFF79BFFE0E7121A0A612A
:10B7300010BD00BF08060220380602204006022085
:10B740003C06022010B9010038B504464FF0200332
:10B75000EFF3118583F31188BFF36F8F437B5A0694
:10B7600007D501460948FFF7F3FE637B23F040034A
:10B770006373074B9868031B58425841FFF7FEFE5E
:10B7800085F31188BFF36F8F38BD00BF30060220EC
:10B790000806022070B504460D461646FFF7D4FF92
:10B7A000637B43F002036373EDB12B68A5609D4298
:10B7B0000CD05BB194F90E2093F90E1091420CDC81
:10B7C00069688B4202D01B68002BF5D16B6825603D
:10B7D00063606B681C606C6005E05A68C4E9003205
:10B7E0005A6814605C60731C12D04FF4004500214D
:10B7F00008484FF4A022C5FB06010023FCF7A2FC79
:10B800000549421C04F11800BDE8704000F032BA4E
:10B8100070BD00BFFFFF040049B3010070B50646CC
:10B820000E4D0F4CA868FFF7B5FFAB68304623609C
:10B83000FEF708F94FF02002EFF3118382F311882D
:10B84000BFF36F8F2268A968914204BF0022226073
:10B8500083F31188BFF36F8F70BD00BF080602200D
:10B860003806022010B50C461146064A9068064A72
:10B8700010601A46FFF78EFF2046BDE81040FEF725
:10B88000E1B800BF08060220380602200021044B60
:10B89000084603F12802C3E90A22FFF717BE00BFDA
:10B8A00008060220F8B5224C224BA2681B689A4277
:10B8B00032D04FF02003EFF3118683F31188BFF3EA
:10B8C0006F8F04F12805A1682846FFF741FEA36A9F
:10B8D000A268AB420CD05BB1E16A92F90E0093F919
:10B8E0000E7087420BDC994202D01B68002BF6D108
:10B8F000E36A15605360E36A1A60E26205E0596822
:10B90000C2E9003159680A605A600120FFF736FE2B
:10B9100086F31188BFF36F8F4FF02003EFF3118090
:10B9200083F31188BFF36F8FBDE8F840FEF78AB844
:10B930000806022010B90100F8B5044618B9FFF74F
:10B94000B1FF2046F8BD4FF4004500211C484FF4DC
:10B95000A0220023C5FB0401FCF7F4FB461C0FF0FA
:10B96000E0FD34184FF02003EFF3118783F31188C3
:10B97000BFF36F8F134D144BA8681860FFF7E4FEF8
:10B98000A86812493246183000F074F9AA6838469F
:10B99000537B43F010035373FEF754F80FF0C1FDCF
:10B9A000201A002809DD4FF47A716422002380FBFD
:10B9B0000101FCF717FC0446C3E70024C1E700BF00
:10B9C000FFFF0400080602203806022049B30100E8
:10B9D000014B9868704700BF0806022070B5044606
:10B9E0004FF02003EFF3118683F31188BFF36F8FBD
:10B9F0000FF0DBFC054670B1437BDB0603D18369A6
:10BA00000BB9FFF7F5FD0023AB663146BDE870408A
:10BA100007480FF04EBCD4E902329A4218BF0133F6
:10BA20000221A36004F110000FF0BBFDEDE700BFA1
:10BA3000C720022010B402460B464FF02000EFF35F
:10BA4000118180F31188BFF36F8F94684CB1013C72
:10BA5000946081F31188BFF36F8F00205DF8044B71
:10BA6000704733B981F31188BFF36F8F6FF00F0008
:10BA7000F4E702485DF8044BFFF7F4BEC72002204C
:10BA8000EFF305800D2807D838B1044B586880F4CF
:10BA90000060C0F3C02070470120704700ED00E057
:10BAA000024B9B68187B00F00100704708060220DB
:10BAB00010B502464FF02003EFF3118483F3118891
:10BAC000BFF36F8F437B590704D484F31188BFF30E
:10BAD0006F8F10BD23F0040343730FF0B2FC10B15D
:10BAE0001046FFF785FD2146BDE8104001480FF0E4
:10BAF000E0BB00BFC720022030B587B00E9D0446D2
:10BB000004950D9D03950C9D02950B9D01950A9D35
:10BB10000095FEF799F9044B9B6813B9236607B0AB
:10BB200030BD1B6EFAE700BF080602202DE9F04F7A
:10BB3000284E294DB04687B0B54205F130040FD3E9
:10BB4000FFF7F2FC4FF400490027234C234EDFF8A7
:10BB500090A0444521D307B0BDE8F04FFFF72CBDBE
:10BB600054F8043C059354F8103C049354F8143CE6
:10BB7000039354F8183C029354F81C3C019354F876
:10BB8000203C009354E90A2354E90C01FFF7B4FF69
:10BB900054F8303CDD642546CEE7616A4B1C04D086
:10BBA000256821B92846FFF783FF3034D1E7B34633
:10BBB000BC46C9FB01BC4FF4A02200235846614695
:10BBC000FCF7C0FA5146421C05F1180000F052F88B
:10BBD000EBE700BFFC500220FC500220FFFF0400F6
:10BBE00049B30100034B1B680BB9FDF7F3BE0020FE
:10BBF000704700BF44060220036840B1084A5268FB
:10BC0000904204D01BB19A6881680A449A604268E5
:10BC1000136003685A600023C0E90033704700BF17
:10BC20005850022038B5104B1B78002B0F4B18BF13
:10BC30004FF0FF301C6808BF6FF000409C420AD0F4
:10BC40004CB1A568FFF7CEFF281A00280ADBA468CC
:10BC5000FFF7C8FF201A064B1B6913B19842A8BF13
:10BC6000184638BD0020F6E7C720022058500220B1
:10BC70000806022070B504461646C1604FF0200346
:10BC8000EFF3118583F31188BFF36F8FFFF7AAFFDE
:10BC9000012EACBF80190130174BA0601A689A4280
:10BCA00001D05E6832B95A68236062605A681460D5
:10BCB0005C600BE09068A168884216DD411A9160D3
:10BCC0005168C4E9002151680C6054601A689A42B6
:10BCD00006D0944204D1FFF7A5FF0021FDF740FEF6
:10BCE00085F31188BFF36F8F70BD091A9642A1606A
:10BCF000D9D01268D6E700BF585002202DE9F04B8A
:10BD00000446FFF7EDFC4FF02003EFF3118583F3BA
:10BD10001188BFF36F8F214F214EB846DFF8849012
:10BD20003460D9F8004032684C45D7E900BC05D0F2
:10BD300024B1A368934214DD9B1AA36000241BEB7B
:10BD400002004CEBE271C8E900013460FFF76AFFC2
:10BD50002146FDF705FE85F31188BFF36F8FBDE81F
:10BD6000F08B1BEB03004CEBE371D31A3360002321
:10BD7000C7E90001A3602046FFF73EFF85F3118865
:10BD8000BFF36F8FE36898474FF02003EFF31185FF
:10BD900083F31188BFF36F8FC3E700BF0000022059
:10BDA00044060220585002202DE918484FF0200385
:10BDB000EFF3118483F31188BFF36F8FFDF70AFE51
:10BDC000074BD3E9002312EB000B43F1000C58465C
:10BDD000614684F31188BFF36F8FBDE8188800BFF8
:10BDE00000000220026A38B5002A044602DD0E492E
:10BDF000FFF740FF636A01336362A3690BB120461A
:10BE0000984754F8105FA5420DD065B128460FF051
:10BE100037FA6B7BDB0604D1AB6913B92846FFF711
:10BE2000E7FB0023AB6638BDE5BD00002DE9F3411B
:10BE30000027144E044688464FF4004530463946E4
:10BE40000023C5FB02014FF4A022FCF77BF9394621
:10BE5000009030464FF4A0220023C5FB0801FCF7F8
:10BE600071F9019020460FF01CFB009B20462362D5
:10BE70000023019A0449636202B0BDE8F041FFF774
:10BE8000F9BE00BFFFFF0400E5BD0000704700BF22
:10BE900005F0AABB08B5074B1A6842F000421A60C9
:10BEA0001B68DB0702D4FFF7F1FF08BDFFF7F0FFC7
:10BEB00008BD00BF4806022010B5084C23684BB9E6
:10BEC0000123236000F01AF82368002B01DB022312
:10BED000236010BD0F20FFF7D9FF10BD48060220D8
:10BEE0000FB408B52D200EF0ACFDBDE808404FF0B2
:10BEF000FF3004B0704700BFFFF7CCBFF0B593B080
:10BF000005F0A4F920B92C4901A805F013FA18B1DD
:10BF1000FFF7C0FF13B0F0BDFEF7AEFF03F048FD22
:10BF200002460028F4D120234FF4804008214FF42A
:10BF3000405C224FCDE91022214E039305930793D5
:10BF4000204D214C214A224B09900D900DEB010010
:10BF5000CDF82CC0CDE90E110297049606950894F1
:10BF60000A920C9300F096FB0028D1D103F034FB29
:10BF70000028CDD105F06EFE0028C9D102F052F99B
:10BF80000028C5D106F07AF80028C1D106F050FC8F
:10BF90000028BDD104F092FD0028B9D100F0BAF814
:10BFA0000028B5D101F064F90028B1D104F0B8FC43
:10BFB0000028AFD0ACE700BF1CBA01000000012090
:10BFC000400001202000012060700120600001205D
:10BFD00060300120022808B50ED022D90A280BD0E3
:10BFE000662819D140F201239A4229D040F2022357
:10BFF0009A4211D1134808BDA2F582720A2A1BD8B1
:10C00000012340F20341104803FA02F20A4200F110
:10C01000280318BF184608BD16200EF012FD002098
:10C0200008BD0128F8D140F203239A4206D0B2F5A8
:10C03000017FF1D1054808BD034808BD044808BD8B
:10C04000044808BDB4B901003CB90100DCB90100E5
:10C050008CB9010014B9010038B5054603F0CEFBD8
:10C06000044650B9234BAB431AD0234BAB4315D0F6
:10C07000224BAB4338D1224838BD83680269022B7A
:10C0800010D01FD90A2B0DD0662B24D140F20123EA
:10C090009A4227D040F202239A421CD1194838BD57
:10C0A000194838BDA2F582720A2A19D8012340F234
:10C0B0000341164803FA02F20A4200F1280418BFAD
:10C0C000204638BD012B06D140F203239A42E7D027
:10C0D000B2F5017FCFD016200EF0B3FC002038BDA2
:10C0E0000A4838BD0A4838BD09200EF0AAFC20468F
:10C0F00038BD00BF3254764900009A7843547649DF
:10C10000DCB90100B4B901008CB901003CB90100EF
:10C1100014B9010070B586B01D4902A805F00AF9EE
:10C1200000BB0146044640F20122662005F094FD62
:10C13000184E00280546306010DB17480EF028FB2B
:10C1400023460246144928460194009405F034FD24
:10C15000054611480EF01CFBA84207D005242046D6
:10C1600006B070BD6924204606B070BD3068CDE9C8
:10C17000004403A923460A2205F000FE0128EDDD54
:10C1800003A8022205490EF018FB0028E7D0E5E7D6
:10C19000645002206050022034BA010040BA01000D
:10C1A000014B1860704700BF58160220F0B56C4B69
:10C1B00083B01B78002B00F0AD806A4B1C68A2682E
:10C1C00063689A422DD04BF6EF63ADF800302378C8
:10C1D0006E468DF80430636805219A422ABF2769AC
:10C1E0009F1ABF1A9A4294BF0025E568BFB288BF64
:10C1F0005B1B304688BF9DB2ADF802700EF0B5FCF7
:10C20000BDF80210A0680EF0B0FCA36822691F44BC
:10C21000974208BFE368A76008BFA360002D40F005
:10C220008D80514B1C68A26863689A422CD04BF6F3
:10C23000EF63ADF8003023786E468DF80430636804
:10C2400005219A422ABF27699F1ABF1A9A4294BFB2
:10C250000025E568BFB288BF5B1B304688BF9DB232
:10C26000ADF802700EF081FCBDF80210A0680EF06F
:10C270007CFCA36822691F44974208BFE368A7605B
:10C2800008BFA360002D48D1384B1C68A2686368C2
:10C290009A422BD04BF6EF63ADF8003023786E4610
:10C2A0008DF80430636805219A422ABF27699F1AD6
:10C2B000BF1A9A4294BF0025E568BFB288BF5B1BD6
:10C2C000304688BF9DB2ADF802700EF04EFCBDF84E
:10C2D0000210A0680EF049FCA36822691F4497422F
:10C2E00008BFE368A76008BFA3600DB903B0F0BD45
:10C2F00030460521ADF802500EF037FCBDF80210B3
:10C30000E0680EF032FCBDF80220E3681344A3603D
:10C3100003B0F0BDFEF7A8FD4FE705213046ADF8AC
:10C3200002500EF022FCBDF80210E0680EF01DFC79
:10C33000BDF80220E3681344A360A5E70521304659
:10C34000ADF802500EF011FCBDF80210E0680EF0DE
:10C350000CFCBDF80220E3681344A36061E700BF52
:10C36000C8200220541602204C160220501602202B
:10C3700000222DE9F04FB04B83B01B6819695C694E
:10C38000187C1A74587C5A74987C9A74D87CDA7425
:10C39000187D1A75587D5A75987D9A75D87DDA750D
:10C3A000B9B10139032914D8DFE811F0D60003012F
:10C3B000040016000125032000226FF05F019F4C4E
:10C3C00025701C7A1872587A5A72987A9A72DA7AA8
:10C3D000D97203B0BDE8F08F042100226FF05F0036
:10C3E0001C7A1972597A5A7294499C7A9A72DC7A38
:10C3F000D8720A700B78002B00F01781904B1C68E4
:10C40000A26863689A422DD04BF6EF63ADF8003016
:10C4100023786E468DF80430636805219A422ABF5E
:10C4200027699F1ABF1A9A4294BF0025E568BFB2D8
:10C4300088BF5B1B304688BF9DB2ADF802700EF01E
:10C4400094FBBDF80210A0680EF08FFBA368226970
:10C450001F44974208BFE368A76008BFA360002D90
:10C4600040F0D280774B1C68A26863689A422DD056
:10C470004BF6EF63ADF8003023786E468DF804304C
:10C48000636805219A422ABF27699F1ABF1A9A42F8
:10C4900094BF0025E568BFB288BF5B1B304688BFEC
:10C4A0009DB2ADF802700EF060FBBDF80210A068FE
:10C4B0000EF05BFBA36822691F44974208BFE36844
:10C4C000A76008BFA360002D40F08D805E4B1C6804
:10C4D000A26863689A423FF47CAF4BF6EF63ADF815
:10C4E000003023786E468DF80430636805219A4247
:10C4F0002ABF27699F1ABF1A9A4294BF0025E56890
:10C50000BFB288BF5B1B304688BF9DB2ADF80270DA
:10C510000EF02BFBBDF80210A0680EF026FBA368FE
:10C5200022691F44974208BFE368A76008BFA36061
:10C53000002D3FF44EAF05213046ADF802500EF00D
:10C5400014FBBDF80210E0680EF00FFBBDF80220EE
:10C55000E3681344A3603CE7384A117809B100212D
:10C560001170A568002D39D04FF0000CDFF8D4A071
:10C57000DFF8CCB03449E14666466246D1F800E0C7
:10C58000DAF80080DBF8007008E0632916D0612932
:10C5900004BF074601260132AA4213D0911C04EBC6
:10C5A0008101486801786229EFD180464FF0010986
:10C5B000F1E7FEF751FC03B0BDE8F08F86464FF07F
:10C5C000010CE8E7A6BBB9F1000F01D0CAF8008062
:10C5D000BCF1000F02D01C4AC2F800E0012000228A
:10C5E0006FF05F01EDE605213046ADF802500EF028
:10C5F000BCFABDF80210E0680EF0B7FABDF80220F0
:10C60000E3681344A36061E705213046ADF80250AA
:10C610000EF0ABFABDF80210E0680EF0A6FABDF815
:10C620000220E3681344A3601CE7FEF71DFCE5E667
:10C63000CBF80070C7E700BF58160220C8200220C0
:10C64000541602204C16022050160220014B187876
:10C65000704700BFC8200220002070470B4BD3E971
:10C660000023134498420DD282420BD810B50446E1
:10C6700000F0E0FC40B1064A84600260BDE8104072
:10C6800000F020BC04F0A4BF10BD00BF5C16022067
:10C690000100020000282BD030B589B001AA6946FC
:10C6A000044600F025FB034640B1134A04F128007C
:10C6B00003C882E80300184609B030BDDDE9001266
:10C6C000204600F04BF803460028EED10B4B0C49F6
:10C6D0000C480D4A03930D4D0D4B049105900D49E7
:10C6E00002A807930695029203F0ECFA0346DCE7F2
:10C6F0000E231846704700BF5C160220C5CF00000D
:10C7000095D0000085CC0000C5CE00005DC60000BD
:10C7100059C600006416022060B108B54368DBB258
:10C72000022B0ED003681B0C022B05D0042B0ED05D
:10C73000002008BD00207047806804F049FF0020F9
:10C7400008BD0146BDE80840034803F0A5B902480A
:10C7500003F018FB002008BD64160220002800F03A
:10C76000FF802DE9F04F056895B0002D00F0EE80B8
:10C770008368002B00F0EA800769002F00F0E68054
:10C78000846A002C00F0E28044681B2C40F2E380B5
:10C79000C4680B2C40F2DF80D0F814E0BEF1170F14
:10C7A00040F2D980002604466F48CDE90012DFF838
:10C7B000D8A16E490680A06BDFF8D0C1DFF8D08128
:10C7C000DFF8D0B1DFF8D09172460E60CAF80000F1
:10C7D00031463846CCF80060CBF80030C8F800602D
:10C7E000C9F800600EF04CF8E36938463B60A36975
:10C7F0007B60FFF7D5FC01224FF0040C5C4B5D49D8
:10C80000C3F810560968802004915B49DDF810E0F8
:10C81000C3F8146609682E7003916E70EE70AA70EA
:10C820000399A16ADBF800E06960E16A019CA960F4
:10C83000EC60009C5149AF61C5F814E02C61C3F86D
:10C8400090250C68A1F592610594059CC3F898C5E4
:10C85000D1F898444FF480670694069C1024C3F8DE
:10C86000A045D1F8A044464D0794079C4024C3F846
:10C87000A845D1F8A8440894089CC3F8AC05D1F8A1
:10C88000AC0409900998C3F8006108680A900A98F6
:10C89000C3F8086188680B900B98C3F810610869A9
:10C8A0000C900C98C3F8186188690D900D98C3F826
:10C8B0001C61C86901F501710E900E98D3F804034C
:10C8C0001043C3F804030C682E480F940F9CD3F850
:10C8D000044344EA0C04C3F804430C681094109C0D
:10C8E000D3F8044344F01004C3F804430C681194D3
:10C8F000119CD3F8044344F04004C3F804430C688B
:10C900001294129CD3F8044344F08004C3F8044307
:10C91000DAF8003009685B011391DBB21399C8F8AB
:10C92000002080F82A33C0F8847147600296C5F869
:10C930001066D5F810360293029BD8F80030012B10
:10C94000FBD0D9F8000015B0BDE8F08F4CF20E0016
:10C9500015B0BDE8F08F4CF2090015B0BDE8F08FBE
:10C960004CF20E00704700BFB81C02207416022063
:10C9700000A0024010A6024014A6024090A502406A
:10C980000050004000E100E06C1602207816022002
:10C99000701602207C160220681602202DE9F0474E
:10C9A0004FF48065A94C86B0C4F88450BFF34F8F14
:10C9B000BFF36F8FA64EC4F88451D6F80C331F0610
:10C9C00069D4A34BD3F80C23D00775D4D3F80C2328
:10C9D00012F0400259D1D3F80C13490741D59D4FAD
:10C9E0003968012900F0C9809B4BDFF894821F68E9
:10C9F0003A6872B300210C4602E00134944226D218
:10CA000007EBC405AB68002BF7D06E68F6B2012EB9
:10CA1000F3D16868B8F80030B3EB104FEDD16A6815
:10CA2000013322F0FF0242F002026A60A868A8F80F
:10CA30000030FFF771FE314628B96B6823F0FF0321
:10CA400043F003036B603A6801349442D8D3002961
:10CA5000CFD100217E4A814BC2F808111B68039395
:10CA6000039B7B4BD3F80C33DB0643D44FF480613C
:10CA70007B4B764A1B685B01DBB282F82A33C2F833
:10CA80008411516006B0BDE8F0870622714B1A6030
:10CA900006B0BDE8F087FFF76BFCFFF7D7FD002875
:10CAA00066D1704BC6F81C011B680193019B684B53
:10CAB000D3F80C23D00789D500216B4AC3F80011A5
:10CAC000126803240292029AD3F814366149A3F53E
:10CAD0000043013B022B8CBF0323644A0C6098BFC8
:10CAE00052F82330624A1846136006B0BDE8F0479A
:10CAF000FFF702BA5F4BDFF888811F683A6872B3AC
:10CB000000210C4602E00134944226D207EBC40512
:10CB1000AB68002BF7D06E68F6B2012EF3D16868CF
:10CB2000B8F80030B3EB104FEDD16A68013322F052
:10CB3000FF0242F002026A60A868A8F80030FFF71E
:10CB4000EBFD314628B96B6823F0FF0343F0030384
:10CB50006B603A6801349442D8D30029CFD10021C8
:10CB60003B4A454BC2F810111B680493049B7DE7B8
:10CB7000E02384F82A3365608AE73849C3F808213E
:10CB80003E4A0B681268059393683A48324903603D
:10CB9000D2F80480059AC1F800808BB1B8F1000F7B
:10CBA0000ED01B68102B03D8D8F80010102909D913
:10CBB0004CF2060303222E4918460B603A6094E7B4
:10CBC0001023F7E7DFF8B89059B3002008F1040A02
:10CBD000044602E001348C4221D2E50008EB050353
:10CBE0009A68002AF6D05E68F6B2012EF2D1D3F828
:10CBF00004C0B9F80020B2EB1C4FEBD159680132E8
:10CC000021F0FF0141F0020159609868A9F8002065
:10CC1000FFF782FD68B13046D8F80010DAE7002847
:10CC2000D2D102200E4B4FF48061084A1B68386055
:10CC300021E75AF80530304623F0FF0343F00303A1
:10CC40004AF80530D8F80010C4E700BF00E100E062
:10CC500000A00240701602207416022008A10240B3
:10CC60006C1602201CA1024000A1024044BA01003F
:10CC7000681602207816022010A102407C160220BD
:10CC8000B81C022030B4184B1C6825686DB1A3682D
:10CC9000834227D0002302E08968814219D0013302
:10CCA000DA00AB4204EB0201F6D1104B1C68256898
:10CCB0006DB1A368834215D0002302E089688142E8
:10CCC00007D00133DA009D4204EB0201F6D130BCFB
:10CCD00070470432A35823F0FF0343F00303A3502B
:10CCE00030BC70470422F5E7781602207416022043
:10CCF000002800F0B880002900F0B580002A00F07C
:10CD0000B2802DE9F04F046A85B0002C00F0A680B7
:10CD1000406A002800F0A28042F687454FF0000AE2
:10CD2000554EA84286F800A040F2A0800827DFF800
:10CD30008091204616460D4644225146C9F80040CF
:10CD40000DF09EFDD9F8002004F14403DFF8648162
:10CD500082F801A082F802A082F803A0177018469A
:10CD600044225146C8F800300DF08AFDD8F8002062
:10CD700004F18803DFF840B1177082F801A082F84F
:10CD800002A082F803A018464FF400725146CBF877
:10CD900000300DF075FD394B04F5227CC3F800C05E
:10CDA000514660464FF400720DF06AFD4FF4205C6E
:10CDB00006214FF0010E4FF401304FF48832304B12
:10CDC00004F591645C602F4CC3F808C09981A3F806
:10CDD00000E019461C612C4BDFF8E0C020612B48B5
:10CDE000636003F5C073A060C4F800C02848E36026
:10CDF000626104F09FFA002832D14FF0020C202427
:10CE0000D9F80010DBF8002029601C4BD8F800107E
:10CE1000DFF8ACE01F4D3160CEF800201B681E49E2
:10CE200002F500722A601D4E1D4A1E4D0B6003F56F
:10CE300000731D4933602880C2F814C509681B4B74
:10CE400003910399C2F81C7519683B440291029939
:10CE5000C2F824451B680193019B01E04CF20700D6
:10CE600005B0BDE8F08F4CF20E0070474CF20400A4
:10CE700005B0BDE8F08F00BFC9200220A81602202F
:10CE800094160220B816022080000400000104005D
:10CE9000801602208C16022088160220841602209A
:10CEA00000A00240BA1C022014A502401CA50240AA
:10CEB000B4160220AC160220B01602204000080072
:10CEC0009016022000285ED070B4334B83B01A68ED
:10CED000324B82421ED81B6831498342096803D80D
:10CEE000304C2468844246D881420ED92E4B1B78A0
:10CEF000002B4BD1831A2D499E099B060A682C4CA6
:10CF00004FF003014FF0020514D04CF2100003B0B3
:10CF100070BC70471B689842F7D3224A126890424F
:10CF2000F3D20121C31A234A9E099B060D461268BB
:10CF3000214CEAD14368DBB29D421FD1202002EB95
:10CF4000C60253681D4D03F47F432E8843F001034E
:10CF500043EA0643536000BF0138FCD10122184B5D
:10CF600043F8212022682B880192019A01332B80FB
:10CF700003B070BC70478142D3D9B7E74CF20700C9
:10CF800003B070BC70474CF20E0070474CF20F00BB
:10CF900003B070BC704700BF9016022088160220B4
:10CFA0008C16022084160220C9200220B41602200A
:10CFB0000CA00240AC16022004A00240BA1C0220C1
:10CFC00000A00240184B1B7863BBF0B4174A03F073
:10CFD000FF001468164B25681E68A5B10746C100FE
:10CFE00063185A68D2B2032A04D19F605A6822F0AB
:10CFF000FF025A605A6812F0FF0F01D19B682BB1F3
:10D000000130A842EBD10020F0BC704706EB801045
:10D0100021448860436823F0FF0343F00203436028
:10D02000F0BC704700207047C9200220B4160220CF
:10D03000B0160220F0B4154A154B14681E68256816
:10D04000ADB100200746C10063185A68D2B2032A66
:10D0500004D19F605A6822F0FF025A605A6812F0A9
:10D06000FF0F01D19B682BB101308542EBD100202D
:10D07000F0BC704706EB801021448860436823F0C1
:10D08000FF0343F001034360F0BC7047AC1602207D
:10D09000A8160220034B1B780BB904F08FBA0020AE
:10D0A000704700BFC92002200B7870B50646EBB16F
:10D0B000084600240A46202B154612D0137001346E
:10D0C00010F8013F0A191546002BF4D10024084638
:10D0D0002C700DF099FA064B53F826305860204614
:10D0E00070BD10F8013F002BE5D1EFE70D46EDE7ED
:10D0F000D41702200B7870B50646EBB10846002421
:10D100000A46202B154612D01370013410F8013F47
:10D110000A191546002BF4D10024084B2C70084640
:10D1200053F826500DF070FA2860204670BD10F8B4
:10D13000013F002BE5D1EFE70D46EDE7D4170220C4
:10D1400008B58022002102480DF09AFB002008BD9E
:10D15000D4160220F0B51F4C83B006461E49204667
:10D160000DF0EBFA10BB05460146802220460DF07B
:10D1700087FB1A4B0195186880222B4600952146A3
:10D1800004F0FCFD074616480DF002FB87420546F9
:10D1900014DB0246214612480DF00FFB70B93046F1
:10D1A000611903B0BDE8F040FFF7CABF20468022F6
:10D1B00000210DF065FB002003B0F0BD09480DF023
:10D1C000E7FA0449024607480DF0F7FA4FF0FF303E
:10D1D000F2E700BFD416022050BA0100D016022098
:10D1E00040BA010058BA0100F0B51C4C83B080224F
:10D1F0000021064620460DF043FB0023184A214635
:10D200001068CDE90033802204F0B8FD07461548C8
:10D210000DF0BEFA874218DB05460246214611484A
:10D220000DF0CBFA88B961193046FFF73DFF30B1F8
:10D230000D4B53F826301A685A6003B0F0BD3046E3
:10D2400003B0BDE8F040FFF785BF08480DF0A0FA35
:10D250000249024605480DF0B0FAE9E7D41602206B
:10D26000D016022060BA0100D417022058BA01007B
:10D270004FF0FF3310B5094C2822002108482360E5
:10D280000DF0FEFA40F201220021662004F0E4FCD9
:10D2900000282060B4BF0320002010BDD01602205B
:10D2A000D41702202DE9F041662882B040F0CA80F0
:10D2B000B1F5007F40F0AD8040F202239A4240F089
:10D2C000A880634C25684DB36368002B00F09D80F7
:10D2D000A368002B00F09B80E368002B00F09F8088
:10D2E0002369002B00F09D806369002B00F0A6806D
:10D2F000A369002B00F0A480E369002B00F0938069
:10D30000236A53B1636A092543B10C200DF099FBE0
:10D310004FF0FF3002B0BDE8F0810825782004F01E
:10D3200023F944F825000028EFD0782200210DF0E1
:10D33000A7FA012103264FF0FF3054F82530802250
:10D34000996054F8253000211E67586041480DF05F
:10D3500097FA414F414A80213E48FDF757FC3D482E
:10D36000D7F8008000260DF013FA334602463949FB
:10D3700040460196009604F01FFC804635480DF0AB
:10D3800007FA404521D1DFF8E0803146802240464F
:10D390000DF076FA38683346CDE9006641468022C2
:10D3A00004F0ECFC07462E480DF0F2F987420646E1
:10D3B0003BDB024641462A480DF0FFF9A8BB08EBCB
:10D3C00006012846FFF796FE78B154F8250004F0D0
:10D3D000E9F87822002154F825000DF051FA0023D5
:10D3E0004FF0FF3044F8253094E72846FFF7B2FEAF
:10D3F0000028EAD1022254F8253045F0F14040F4EB
:10D40000D0109A6002B0BDE8F081012586E70225C0
:10D4100084E716200DF015FB4FF0FF307AE7032567
:10D420007CE704257AE7072578E70E480DF0B0F988
:10D430000D4902460B480DF0C0F9C6E705256DE71A
:10D4400006256BE72F200DF0FCFA4FF0FF3061E767
:10D45000D417022054170220D0160220DCBA010093
:10D46000ECBA010058BA0100D41602202DE9F04FA1
:10D4700083B0002900F01E81642A914600F21A81CF
:10D480000446084688460DF083F9642800F21281AC
:10D490008B4BA34340F0068124F0F14424F4D014D4
:10D4A000092C00F3FF80874F57F82430002B00F041
:10D4B000F9809A68002A00F0F580002CC0F2F28012
:10D4C0009B68022B40F0EE807F4E80220021304688
:10D4D0000DF0D6F97D4A80213046FDF797FB57F8CD
:10D4E00024300546C0F180011B68794A3018FDF7E9
:10D4F0008DFB57F8243005441B6F03F00302032A09
:10D5000000F0BD809B074CBF724B734BC5F180018F
:10D510007019724AFDF77AFB0544C5F18001701954
:10D5200043466F4AFDF772FB0544802D00F3BA8035
:10D53000DFF8C4A16448DAF800500DF029F900239F
:10D5400002460193284600935F4904F035FB0546E7
:10D550005D480DF01DF9A84240F0A4802046FFF779
:10D56000F9FD0546002840F09D800146802256487E
:10D570000DF086F95B4A80215348FDF747FB57F8C9
:10D580002430C0F180011B68574A3044FDF73EFB50
:10D590004D48DAF800B00DF0FBF82B460246019535
:10D5A00000954949584604F007FB054646480DF0EA
:10D5B000EFF8A84276D12046FFF7CCFD05460028BB
:10D5C00070D1032157F824304A46996057F8240057
:10D5D00041460C300DF027F9294680223A480DF0DB
:10D5E0004FF9424A80213848FDF710FB57F82430A4
:10D5F000C0F180011B683C4A3044FDF707FB32480C
:10D60000DAF800800DF0C4F82B460246019500952B
:10D610002D49404604F0D0FA05462B480DF0B8F8E5
:10D62000A84202D12046FFF7DFFD802200212648D4
:10D630000DF026F92E4A80212348FDF7E7FA002352
:10D64000C0F180010546224A3018FDF7DFFA57F88D
:10D6500024300544C5F180015B6F1D4A7019FDF748
:10D66000D5FA57F82430291870180C33C1F180010D
:10D670001A4AFDF7CBFA002003B0BDE8F08FC5F1E0
:10D6800080011C4B154A7019FDF7C0FA0544C5F11D
:10D69000800170194346124AFDF7B8FA0544802DFF
:10D6A0007FF746AF09200DF0CCF94FF0FF3003B003
:10D6B000BDE8F08F0E200DF0C4F94FF0FF30DBE72E
:10D6C00000009A78D41702205417022078BA01007B
:10D6D00084BA0100A0BA0100A8BA010090BA010002
:10D6E00098BA0100ACBA0100B8BA0100BCBA010096
:10D6F000CCBA010088BA0100D01602202DE9F04111
:10D70000454B82B083437BD120F0F14424F4D01404
:10D71000092C75DC414D55F82400002870D0836831
:10D72000002B6DD0002C6BDB8368032B0DD003F036
:10D7300039FF7822002155F824000DF0A1F80020CF
:10D7400045F8240002B0BDE8F081354E802200216A
:10D7500030460DF095F8334A80213046FDF756FAF1
:10D7600055F82430C0F180011B682F4A3044DFF89F
:10D77000C080FDF74BFA3046D8F800700DF008F87D
:10D780000023024631463846CDE9003304F014FA4E
:10D79000074630460CF0FCFFB84237D12046FFF771
:10D7A000D9FC074690BB0146802230460DF068F850
:10D7B0001E4A80213046FDF729FA55F82430C0F181
:10D7C00080011B68184A3044FDF720FA3046D8F82B
:10D7D00000800CF0DDFF3B46024601970097314682
:10D7E000404604F0E9F9074630460CF0D1FFB84254
:10D7F0000CD12046FFF7AEFC40B955F8240096E75F
:10D8000009200DF01EF94FF0FF309BE723200DF0AB
:10D8100018F94FF0FF3095E700009A78D4170220EE
:10D82000541702206CBA0100B8BA010078BA01009E
:10D83000D01602202DE9F04140F20224A14202D18B
:10D84000511E012906D916200DF0FBF84FF0FF30CC
:10D85000BDE8F081002BF6D006990029F3D03C49B1
:10D86000814301D00920EFE720F0F14424F4D014E3
:10D87000092CF7DC374D55F824100029F2D08868C0
:10D880000028EFD0002CEDDB022A8A6837D1032A6A
:10D8900056D1069A042AD6D1DFF8C8801B684F6F8C
:10D8A00080224B67404600210CF0EAFF2A4A802183
:10D8B0004046FDF7ABF90123C0F180010646274A37
:10D8C0004044FDF7A3F955F824300644C6F1800121
:10D8D0005B6F224A08EB0600FDF798F955F82430F3
:10D8E000311808EB01000C33C1F180011C4AFDF72F
:10D8F0008DF955F824304FF0FF305F67A4E7FAB197
:10D900008A68032A1CD08A68042A19D0069A9008CB
:10D91000421E012A97D8069A920794D11A68022AC1
:10D9200010D00A2A8FD10222022806D15B68022B6E
:10D930000AD00A2B87D142F002020A67002083E74F
:10D940000E2081E70122EFE742F00102F5E700BF78
:10D9500000009A78D4170220CCBA010084BA0100E2
:10D9600090BA01005417022010B540F20224A142DF
:10D9700002D1511E012905D916200DF062F84FF091
:10D98000FF3010BD002BF7D0029B002BF4D0234BAF
:10D99000834305D009200DF054F84FF0FF3010BD3F
:10D9A00020F0F14020F4D0100928F3DC1C4B53F890
:10D9B0002030002BEED099680029EBD00028E9DB5D
:10D9C0000299022A09689A6803D1032A1FD00E20FF
:10D9D000D3E7002AFBD09A68042AF8D0072901F07F
:10D9E0000302C9D9002AC7D11B6F990703D50A21A1
:10D9F000012202980160DB0704D50223029941F855
:10DA000022300132029B92001A600020B5E70429FF
:10DA1000B2D15B6F029A00201360AEE700009A78E3
:10DA2000D4170220002900F09B83F0B5A24C0228F5
:10DA300083B00D46236800F093800A283ED01BB1C6
:10DA40009B68032B00F0268163681BB19B68032B46
:10DA500000F00F81A3681BB19B68032B00F0F880D6
:10DA6000E3681BB19B68032B00F0E18023691BB1C5
:10DA70009B68032B00F0228163691BB19B68032B19
:10DA800000F06081A3691BB19B68032B00F0498102
:10DA9000E3691BB19B68032B00F03281236A1BB141
:10DAA0009B68032B00F01B81636A1BB19B68032BEF
:10DAB00000F0AC804FF0FF3003B0F0BD1BB19B68AD
:10DAC000032B00F0198363681BB19B68032B00F0E4
:10DAD000E182A3681BB19B68032B00F0BB82E36863
:10DAE0001BB19E68032E00F0D68123691BB19B6891
:10DAF000032B00F0E98163691BB19B68032B00F0E5
:10DB0000FB81A3691BB19B68032B00F00D82E369C5
:10DB10001BB19B68032B00F01F82236A1BB19B681B
:10DB2000032B00F03382636A002BC3D09B68032B66
:10DB3000C0D128460CF02CFE0646606A0C300CF072
:10DB400027FE8642B6D1616A28460C310CF028FEC9
:10DB50000028AFD1636A1A6F9207ABD509261AE184
:10DB60001BB19B68032B00F0E18263681BB19B68CB
:10DB7000032B00F0A982A3681BB19B68032B00F064
:10DB80004F82E3681BB19E68032E00F0EC8023698E
:10DB90001BB19B68032B00F0308163691BB19B684C
:10DBA000032B00F04481A3691BB19B68032B00F099
:10DBB0005881E3691BB19B68032B00F00182236A43
:10DBC0001BB19B68032B00F01382636A002B3FF4A8
:10DBD00071AF9B68032B7FF46DAF28460CF0D8FD26
:10DBE0000646606A0C300CF0D3FD86427FF462AFCB
:10DBF000616A28460C310CF0D3FD00287FF45AAF3F
:10DC0000636A1A6FD2077FF555AFA7E728460CF075
:10DC1000BFFD0646606A0C300CF0BAFD86427FF408
:10DC200049AF616A28460C310CF0BAFD42E728463C
:10DC30000CF0AEFD0646E0680C300CF0A9FD864203
:10DC40007FF414AFE16828460C310CF0A9FD0DE714
:10DC500028460CF09DFD0646A0680C300CF098FD9F
:10DC600086427FF4FDAEA16828460C310CF098FD89
:10DC7000F6E628460CF08CFD064660680C300CF089
:10DC800087FD86427FF4E6AE616828460C310CF0D1
:10DC900087FDDFE608460CF07BFD064620680C3069
:10DCA0000CF076FDB0427FF4CFAE216828460C31EF
:10DCB0000CF076FDC8E600BFD417022028460CF011
:10DCC00067FD064620690C300CF062FD86427FF449
:10DCD000D3AE216928460C310CF062FDCCE6284613
:10DCE0000CF056FD0646206A0C300CF051FD8642C1
:10DCF0007FF4DAAE216A28460C310CF051FDD3E6F0
:10DD000028460CF045FD0646E0690C300CF040FD5D
:10DD100086427FF4C3AEE16928460C310CF040FD29
:10DD2000BCE628460CF034FD0646A0690C300CF029
:10DD30002FFD86427FF4ACAEA16928460C310CF071
:10DD40002FFDA5E628460CF023FD064660690C3041
:10DD50000CF01EFD86427FF495AE616928460C31B9
:10DD60000CF01EFD8EE628460CF012FD0746E0681A
:10DD70000C300CF00DFD87427FF409AFE1682846B6
:10DD80000C310CF00DFD00287FF401AFE3681A6F31
:10DD9000D1077FF5FCAE5868431C7FF48DAEB94DBA
:10DDA0008022002128460CF06BFDB74A80212846CE
:10DDB000FCF72CFF54F82630C0F18001B34A1B68F1
:10DDC0002844FCF723FFB24B28461F680CF0E0FC08
:10DDD0000023024629463846CDE9003303F0ECFE25
:10DDE000074628460CF0D4FCB84202D13046FFF773
:10DDF000FBF954F8263058685EE628460CF0C8FC5B
:10DE0000064620690C300CF0C3FC86427FF4C5AE98
:10DE1000216928460C310CF0C3FC00287FF4BDAE0C
:10DE200023691A6FD2077FF5B8AE0426B3E72846F8
:10DE30000CF0AEFC064660690C300CF0A9FC864282
:10DE40007FF4B1AE616928460C310CF0A9FC0028C2
:10DE50007FF4A9AE63691A6FD7077FF5A4AE0526D4
:10DE600099E728460CF094FC0646A0690C300CF0AB
:10DE70008FFC86427FF49DAEA16928460C310CF0E0
:10DE80008FFC00287FF495AEA3691A6FD6077FF543
:10DE900090AE06267FE728460CF07AFC0746E0683D
:10DEA0000C300CF075FC87427FF41FAEE168284609
:10DEB0000C310CF075FC00287FF417AEE3681A6F84
:10DEC00091073FF568AF10E628460CF061FC064666
:10DED00020690C300CF05CFC86427FF40CAE2169AA
:10DEE00028460C310CF05CFC00287FF404AE23695A
:10DEF0001A6F920799D4FEE528460CF049FC0646B5
:10DF000060690C300CF044FC86427FF4FAAD616924
:10DF100028460C310CF044FC00287FF4F2AD636914
:10DF20001A6F97079BD4ECE528460CF031FC0646A7
:10DF3000A0690C300CF02CFC86427FF4E8ADA1699E
:10DF400028460C310CF02CFC00287FF4E0ADA369CE
:10DF50001A6F96079DD4DAE528460CF019FC0646A0
:10DF6000E0690C300CF014FC86427FF4D6ADE16918
:10DF700028460C310CF014FC00287FF4CEADE36988
:10DF80001A6F90077FF5C9AD072604E728460CF005
:10DF9000FFFB0646206A0C300CF0FAFB86427FF449
:10DFA000C2AD216A28460C310CF0FAFB00287FF440
:10DFB000BAAD236A1A6F91077FF5B5AD0826EAE678
:10DFC00028460CF0E5FB0646E0690C300CF0E0FB5F
:10DFD00086427FF4F4ADE16928460C310CF0E0FB99
:10DFE00000287FF4ECADE3691A6FD007CCD4E6E5E6
:10DFF00028460CF0CDFB0646206A0C300CF0C8FB1E
:10E0000086427FF4E2AD216A28460C310CF0C8FB51
:10E0100000287FF4DAAD236A1A6FD107CED4D4E595
:10E0200028460CF0B5FB0646A0680C300CF0B0FB9F
:10E0300086427FF4A6ADA16828460C310CF0B0FBF7
:10E0400000287FF49EADA3681A6FD0077FF599ADC5
:10E050000226A0E628460CF09BFB0646A0680C3082
:10E060000CF096FB86427FF43AADA16828460C314D
:10E070000CF096FB00287FF432ADA3681A6F90076E
:10E08000E6D42CE554170220BCBA0100B8BA01004E
:10E09000D016022028460CF07BFB064660680C3048
:10E0A0000CF076FB86427FF414AD616828460C3193
:10E0B0000CF076FB00287FF40CAD63681A6F9607AE
:10E0C0007FF507AD012666E628460CF061FB0646A3
:10E0D00060680C300CF05CFB86427FF44CAD6168EC
:10E0E00028460C310CF05CFB00287FF444AD6368DB
:10E0F0001A6FD607E6D43EE508460CF049FB064603
:10E1000020680C300CF044FB86427FF4DCAC2168C4
:10E1100028460C310CF044FB064600287FF4D3ACB3
:10E1200023681A6F97073FF536AECCE408460CF02B
:10E130002FFB064620680C300CF02AFB86427FF449
:10E1400014AD216828460C310CF02AFB0646002845
:10E150007FF40BAD23681A6FD7073FF51CAE04E5BB
:10E160004FF0FF30704700BF10B50446006803F061
:10E1700011FFA06818B1BDE8104003F013BA10BD3C
:10E180000E289ABF024B53F820002D20704700BF85
:10E19000F8BA010070B5002582B002AC44F8045D05
:10E1A00006460D4620461946144603F0C1FE60B9E6
:10E1B000019B082258729872D872184644EA0644A5
:10E1C000DC601D611A7202B070BD019B184602B07E
:10E1D00070BD00BF70B50C460546114620461E4670
:10E1E00003F0BAFE00B970BD206808B103F0D2FE9A
:10E1F000204603F0C7FE2E60232070BD38B50546CB
:10E2000001F08CFA044608B1204638BD284601F0DA
:10E21000F5FA0028F8D04468002CF5D000234360BC
:10E22000204638BD38B50023074D084C194620223A
:10E2300007482B6023600CF023FB03F073FE0030D3
:10E2400018BF0120404238BD0C18022008180220D7
:10E250001418022000232DE9F04120F0080682B0B6
:10E26000022E009340F088804B1E012B0C4656D89E
:10E270000746002A4FD1012908BF0126414A2146FD
:10E28000684601F0B5F9009B8046002B50D0002174
:10E2900002A840F8041DC3E902741E6103F048FEA1
:10E2A000002842D147F201024FF0FF330821019DBF
:10E2B00042EA0842EA606872A872E87229722B7416
:10E2C0006B74AB74EB740A2F0CBF02220122AB6893
:10E2D000EE610C33AC616A61AB6047F20101284624
:10E2E000009F03F039FE064638B3286808B103F0F2
:10E2F00051FE284603F046FE012323253B6040469D
:10E3000001F0CAF928460CF09CFB4FF0FF3840465C
:10E3100002B0BDE8F08101290CD0022AAED016204F
:10E320000CF08FFB4FF0FF38F1E7019D002DCAD1B3
:10E330000C25E4E7012AA1D0F1E74FF0FF334FF6B7
:10E34000FF720221404601F0E9F905460028D6D1C6
:10E35000404601F053FA18B145680DB14660CEE76A
:10E36000022CD4D1009B1A6842F400321A601A6859
:10E3700042F400221A60CAE72F200CF062FB4FF033
:10E38000FF38C4E769E100002DE9F04182B006469C
:10E3900001F034FA002863D00446002102A827685F
:10E3A00040F8041DD4F8148003F0C2FD00283AD1CF
:10E3B00047F209030822019D43EA0643EB60C5F8D2
:10E3C00010806872A872E8722A72236847F2090105
:10E3D0001B0C1B0443F00D0323602368284623F421
:10E3E00000332360236823F40023236003F0B4FD8B
:10E3F00040BB4FF0FF334FF6FF720E21304601F065
:10E400008DF90446A0B1174C54F8260020B103F052
:10E41000B9FD002344F82630304601F03DF90020D4
:10E4200002B0BDE8F081019D0C20002DCDD112E09D
:10E43000304601F0E3F90028E5D04368002BE2D034
:10E440004460E0E7286808B103F0A4FD284603F023
:10E4500099FD232027600CF0F4FA4FF0FF30DFE73E
:10E460000920F8E7141802202DE9F043002483B0B6
:10E47000884617469946019405460A9E01F0BEF962
:10E48000002800F0C080C3680446012B5CD02268DD
:10E49000910340F1A680394601A803F049FD002808
:10E4A00040F0AB800C22019B1A7258729872D8729D
:10E4B000EEB1A26871688A4208D1022A03F11C00F9
:10E4C000317845D00A2A01D1242968D0186810B1C2
:10E4D00003F060FD019B184603F054FD16200CF07C
:10E4E000B0FA4FF0FF36304603B0BDE8F08347F294
:10E4F00006021646C3F81490616942EA0542DA60E2
:10E5000019615F60B8F1000F04D03A4641461868BF
:10E510000CF089F927682368314623F4003323601F
:10E52000236843F480132360019E304603F014FDFA
:10E530008046C0B1306808B103F02CFD304603F0CE
:10E5400021FD27602320CAE7002EA0D01620C6E7B1
:10E550001029BBD1042231895A83198306F10C0199
:10E560000CF061F922E04FF400324FF0FF33114616
:10E57000284601F0D3F840B1236843F40033236008
:10E58000236823F480132360A9E7284601F036F9B5
:10E590000346B8B14068A8B1C3F80480ECE7102284
:10E5A00031895A831983B1180CF03DF947F20702FB
:10E5B000019B16469968588B04310144C3F81490A6
:10E5C000996099E7236823F4801323600F4C54F873
:10E5D000253018469E6903F0D5FC002344F8253009
:10E5E00081E72268D2000AD4022B0AD023689BB2AA
:10E5F000052B0CBF2320392071E70C206FE7392051
:10E600006DE723206BE7092069E700BF141802209B
:10E610002DE9F04F85B00F9D002A00F0C3808A4697
:10E6200098468146164601F0E9F80446002800F0B5
:10E63000BC8003681A031FD403689BB2062B00F04A
:10E64000AE8003689BB2072B0CBF4FF0090B4FF055
:10E65000390BA0690368DB689847013003D0236851
:10E6600043F48033236058460CF0EBF94FF0FF354C
:10E67000284605B0BDE8F08F18F0020F09BF076803
:10E68000002787F00067C7F3C06718F0100F47D165
:10E690002368DB0324D52368A06923F48033236037
:10E6A0000368DB68984701301AD005B12D680E9BCE
:10E6B000CDE900A6CDE90235A06942460368694666
:10E6C0009B689847431C05465CD0A0690368DB68DB
:10E6D00098470130CCD0236843F480332360C7E7E8
:10E6E000002F33D14FF0230BB3E723681A01DCD49A
:10E6F0004FF48032E3691146002B08BF4FF0FF331F
:10E70000484601F00BF883460028A2D1484601F0A4
:10E7100075F820B1D0F804B0BBF1000F2FD101275C
:10E720002368D8030FD52368A06923F480332360BE
:10E730000368DB689847411C05D08642B5DDE36875
:10E74000012BB2D1D1E7002FCCD0D1E74FF48032EA
:10E75000E3691146002B08BF4FF0FF33484600F035
:10E76000DDFF834600287FF474AF484601F046F889
:10E7700000288DD0D0F804B0BBF1000F88D0002362
:10E78000436066E7A0690368DB68984701300FD0F3
:10E7900023684FF0230B43F48033236063E74FF08B
:10E7A000090B56E74FF0160B5DE74FF0090B5AE7E0
:10E7B0004FF0230B57E700BF2DE9F04182B000294D
:10E7C00043D0002A41D006460F4601F017F805460F
:10E7D000002800F0928003689BB2022B04D00368EB
:10E7E0009BB2042B40F08980296811F0805178D1C8
:10E7F00002A840F8041DD5F8148003F099FB70BB03
:10E8000008213304019C43F4E04242F00202E2603A
:10E81000C4F810806072A072E072217243F4E04389
:10E8200043F00203E360A3686A6904332261A360D2
:10E83000AB687A68934208D1022B04F118003A7849
:10E8400035D00A2B01D1242A0ED0162420460CF0F4
:10E85000F8F84FF0FF34204602B0BDE8F081019C8B
:10E86000002C4CD03304D9E710223B89B918E2823E
:10E87000A3820BF0D8FFA368E28A47F20201134497
:10E88000A360D5F800802B68204643F080532B60AE
:10E8900003F062FB0746A8B1206808B103F07AFBD9
:10E8A000204603F06FFB2324C5F80080CEE7102A32
:10E8B000CBD104223B8907F10C01E282A3820BF049
:10E8C000B2FFD8E74FF0FF334FF6FF720521304615
:10E8D00000F024FF044630B1732CB7D0C5F8008097
:10E8E000B4E77224B2E7304600F088FF0028B2D0C7
:10E8F0004468002CAFD04760EEE70924A6E70C245B
:10E90000A4E700BF2DE9F04182B089B382B3074686
:10E910000E4600F073FF054600287BD003689BB2CB
:10E92000022B77D1002102A840F8041DD5F81480ED
:10E9300003F0FEFA30BB47F205030822019C43EACC
:10E940000743E360C4F810806072A072E072227224
:10E95000A3680433A360AB687268934208D1022BAA
:10E9600004F1180032783CD00A2B01D1242A0ED0B1
:10E97000162420460CF065F84FF0FF34204602B014
:10E98000BDE8F081019C002CE2D10C24F1E71022BB
:10E990003389B118E282A3820BF045FFA368E28AB3
:10E9A00047F205011344A3602B6820461B0C1B048F
:10E9B00043F003032B602E6803F0CEFA8046D8B9EB
:10E9C0004FF0FF334FF6FF720421384600F0A6FEE9
:10E9D000044608B32B681B0C1B0443F002032B6096
:10E9E000C7E7102AC4D10422338906F10C01E28260
:10E9F000A3820BF018FFD1E7206808B103F0CAFA30
:10EA0000360C3604204646F0020603F0BBFA2324F7
:10EA10002E60AEE70924ACE7384600F0EFFE002890
:10EA2000ACD04468002CA9D0C0F80480D2E700BF65
:10EA30002DE9F04182B0064600F0E0FE002867D0E4
:10EA4000036805469BB2042B62D10021324A30464E
:10EA500000F036FE014600285CD102A840F8041DF3
:10EA60006F6903F065FAA8BB47F208030822019C0E
:10EA700043EA0643E36027616072A072E07222728B
:10EA8000A36847F208010433A3602B6820461B0CDF
:10EA90001B0443F006032B602F6803F05DFA8046E9
:10EAA000E8B94FF0FF334FF6FF720721304600F010
:10EAB00035FE044608B32B681B0C1B0443F004030B
:10EAC0002B6020460BF0BDFF4FF0FF34204602B014
:10EAD000BDE8F081019C002CD2D10C24F1E7206824
:10EAE00008B103F057FA3F0C3F04204647F00407F3
:10EAF00003F048FA23242F60E3E7304600F07EFE5F
:10EB00000028E3D04468002CE0D0C0F80480D2E7AD
:10EB10000924D6E72324D4E769E100002DE9F04F6A
:10EB2000002585B00F4690460295064600F066FE29
:10EB30000446002800F01C8103689BB2072B0AD111
:10EB4000036805681B0116D415F4803519D00568D3
:10EB500015F4803524D14FF00909029B13B12846E2
:10EB600000F09AFD48464FF0FF390BF06AFF484627
:10EB700005B0BDE8F08F15F480356DD14FF0230955
:10EB8000EBE74FF480324FF0FF331146304600F090
:10EB9000C5FD814600287ED0256815F48035DCD07F
:10EBA0004FF0FF300023CDE90003754AE16802A869
:10EBB00000F01EFD029B0546002B00F0DD800021C9
:10EBC000226904A81A61A26840F8041D9A60E268EC
:10EBD000DA60D4F8149003F0ABF9002843D147F27F
:10EBE0000C030821DDF80CB043EA0643CBF80C30E7
:10EBF000CBF810908BF809008BF80A008BF80B000B
:10EC00008BF80810236847F20C011B0C1B0443F01F
:10EC1000080323605846D4F8009003F09DF982461B
:10EC200048BB226800994FF0FF330A402260092157
:10EC30004FF6FF72304600F071FD8146002800F06B
:10EC400085802368019A1A43226023681B0C1B04E9
:10EC500043F00703236080E76FF000624FF000632A
:10EC6000CDE90023A1E7DDF80CB04FF00C09BBF1B2
:10EC7000000FC7D171E7DBF8000008B103F08AF993
:10EC80004FEA194958464FEA094903F07BF949F020
:10EC90000703236072E7304600F0B0FD30B1D0F8D2
:10ECA0000490B9F1000F01D0456075E72368D903DE
:10ECB0003FF576AF334D029955F826309B694B618D
:10ECC00047B18B680A2B24D0022B03D1D8F800203F
:10ECD000102A32D00A682C48024042F005020A602D
:10ECE000029A116841F400311160116841F4002169
:10ECF00011602368034043F00703236055F82600A2
:10ED000003F040F90023484645F8263005B0BDE839
:10ED1000F08FD8F80020242ADCD13A7010227B60D2
:10ED200055F8263007F110009B8B3B8155F82610D3
:10ED300020310BF078FD0299CCE73A707B6055F8F2
:10ED4000263007F10C009B8B0422EEE7304600F0E2
:10ED500055FD38B1D0F80490B9F1000F02D0C0F8D9
:10ED600004A06EE72368019AA94613432360A1E734
:10ED700005464FF00909F0E64FF00C09F2E600BF36
:10ED800069E10000141802200000FFFF2DE9F041A6
:10ED9000012982B040F0988015461E46074600F0D3
:10EDA0002DFD0446002800F09580142D6ED0192DFD
:10EDB00062D1002E00F0908030460BF0E9FC089BF9
:10EDC000984240F0898023689BB2022B40F08280F9
:10EDD0003146A068FEF726FE009001307ED0236801
:10EDE0009A025ED423685B025BD400222668236803
:10EDF00002A843F400132360042140F8042DD4F842
:10EE0000148003F095F8002858D147F20303082234
:10EE1000019D43EA0743EB60C5F810806872A87251
:10EE2000E8722A724FF0080C002310203021AA68E3
:10EE30006B756244AA60AB75EB75AB76EB7685F8C3
:10EE400014C0287669760422694628680BF0EBFC2A
:10EE500047F20301284603F07FF8804618BB4FF4C1
:10EE600080024FF0FF331146384600F057FC05464C
:10EE7000002835D0266000E02A2528460BF0E1FD69
:10EE80004FF0FF35284602B0BDE8F08126B3089B5D
:10EE9000042B23D100253368C361284602B0BDE8A6
:10EEA000F0812325E9E7286808B103F073F82846C4
:10EEB00003F068F8232526602660DEE7019D002D1B
:10EEC000B0D126600C25D8E72A200BF0BAFD4FF010
:10EED000FF35D7E70925D0E70E25CEE71625CCE785
:10EEE000384600F08BFC20B1456815B1C0F80480AD
:10EEF000C0E72660C6E700BF00F0A0BC2DE9F04FD8
:10EF00004FF0000C01246C4EDFF8B8A1DFF8B89187
:10EF100085B0074615460193A6F800C0CAF8004020
:10EF2000C9F8004071B108460A2261460BF08FFB18
:10EF30004FF6FE73421E9A4200F28680030243EAB5
:10EF400020203080DFF88481D8F80030002B77D182
:10EF50005A4A13605A4A1360002F65D038460BF0A6
:10EF600017FC834625B1EA6912B1516866296FD052
:10EF70004FF0FF32002104AE46F8041D30465946DA
:10EF8000009202F0D5FF009A00284FD147F20D0100
:10EF90004FF0080C039C41EA0241E160226160727B
:10EFA000A072E07284F808C0002D6AD06A6822F06E
:10EFB000080102296ED1A968022908BFCAF8001009
:10EFC0000A2A14BF01220222A261EA68C9F80010CD
:10EFD0002262AA68E2612A686261A2681032A260B5
:10EFE0002FB1206818B15A4639460BF01CFC01239A
:10EFF00047F20D012046C8F8003002F0ADFF0028AE
:10F0000046D14FF0FF33039331462046FBF782FE93
:10F01000D8F80030012BF7D0294B186860BB274B7C
:10F02000019A1B6813600CE0BB469BE7039C002C15
:10F03000BAD10C200023C8F8003005B0BDE8F08F2D
:10F04000732005B0BDE8F08F162005B0BDE8F08F45
:10F050009168B1F5007F8BD140F20221D0688842DF
:10F0600086D19169002983D06868FEF7DBFC431CD8
:10F070003FF47EAF02467DE7114B18680028E0D0D0
:10F08000D8E72946102204F114000BF0F9FBA4E79D
:10F090002320CFE72F200BF0D4FCA2681032A2600F
:10F0A00017B94FF0FF30C5E720680028F9D05A465D
:10F0B00039460BF0B8FBF4E7BC1C02200C18022008
:10F0C00004180220FC170220001802200818022051
:10F0D00038B50B4C2368022B00D038BD30B1054643
:10F0E000406902F05FFA284602F05CFA0023054A04
:10F0F0000549236013600868BDE8384002F04ABF44
:10F100000818022004180220101802202DE9F04FE0
:10F1100001F41043B3F5104F054689B00E46C068A0
:10F120004ED0040C204600F069FB48F20D039E42CD
:10F130000746A04631D0002F3ED0404633462A46EF
:10F14000394603F0E9FA98B348F207039E4252D8D1
:10F1500048F206039E4280F0528148F202039E422A
:10F1600000F0248178D948F203039E4200F05F81C9
:10F1700048F205039E421FD13B689BB2032B17D177
:10F180006B69002B00F0E4810E2B00F29381B84AEA
:10F1900052F823307B6000200BE0DFF8EC922F6800
:10F1A000D9F80030012B15D017B1384602F0F2FE25
:10F1B000002009B0BDE8F08F28680028F6D1F7E7F5
:10F1C00000F0D4FA804600F019FB07464446002FB1
:10F1D000B3D1F1E76B69002B4DD00E2B96BFA44A3B
:10F1E0002D2152F823100223A24A1160C9F80030E1
:10F1F000002FDAD1DCE748F20C039E4200F02481B4
:10F2000017D848F208039E4200F0E98048F209034B
:10F210009E42D1D13B689BB20D2BC9D168690028B1
:10F2200000F09E810E2800F24581914B53F820306A
:10F23000B0E749F201039E4200F09B8049F20203CD
:10F240009E42B9D13B689BB2072BB1D13B680020ED
:10F2500043F480333B60ACE748F201039E42ABD1FC
:10F260003B68012BA4D168690028DBD102233B60F5
:10F27000AB697B619DE7804B1F60AC6963011846F9
:10F28000039302F071F90290002800F00381E50079
:10F290002819800002F068F9002800F00D81002C88
:10F2A0005FD005F1100283180193029B0424DFF85C
:10F2B000DCA1DFF8DCB100F1100803F120061DE04D
:10F2C0000A2248F80C2C4FF02402404608F8102C73
:10F2D00028F8083C56F8102C0BF0A5FA56F8103C0C
:10F2E00008F108081C443B1946F8083C019B46F805
:10F2F000046C43452C4406F120062CD03B593A19A6
:10F3000046F8203C5368DAF80010022B14BF0220A4
:10F310000A20DBF8003046E9070146F8143C108A61
:10F32000A8F1100346F8100C558A46F80C3C534BD4
:10F330001434042807EB04011B88C1D110220220D9
:10F3400028F8083C48F80C0C08F8102C56F8102C3B
:10F35000A8F10400C0E70022DDE902130B4443F8E2
:10F36000042C0222464BC9F80020029A00201A60A1
:10F370001FE73C6814F4002400F0A280AB68042B63
:10F3800000F2FC80002329686A68CDE90633CDE9E4
:10F390000412B86904A903685B689847013000F05B
:10F3A000D3803B6843F480333B6001E73B68D8007F
:10F3B0007FF5FEAE3B6823F080533B606869002810
:10F3C00000F097800E288EBF2D23294B53F8203054
:10F3D00000207B603B6843F480233B60E9E63B68A8
:10F3E0009BB2062B7FF4E4AE686900287FF41AAF65
:10F3F0003B681B0C1B0443F007033B60D9E63B68EA
:10F40000D9027FF5D5AE6B69002B5ED13B6843F422
:10F4100000333B603B6823F080633B603B681A012C
:10F420003FF5C6AE174B012043F82450C1E63B68B8
:10F430009B027FF5BDAE686900287FF4F3AE3B68A0
:10F4400043F480033B60B4E63B689BB2082B7FF437
:10F45000AFAE6B69002B7FF497AE0A4B012043F8E7
:10F4600024503B681B0C1B0443F009033B60A0E6DF
:10F47000F8BA01000418022010180220BC1C022057
:10F480000C1802201418022008180220001802206C
:10F49000FC17022002F086F80C2002234B494C4A4C
:10F4A00008602F6802991160C9F80030002F7FF4BE
:10F4B0007CAE7DE62D236DE60C22444B1A6050E7AE
:10F4C000286802F067FD204673E60E2B8EBF2D23C1
:10F4D000404A52F823307B603B6843F480233B6012
:10F4E0006B696B2B3B6842D023F0806300203B604C
:10F4F0005FE63B6843F400333B603B6843F4002322
:10F500003B603B681B0C1B0443F005033B6050E66B
:10F5100002231026436006702B8A05F11401038133
:10F520000C300BF080F96B682A68CDE90646CDE90E
:10F530000423B86904A903685B68984701307FF425
:10F5400030AF204602F02EF8286802F023FD2FE6A7
:10F550003B6800201B0C1B0443F004033B6028E6BF
:10F560003B681B0C1B0443F00E033B6021E613F0C9
:10F57000806319D00C2300207B601AE66B8A002B75
:10F580003FF400AF242001F0EFFF04460028DBD059
:10F590006A8A102A0ED0042ABAD0286802F0FAFC2F
:10F5A000204601F0FFFF03E63A68184642F0806209
:10F5B0003A60FEE50A232426436006702B8A05F193
:10F5C0001401038110300BF02EF9ACE7041802206F
:10F5D0000C180220F8BA010008B54FF4807200211F
:10F5E00002480BF04DF9002008BD00BFCC200220DE
:10F5F000F8B5284B06461D680846E5B11C6A002C84
:10F600003BD01C6C002C3AD01C6E002C39D0D3F8A7
:10F61000801079B1D3F8A010A9B3D3F8C010A1B36A
:10F62000D3F8E01099B34FF0FF350C200BF009FA36
:10F630002846F8BD04254FF0010C4FF0FF376C0150
:10F6400043F804C01C4411466761224602F074F975
:10F650000346A06158B11B681B68984710B9346015
:10F660002846F8BDA06902F085F90023A361204671
:10F67000202200210BF004F9D5E70125DBE7022564
:10F68000D9E70325D7E70525D5E70625D3E70725DD
:10F69000D1E700BFCC200220072800D9704710B561
:10F6A000064C04EB4014A06908B102F063F920464F
:10F6B000BDE81040202200210BF0E2B8CC2002204F
:10F6C00007282DE9F04118D8134D44012B592F1963
:10F6D0009BB1084611463A46D7F8188002F02CF93B
:10F6E000B861B8B103681B689847064648B94046F8
:10F6F00002F040F93046BDE8F08105263046BDE80D
:10F70000F081B86902F036F92819C0F8188030463F
:10F71000BDE8F0810426F7E7CC200220F0B5124EB8
:10F720004001345883B014408C42019306EB00072B
:10F7300013D07B688BB933581B0111D40D46144686
:10F740003E4606E0736843B901A93846FBF7E2FA82
:10F7500020B933682340AB42F4D1002003B0F0BDA0
:10F76000732003B0F0BD00BFCC200220224B1A68EA
:10F7700012B15A69824231D01A6A12B15A6B82426E
:10F780002ED01A6C12B15A6D82422BD01A6E12B161
:10F790005A6F824228D0D3F880201AB1D3F894202F
:10F7A000824223D0D3F8A0201AB1D3F8B4208242E9
:10F7B0001ED0D3F8C0201AB1D3F8D420824219D079
:10F7C000D3F8E0203AB1D3F8F430834214BF4FF0BD
:10F7D000FF30072070474FF0FF3070470020704720
:10F7E00001207047022070470320704704207047B3
:10F7F0000520704706207047CC200220072807D834
:10F80000044B40011A581844002A08BF00207047D2
:10F8100000207047CC20022019B1072802D9082304
:10F820000B607047044B40011A58002AF7D01B5850
:10F83000C3F302430B607047CC20022070B5072849
:10F84000049D1FD8124C400126580444D6B101290A
:10F8500012D1042A10D14BB145B12A68042A05D12E
:10F860000022616810461960626070BD16200BF0BE
:10F87000E8F84FF0FF3070BD2A200BF0E2F84FF0AF
:10F88000FF3070BD09200BF0DCF84FF0FF3070BD89
:10F89000CC200220072810B516D8114C4301E0589F
:10F8A00090B1012905D0022914D1E058C0F3C060FD
:10F8B00010BD12F00100E2581ABF002042F00062B1
:10F8C00022F00062E25010BD09200BF0BAF84FF0B0
:10F8D000FF3010BD16200BF0B4F84FF0FF3010BD14
:10F8E000CC2002202DE9F0412E4CFBF7ADFA032786
:10F8F0002D4D2E4E04F1800802E0083444453BD0E3
:10F9000014F8043C022BF8D120682988026892B2CE
:10F91000914233D0298A914232D0298C91421CD015
:10F920002B8E93422ED0B5F8403093422FD0B5F8AD
:10F93000503093422DD0B5F8603093422BD0B5F8BB
:10F940007030934229D0B5F88030934227D0B5F873
:10F950009030934208BF0923CFD105EB03135A68B7
:10F96000D968904780B90122206804F8042CF36814
:10F97000083498474445C3D1BDE8F0810023ECE743
:10F980000123EAE70323E8E704F8047CB5E704234E
:10F99000E3E70523E1E70623DFE70723DDE70823A5
:10F9A000DBE700BF7019022034180220D4180220AF
:10F9B00008B5A022002102480AF062FF002008BD1D
:10F9C000341802200388002B45D042680146002AE3
:10F9D00050D0304A108883423DD02DE9F047148A38
:10F9E000A34235D0158CAB4232D0168EB3422FD005
:10F9F000B2F84070BB422BD0B2F850C0634527D05C
:10FA0000B2F860E0734523D0B2F8708043451FD050
:10FA1000B2F880904B451BD0B2F890A0534517D058
:10FA2000E0B15CB365B36EB377B3BCF1000F2DD01A
:10FA3000BEF1000F20D0B8F1000F29D0B9F1000FAE
:10FA40000BD00920BAF1000F08D00420BDE8F087E0
:10FA50000720BDE8F08707207047082000011352F7
:10FA60004B68024453608B6800209360CB68D3607E
:10FA7000BDE8F0870E2070470620EFE70120EDE794
:10FA80000220EBE70320E9E70420E7E70520E5E7AC
:10FA90000720E3E73418022038B5864A0B6810883F
:10FAA0009BB2984229D0108A984226D0108C984256
:10FAB00023D0108E984220D0B2F8400098421CD03B
:10FAC000B2F85000984218D0B2F86000984214D0B2
:10FAD000B2F87000984210D0B2F8800098420CD072
:10FAE000B2F890209A4208D08868002800F0A980D7
:10FAF000714B1B699847002038BD8868002800F0CA
:10FB000091806E4A1568002D3BD09468002C00F05F
:10FB10009A801469002C00F098809469002C00F001
:10FB20009680146A002C00F09480946A002C00F0F7
:10FB30008680146B002C00F09080946B002C00F0F9
:10FB40009080146C002C00F09080946C002C00F0DD
:10FB50009080146D002C00F09280946D002C00F0C9
:10FB60009080146E002C00F09280946E002C00F0B7
:10FB70009080146F002C00F08E80946F002CB7D111
:10FB80000F2502EBC50442F83500A3804C4B1A78D0
:10FB9000012A60D01A7A012A47D01A7C012A5ED045
:10FBA0001A7E012A5FD093F82020012A5FD093F8B3
:10FBB0002820012A5FD093F83020012A5DD093F8E5
:10FBC0003820012A5FD093F84020012A5DD093F8B5
:10FBD0004820012A61D093F85020012A5FD093F881
:10FBE0005820012A5DD093F86020012A5BD093F859
:10FBF0006820012A59D093F87020012A57D093F831
:10FC00007820012A10D0102D1BD000242B4B2A4A1B
:10FC100003EBC50043F83540848088681369984732
:10FC2000204638BD1025B1E70F22022403EBC200A5
:10FC3000416003F83240FBF7FFF8012038BD05258D
:10FC40009FE7002038BD01259BE7022599E70325A2
:10FC500097E7042595E70022E7E7062591E70222CA
:10FC6000E3E707258DE70322DFE7082589E704227C
:10FC7000DBE7092585E70522D7E70622D5E70A2530
:10FC80007FE70B257DE70722CFE70822CDE70C258C
:10FC900077E70D2575E70E2573E70922C5E70A22E8
:10FCA000C3E70B22C1E70C22BFE70D22BDE70E22FE
:10FCB000BBE700BF34180220D4180220EC18022041
:10FCC0006C190220F0B4002952D0002850D083686B
:10FCD000002B4DD00369002B4AD04368002B47D03E
:10FCE000C368002B44D00368002B41D04369002B2C
:10FCF0003ED00126002504460F461F4A1F4BDFF861
:10FD000080C01674167682F8206082F8286082F827
:10FD1000306082F8386082F8406082F8486082F88B
:10FD2000506082F8586082F8606082F8686082F8FB
:10FD3000706082F878601D619D611D629D621D6327
:10FD40009D631D649D641D659D651D669D661D67A3
:10FD50009D67167016721D609D600FCCACE80F0099
:10FD600094E803008CE803003E602846F0BC70472E
:10FD70000E252846F0BC70476C190220EC180220B2
:10FD8000D418022000283AD02DE9F04780461D4CB7
:10FD900004F1A005A368103403B19847AC42F9D12F
:10FDA0004FF001090026184C184DDFF864A004F14B
:10FDB000800714F8043C012B05D0DAF80C302068D9
:10FDC000984704F8049C55F8040C083428B1DAF874
:10FDD000103098472E8045F8046CBC4205F10805A8
:10FDE000E7D1D8F800001822013800EB40000AEBF8
:10FDF000C00000210AF044FD0020BDE8F0870E207D
:10FE0000704700BF3418022070190220F018022039
:10FE1000D418022068B171B1094A53686BB14B68BC
:10FE2000088023F0FF0343F0020312684B6008468A
:10FE30001047072070470E2070470820704700BF0A
:10FE4000D41802205AB3E8B100232DE9F041DFF8BD
:10FE500058801360D8F804301BB316460C4605468C
:10FE600098470746C8B1C46074B12046D8F8083036
:10FE70009847B86060B93846D8F80C3098470420E5
:10FE8000BDE8F08107207047047244728472C47226
:10FE90003D8037600020BDE8F0810420F0E70E20AF
:10FEA00070470820ECE700BFD418022000283DD09E
:10FEB000002900F0918038B5524C6368002B37D090
:10FEC000514A08465368994234D0D36898423DD08D
:10FED000536998423FD0D369984241D0536A9842BF
:10FEE00044D0D36A984247D0536B98424AD0D36BE0
:10FEF00098424DD0536C984250D0D36C984253D016
:10FF0000536D984256D0D36D984259D0536E984253
:10FF10005CD0D36E984261D0536F984264D0D36F57
:10FF2000834267D0E3689847002038BD07207047B8
:10FF3000082038BD11780329C7D1002101251846B2
:10FF4000E46802F83150A047002038BD117A032937
:10FF5000BED10121F2E7117C0329BCD10221EDE7DA
:10FF6000117E0329EAD0536A9842BAD192F8201040
:10FF70000329B6D10421E1E792F828100329B3D16F
:10FF80000521DBE792F830100329B0D10621D5E72F
:10FF900092F838100329ADD10721CFE792F840102D
:10FFA0000329AAD10821C9E792F848100329A7D14B
:10FFB0000921C3E792F850100329A4D10A21BDE713
:10FFC00092F858100329A1D10B21B7E792F86010DD
:10FFD00003299ED10C21B1E70E20704792F86810DA
:10FFE000032999D10D21A9E792F87010032996D120
:10FFF0000E21A3E792F87830032B93D103460F210B
:020000040001F9
:100000009CE700BFD41802206C19022000283DD0C4
:10001000002900F08B8038B54F4A5368002B37D049
:100020004E4B1C68A14235D09C68A1423DD01C6952
:10003000A1423FD09C69A14241D01C6AA14243D059
:100040009C6AA14245D01C6BA14247D09C6BA14247
:1000500049D01C6CA1424BD09C6CA1424ED01C6D6F
:10006000A14251D09C6DA14254D01C6EA14257D0E8
:100070009C6EA1425CD01C6FA1425FD09C6F8C42F1
:1000800062D0084613699847002038BD07207047A2
:10009000082038BD9C888442C6D10024002003EB90
:1000A000C40543F83400A880EBE79C898442BED1A4
:1000B0000124F3E79C8A8442BCD10224EEE79C8BA6
:1000C0008442BAD10324E9E79C8C8442B8D1042449
:1000D000E4E79C8D8442B6D10524DFE79C8E844200
:1000E000B4D10624DAE79C8F8442B2D10724D5E745
:1000F000B3F844408442AFD10824CFE7B3F84C4072
:100100008442ACD10924C9E7B3F854408442A9D150
:100110000A24C3E7B3F85C408442A6D10B24BDE7B0
:10012000B3F864408442A3D10C24B7E70E20704793
:10013000B3F86C4084429ED10D24AFE7B3F874400D
:1001400084429BD10E24A9E7B3F87C40844208BFC7
:100150000F2496D1A2E700BFD4180220EC18022089
:1001600010B50446006802F0F7FFA06818B1BDE8BA
:10017000104001F017BA10BD70B5524A054600682C
:1001800012880668504BB2EB164F84B00C461860CC
:100190002BD044F201039C4203D044F202039C4260
:1001A00007D14A4E33685B0706D4286808B102F0CD
:1001B000D3FF002004B070BD022001F0D5F9022267
:1001C000048069682C68424B1B68CDE900410290AD
:1001D00003921A68184669465368984700203368A6
:1001E00043F48033336004B070BD384E326811027E
:1001F00010D542F2020294420CD14368002B5DD12B
:10020000336843F080733360336823F40003336052
:100210003368BEE7326892020FD542F2030294427D
:100220000BD14368002B3ED002F096FF00203368CC
:1002300023F40013336004B070BD42F20102944213
:100240000AD11B685B68002BB3D133681B0C1B04FD
:1002500043F002033360ACE742F20402944298D1C7
:100260001B685B6893B9336843F480033360336879
:100270009BB2032B33681BD09BB2042BD6D13368BF
:100280001B0C1B0443F002033360CFE70028CDD0E2
:1002900033689BB2032BC7D133681B0C1B0443F09C
:1002A00002033360C0E7336843F480033360BDE783
:1002B0001B0C1B0443F004033360B7E702F04CFF50
:1002C000A2E700BFBE1C0220F0190220EC19022098
:1002D000F41902202DE9F04F684CB7B0A04240F06D
:1002E000C7808846002900F0B780C02A40F0B4805B
:1002F000634D99462B689BB2042B40F0B3800221DA
:100300004FF0B60C064600242B680DF10E0223F4C4
:1003100080332B60DFF870A108AB5A4FCDF814C0C2
:1003200007910493069209EA010BDAF800004A46A5
:10033000036804A99B689847002811DABBF1000FF5
:100340006AD12B68D803F0D40CB1EEE730B9394646
:100350003046FAF7DFFC2B68D903F7D50446E4E70B
:10036000034644F20201BDF80E208A4269D044F2ED
:1003700001018A4201936FD1DDE90A7001220C99D3
:10038000099EC8E90401C8E902670D980E9988F82A
:1003900000200F9AC8F818001098C8F81C10C8F868
:1003A00020209DF85D10DDF84D20C8F82400DDF810
:1003B000510088F84010DDF85510C8F83020DDF8FD
:1003C0005920C8F83400BDF84400C8F83810C8F8FF
:1003D0003C20DDF846109DF84A20A8F82800C8F80F
:1003E0002A1088F82E2008F1420078220DF15E01D3
:1003F0000AF019FA019BDAF8000001930268D2684A
:1004000090470028019B03DD2A6842F480322A606D
:10041000184637B0BDE8F08F421C0346A1D10190C9
:100420003CB923200AF00DFB019B184637B0BDE80C
:10043000F08F20460AF005FB019B184637B0BDE857
:10044000F08F4046022208A900F8082B1A460193B3
:100450000AF0E9F9019BCEE716200AF0F2FA4FF014
:10046000FF33D5E739200AF0ECFA4FF0FF33CFE73E
:1004700009200AF0E6FA4FF0FF33C9E74354764902
:10048000EC19022078500220F41902202DE9F047DF
:1004900041F20204224286B0944D04D02C68A4B2EA
:1004A000022C40F0F6802C68A40200F11981B1F50D
:1004B000017F40F009818E49884240F00B81013A6A
:1004C000072A00F2DE80DFE802F077C0CC838F9A43
:1004D000A6042B689BB2042B40F0DB8041F204069B
:1004E000002337468DF808308DF809308DF80A3032
:1004F0008DF80B308DF80C302B68112143F400136C
:1005000068462B6002F0F6FD04460098002C40F08F
:10051000C680002800F0C38011224FF076084FF00B
:10052000490E4FF0430A4FF05409DFF8CCC106A939
:10053000BCF8003080F80E8001339BB246EA0346D7
:1005400041F8146D44718471C471047244728472F0
:10055000C472027180F80CA080F80D9080F80FE052
:10056000DFF898810068ACF800300AF05CF9394691
:100570000098C8F8004002F0D1FD002840F09A80B1
:100580005C4F5B4E39463046FAF7C4FB2C6814F4D6
:100590000014F7D1D8F8000018B102F0DDFDC8F85A
:1005A00000402B685B0266D500202B6823F4800393
:1005B0002B6006B0BDE8F0870E9A022A61D10822AE
:1005C00041F203061B880292ADF80F30374693E7DD
:1005D0000E9A022A55D1202241F203061B8802926C
:1005E000ADF81330374687E70E9A012A49D141F218
:1005F00003061B7802928DF80C3037467CE70E9A82
:10060000012A3ED1022241F203061B7802928DF8A4
:100610000D30374670E72B689BB2022B39D1002290
:10062000012141F204062B688DF808101B0C1B04F5
:1006300043F003032B608DF809208DF80A208DF814
:100640000B208DF80C20374656E70E9A022A18D157
:10065000102241F203061B880292ADF81130374692
:100660004AE70E9A012A0CD11B78012B09D141F2DD
:100670000306374640E70E200AF0E3F94FF0FF305B
:1006800093E716200AF0DDF94FF0FF3006B0BDE821
:10069000F0870E200AF0D5F94FF0FF3089E70368A4
:1006A0001BB1184602F058FD009802F04DFD2320C2
:1006B0000AF0C7F92B680E2023F400132B600AF010
:1006C000C0F94FF0FF3074E72A200AF0BAF94FF072
:1006D000FF306EE709200AF0B4F94FF0FF3068E709
:1006E00073200AF0AEF94FF0FF3062E7EC190220F8
:1006F0004354764978500220BE1C0220F019022093
:100700002DE9F04F814C87B025689846ADB2022D97
:10071000109B40F0DC802568EE0300F1F080256836
:100720002D0200F1E680B1F5017F40F0D6807849D6
:10073000884240F0D880B8F1000F0BD053B1571E5B
:10074000052F07D8DFE807F00F0F030F03031B681F
:10075000012B0BD016200AF074F94FF0FF35284614
:1007600007B0BDE8F08F1B68022BF3D1236811227C
:1007700043F40003002101A823600AF081F811214D
:10078000684602F0B7FC05460098002D40F08A80CC
:10079000002800F0878041F202064FF0490E112236
:1007A0004FF076094FF0430B4FF0540ADFF868C161
:1007B00080F80FE0BCF8003080F80E9001339BB257
:1007C00046EA034ECDF804E045718571C5710572A6
:1007D00045728572C57201A9027180F80CB080F86B
:1007E0000DA0DFF838910068ACF800300AF01BF873
:1007F00031460098C9F8005002F090FC00285CD106
:10080000444E434D31462846FAF784FA23681B02CA
:10081000F8D4D9F80000D8B1256815F080750FD04C
:10082000052F37D8DFE807F01A20262B31030025E3
:10083000437B88F8003002F08FFC0023C9F80030B9
:10084000236823F080732360284607B0BDE8F08F4B
:100850002368054623F080732360F5E7B0F80F3076
:100860000025A8F80030E6E7B0F811300025A8F818
:100870000030E0E7837B002588F80030DBE7B0F844
:1008800013300025A8F80030D5E7037B002588F851
:100890000030D0E716200AF0D4F84FF0FF35D9F831
:1008A0000000C8E703681BB1184602F055FC009829
:1008B00002F04AFC23200AF0C4F823680E2023F437
:1008C000000323604FF0FF350AF0BBF847E70E2026
:1008D0000AF0B7F84FF0FF3541E72A200AF0B1F8E7
:1008E0004FF0FF353BE709200AF0ABF84FF0FF353A
:1008F00035E773200AF0A5F84FF0FF352FE7052004
:100900000AF09FF84FF0FF3529E700BFEC190220ED
:100910004354764978500220BE1C0220F019022070
:10092000002138B5094C0A4D22680A480A4B2A4072
:1009300022600180196002F0D7FB28B923682B40A0
:1009400043F00103236038BD032038BDEC190220B9
:100950000000FFFFBE1C0220F01902202DE9F04329
:10096000012887B063D1B2F5017F60D102295ED141
:100970003A4C23689BB2012B6AD11121684602F0E0
:10098000B9FB05460098002D57D1002855D041F2FB
:1009900001064FF0490C11224FF0760E4FF043093B
:1009A0004FF054082E4F06A93B8880F80FC0013342
:1009B0009BB246EA034C41F814CD45718571C5716F
:1009C000057245728572C572027180F80C9080F8CC
:1009D0000D8080F80EE000683B8009F024FF214B79
:1009E000314600981D6002F099FB002830D11E4E60
:1009F0001E4D31462846FAF78DF923689BB2012B2C
:100A0000F7D0206880B202280CD10022184900F0EB
:100A100093FF02681749126808609047134807B0AF
:100A2000BDE8F0834FF0FF3007B0BDE8F08316203B
:100A30000AF007F84FF0FF30F1E703681BB11846E2
:100A400002F08AFB009802F07FFB232009F0F9FFF7
:100A50000E2009F0F6FF4FF0FF30E0E7EC1902201E
:100A6000BE1C0220F019022078500220435476491F
:100A700061010100F419022008B50E4B98420CD117
:100A80000D4A13689BB2022B0DD1136800201B0C7A
:100A90001B0443F00103136008BD092009F0D1FFD6
:100AA0004FF0FF3008BD0E2009F0CBFF4FF0FF30B4
:100AB00008BD00BF43547649EC190220F0B53B4C09
:100AC000C7B0266816BB01273948276009F060FEC9
:100AD0000546C0F5807331464FF4807206A8029334
:100AE00009F0CEFE2A46324906A809F09CFE06AA65
:100AF000009702AB2A4420212E4800F091FD0646C3
:100B000038B100232320236047B0F0BD0E2047B04A
:100B1000F0BD2220029B27601D4406AF06AB78552E
:100B20002B4440F20122022166205E7001F094F80D
:100B3000071EE6DB204809F02BFE334602461E491D
:100B4000CDE90066384601F037F8023503A933468F
:100B50000A22CDE90066384601F010F9CDE90066B9
:100B600006A92A463346384601F026F8A84203D0A3
:100B7000384601F0BBF8C4E7CDE9006633460A22E7
:100B800003A9384601F0FAF80128F1DD03A8022292
:100B90000A4909F012FE05460028E9D10223384629
:100BA000236001F0A3F82846AEE700BFF819022041
:100BB00034BB0100CC21022044BB010040BA01003B
:100BC00070B504460D461646FBF704FA30B10368CB
:100BD000324629462046BDE8704018474FF0FF30A6
:100BE00070BD00BF10B50446FBF736FA20B143686C
:100BF0002046BDE8104018474FF0FF3010BD00BF41
:100C00002DE9F0470D46DDE9088916461F460446E2
:100C1000FBF722FA58B1CDE90889D0F808E03B4645
:100C2000324629462046F446BDE8F04760474FF07B
:100C3000FF30BDE8F08700BF2DE9F04182B00E46DD
:100C4000174698460546FBF707FA60B104460020B0
:100C5000CDE9000043463A4631462846A468A047FD
:100C600002B0BDE8F0814FF0FF30F9E72DE9F04721
:100C70000D46DDE9088916461F460446FBF7ECF9E8
:100C800058B1CDE90889D0F80CE03B4632462946F8
:100C90002046F446BDE8F04760474FF0FF30BDE81E
:100CA000F08700BF2DE9F04182B00E461746984606
:100CB0000546FBF7D1F960B104460020CDE90000FC
:100CC00043463A4631462846E468A04702B0BDE8AC
:100CD000F0814FF0FF30F9E770B50D461646044637
:100CE000FBF7BAF930B14369324629462046BDE8E0
:100CF000704018474FF0FF3070BD00BF70B50D4613
:100D00000446FBF7A9F928B1836929462046BDE8C6
:100D1000704018474FF0FF3070BD00BF2DE9F04123
:100D20000D4616460446FBF797F940B1C7693246AF
:100D300029462046BC46BDE8F041002360474FF0FD
:100D4000FF30BDE8F08100BF70B50D461646044681
:100D5000FBF782F930B10369324629462046BDE8E7
:100D6000704018474FF0FF3070BD00BF2DE9F041D3
:100D7000DDF818800D4616461F460446FBF76CF951
:100D800058B1CDF81880D0F820E03B4632462946CD
:100D90002046F446BDE8F04160474FF0FF30BDE823
:100DA000F08100BF2DE9F041DDF818800D461646B0
:100DB0001F460446FBF750F958B1CDF81880D0F81B
:100DC00024E03B46324629462046F446BDE8F04141
:100DD00060474FF0FF30BDE8F08100BF02F012B96C
:100DE00002F012B902F012B902F068B92DE9F04F21
:100DF000DFF8CCC083B000900CF13C0BDCF808307D
:100E00002BB1DCF80020009C1078A04206D00CF139
:100E10000C0CE345F2D103B0BDE8F08FDCF804A080
:100E200003EB0A08C245F2D25368CDF804C0D64697
:100E30009C46D2F810909789AEEB0A00DFB3B9F860
:100E4000022090421CD36546002409F1040303E00C
:100E50005A880433824215D833F8046C0134A7420F
:100E600002FB0655A0EB02001E46F1D10020814294
:100E70000DD00EF1010EF045DED1DDF804C0C6E75D
:100E800065464E46338800FB03508142F1D1BEF5E2
:100E9000007FDDF804C0BAD00123084A4FEA5E1192
:100EA00052F821000EF01F0E03FA0EFE4EEA00006B
:100EB00042F82100AFE73846D9E700BFFC1902200D
:100EC000401A0220002850D06D4BD3F88820904261
:100ED0004BD82DE9F04FD3F88CB083B0BBF1000FA5
:100EE00054D00BF1FF32914600264FF01208654FA7
:100EF00001920BF1110E06EB090253F83840013252
:100F0000520804EB440C02F1120153F8315057F827
:100F10002CA053F83E4003EBC80CDCF804C005EBF2
:100F2000450504EB4404DAF810A057F8255057F8AB
:100F300024403AF82CA003EBC10103EBCE0C496826
:100F40002D692469DCF804C0504535F8215034F887
:100F50002C1015D9884211D2A84208D9561CB14587
:100F6000C0F0878002F11308C5E70020704702F146
:100F7000FF394E457DD802F1110EBCE709F101069B
:100F8000B34507D0102E01D0B34508D8002003B0D8
:100F9000BDE8F08F019A102A18BF1646F6D0DFF888
:100FA000E8C003EBC608D8E9242402EB420257F854
:100FB000223007EB8202D2F804E01D69002C56D0E3
:100FC0002A467046A40005EB040951880432914575
:100FD0000844FAD12919B1F802A08244824518D9EF
:100FE00041095CF8212000F01F0422FA04F919F0ED
:100FF000010F07D013E05CF8212022FA04F919F060
:10100000010F0CD1013082454FEA501100F01F044E
:10101000F1D101365E4508F10808C4D3B6E70126D0
:1010200006FA04F49E8922EA0402A0EB0E004CF8B2
:1010300021205C68002EA9D06A88824211D8002144
:101040002B1D03E05A88043382420AD833F8045C2B
:1010500001318E4202FB0544A0EB02001D46F1D196
:1010600094E72B8800FB034003B0BDE8F08F704687
:10107000B0E7BBF1100F08BF0F2690D086E700BF86
:101080007C1A0220401A0220FC19022000284CD0B1
:101090006B4B1A68904248D82DE9F04F5F6883B0D7
:1010A0000097002F51D07A1E964600214FF0010C78
:1010B000644C019201EB0E02013253F83C5052088D
:1010C00002F1010805EB450553F8379054F825A0C7
:1010D00053F8386009EB490503EBCC09D9F80490C3
:1010E00006EB4606DAF810A054F8266054F82550AE
:1010F0003AF829A003EBC80B03EBC7093669DBF804
:1011000004B02D69D9F80490504536F82B6035F8B5
:10111000295013D9A84210D2B04208D9C645414639
:10112000C0F0878008F1010CC4E70020704702F18D
:10113000FF3E71457DD81746BCE73946009A8A4282
:1011400007D0102901D08A4208D8002003B0BDE89A
:10115000F08F019A102A18BF1146F6D0DFF8E8C0C8
:10116000DDF8009003EBC108D8E9022602EB420249
:1011700054F8223004EB8202D2F804E01F69002EFA
:1011800055D03A467046B60007EB060A5588043239
:1011900092452844FAD1BD19B5F802B0834483457D
:1011A00018D945095CF8252000F01F0622FA06FA36
:1011B0001AF0010F07D013E05CF8252022FA06FA96
:1011C0001AF0010F0CD1013083454FEA501500F0A1
:1011D0001F06F1D10131494508F10808C4D3B4E72D
:1011E0000121B1409E8922EA0102A0EB0E004CF8D9
:1011F00025205C68002EA8D07A88824211D8002170
:101200003B1D03E05A88043382420AD833F8045C59
:1012100001318E42A0EB020002FB05441F46F1D1D2
:1012200093E73B8800FB034003B0BDE8F08F7046B6
:10123000B1E7009A102A08BF0F218FD085E700BFC1
:101240007C1A0220401A0220FC19022070B50022EC
:1012500001253348510950F8214002F01F0305FAD7
:1012600003F301322343B2F5007F40F82130F1D17E
:1012700000242C4B21463C222B481C6009F000FB2B
:1012800010210522294B2A4EC3E90044D960596137
:10129000D9615962D9625963D9635964D96459656E
:1012A000D9655966D9665967D9679A601A619A6192
:1012B0001A629A621A639A631A649A641A659A6542
:1012C0001A669A661A679A67C3E92021C3E922441D
:1012D000C3E92421C3E92621C3E92821C3E92A213E
:1012E000C3E92C21C3E92E21C3E93021C3E932210E
:1012F000C3E93421C3E93621C3E93821C3E93A21DE
:10130000C3E93C21C3E93E21C3F80411C3F800211D
:10131000C3F80C11C3F808212046357070BD00BF1A
:10132000FC1902203C1A0220401A02207C1A0220DA
:10133000CA2002202DE9F04F874B87B01B78002B85
:1013400000F08C8028B321B30B78DFF8188203EB10
:10135000031308EBC3035B68B1F80CC06344102BA4
:1013600011D84FF0000A89467C4B7D4F1B684FEA2D
:101370008C0E0093B96891B10AF1010ABAF1050F18
:1013800007F10C07F6D148F2071B584607B0BDE835
:10139000F08F48F20E1B584607B0BDE8F08FBCF145
:1013A000000F61D00D460C46D9F810300EEB030B40
:1013B0005A8833F8046B15449B4502FB0644F7D169
:1013C000D9F80830A342D7D3009B2B44B3F5007F54
:1013D000D2D2634C0AEB4A029200C0F800A0A018D7
:1013E00044F80290009A8B46C0E9012599F8012043
:1013F0005A48012A0360C8D0B9F80C30002BC4D079
:101400000025CDF80490CDF80CA0CDF814B0019BC8
:101410001F781A693B0103EB0709009308EBC90326
:10142000596832F82540029139BB039ADD609A6011
:10143000009B3B441F4608EBC3014B6858F837201C
:10144000013394424B6012D9019B48F837409B8985
:1014500001359D42DBD3DDF814B096E748F2081B56
:10146000584607B0BDE8F08F009B6546AEE7019B8C
:1014700001359B89AB42CAD8EDE7002601F1FF3A5E
:10148000049506EB0A0009EB06020132013058F818
:1014900032C04008324D09EB000109EB0A0301316B
:1014A00001330CEB4C0C58F831E055F82CB058F8DF
:1014B00033C008EBC2020EEB4E0E0CEB4C0CDBF80B
:1014C00010B0526855F82EE055F82CC008EBC10159
:1014D00008EBC3033BF82220DEF810E04968DCF893
:1014E00010C05B6894423EF821103CF823302DD99F
:1014F0009C422DD28C4224D9461CB245C1D2102622
:10150000049D029AB24211D9009B3B441A443344D1
:1015100008EBC20A08EBC309082251460AEB020095
:10152000AAF1080A09F07FF9D145F5D1009B03998A
:101530003B443344013308EBC30248F83310556091
:1015400076E700F1FF3A56459BD9D8E7049DD8E7E6
:10155000049D0AF10106D4E7CA2002203C1A0220A9
:10156000401A02207C1A0220034B1B780BB1FFF7B4
:101570008DBD1846704700BFCA20022038B5084B01
:101580001D7855B101FB00F42046FFF77FFD0546AD
:1015900018B12246002109F073F9284638BD00BF72
:1015A000CA200220044B1B7823B118B10146002049
:1015B000FFF71CBC704700BFCA200220034B1B78FA
:1015C0000BB1FFF77FBC1846704700BFCA2002204E
:1015D000044B1B7823B118B101460120FFF706BC6C
:1015E000704700BFCA2002200023184738B50A4CB4
:1015F0000A4B2578072A28BF0722084603EB451126
:1016000009F011F9237800200133DBB2072B08BF62
:101610000023237038BD00BFCB20022054BB010043
:10162000F0B5E5B09DF8A87158B152B14BB11F2982
:1016300007D919683F2904D93FB1552905D80C2489
:1016400000E01624204665B0F0BD1D4604230021AD
:101650000446164614A84FF4A0728DF80C3009F019
:101660000FF914A804F050FF002329491A4614A8C2
:10167000009305F04BF814A82022214605F06EF8DF
:10168000B8B914A804F046FF21460DF10D0008F08A
:1016900017F90446B8B9C7B114A800F03FF8022002
:1016A00000F042F8014614A800F04CF8A8B10E244E
:1016B000C8E7184A184B11782046072203EB41115E
:1016C00009F0B1F8DDE72324BCE703A9701C402230
:1016D00009F0A9F841232B60B4E70321159806F01F
:1016E00041FF0028E3D1159803AA00F188014123A6
:1016F00006F03CFD0028DAD1314614A82A6800F033
:101700006FF8B22304462B6000289BD0CFE700BFC0
:10171000ED150100CB20022054BB010010B10023C5
:10172000C0E90033704700BF022805D0034B0328EF
:101730000CBF184600207047014870476CBC010080
:101740003CBC010060B159B170B5066866B94B6A1E
:1017500004460D469847606020B12560304670BD54
:1017600002487047024870BD004870BD80C1FFFF4D
:1017700080C0FFFF10B1006800B10078704700BF63
:10178000023802288CBF002001207047806D70470E
:101790000222034B883088600A704B60704700BF9C
:1017A00034BC0100023801288CBF002001207047A2
:1017B00010B5044605F080FE2046BDE81040FFF756
:1017C000F1BE00BF10B5AC210120FFF7D7FE0446E3
:1017D00008B105F00BFE204610BD00BF06F0E4BDC9
:1017E0002DE9F04F0024D7B00DF5AB738846914634
:1017F000CDE906430746FFF7BDFF022859D18523EF
:1018000078680BAE0193224600F1880100960AAB7E
:101810000A9406F059FC2DAD044668B90798A84211
:101820007FD30A9A431B93427BD3831A18463146CF
:10183000079308F0F8FF0A9C002C31DB079B5A1B2A
:10184000002A6EDD00215A1E04F1010A079207A842
:1018500003F8011C5246294601F09EFD041E1FDBC1
:101860000322294607A801F011FEB0F1000B1BDB93
:101870003846FFF77FFF08AA09A906F0B5FE034620
:10188000C8B1002B50DBC3F1A20206A9CDE901913A
:10189000CDF800802A442549254806F0DDFE04469F
:1018A000204657B0BDE8F08F5C46204657B0BDE8F3
:1018B000F08F204CF4E705903846FFF75BFF0228D5
:1018C000059B1DD01846DDE908320090294607A87F
:1018D00001F032FE002822DB5444A34483445A46DC
:1018E000294607A801F058FD041ED9DB07A83022BD
:1018F000294601F0CBFD031E16DBA3445B44C0E781
:101900007B68324618780AA906F08AFE28B933683F
:101910000A9A294607A801F0C7FD0028D3DA044631
:10192000BEE76FF06B04BBE71C46B9E7A8BC01003B
:10193000C4BC010080C6FFFF012838B50D4614461F
:1019400011D002280AD11020FFF70EFE182220B174
:10195000074B456013448460036038BD0C20FFF7DB
:1019600003FE0022F3E71420FFF7FEFD3022EEE72E
:10197000E0BC010010B5044603681B699847236862
:1019800020465B6998472046BDE81040FFF70ABE35
:1019900010B504460C20FFF7E7FDE06028B10023F6
:1019A0002361BDE8104001F01FBC042010BD00BF42
:1019B00070B5064614200D46FFF7D6FD78B12B68AA
:1019C000044643606B6801468360EB68C360AB68A4
:1019D0000361F06801F012FC20B9686870BD4FF037
:1019E000FF3070BD2046FFF7DDFD4FF0FF3070BDCA
:1019F0002DE9F04F824687B0C0688946934601F0D2
:101A00001DFC002872D00546D9F8080020B12B69CA
:101A100013B1EA68002A5CD10023C9F80C30D9F868
:101A20000020D9F80480DAF810100192B8F1000F04
:101A30005AD00BF008030024009310E0DAF81030BD
:101A40003B44CAF81030284601F000FC3C440546EF
:101A5000002838D0A04536D90021D9F80020AE683A
:101A6000A8EB040B761A5E45374628BF5F4632B1B5
:101A70006868019B01443A46181908F0D4FE009B9F
:101A8000002BE0D15E45D9D8DAF80C0001F0CCFB90
:101A9000064670B1D0E90123D0E90301CDE9022364
:101AA000CDE90410DAE9013102A898473046FFF782
:101AB00079FD00232846CAF8103001F0C7FB3C44EA
:101AC00005460028C6D12046C9F8044007B0BDE845
:101AD000F08FD9F80C309A4228BF1A46C9F80C206A
:101AE000296908F0A0FE9AE74446ECE74FF0FF3082
:101AF000ECE700BF10B50446C06801F09FFB50B191
:101B00002469644283681C4401F0A0FB0028F9D1D9
:101B100024EAE47010BD4FF0FF3010BD30B505462B
:101B2000C06885B0A8B91AE0E86801F07DFB0446FA
:101B300070B1D0E90101D4E90332CDE90001CDE96A
:101B40000223D5E90131684698472046FFF72AFD70
:101B5000E86801F079FB0028E6D105B030BD082027
:101B600005B030BD30B50546C06885B0A0B91CE0F1
:101B700001F05AFB044670B1D0E90101D4E9033207
:101B8000CDE90001CDE90223D5E901316846984746
:101B90002046FFF707FDE86801F056FB0446E868B9
:101BA000002CE5D1FFF7FEFCEC6005B030BD00BFB6
:101BB000006801F011BB00BF70B582B00E4614463C
:101BC0000546FDF71BFE002842D003689B033FD566
:101BD0000368214623F400330360036843F4801351
:101BE000036001A801F0CEFA80BB0422019B1A72A7
:101BF00058729872D872DD6084B91846012101F0DC
:101C0000D5FAD0B94FF40032284611464FF0FF33D1
:101C1000FDF784FDA8B9204602B070BD31461868B2
:101C2000224608F000FE0121019801F0BFFA0028C9
:101C3000E8D0019B186801F0CFFA019801F0C4FACE
:101C4000232008F0FEFE4FF0FF30E5E70C20F8E718
:101C50001620F6E701F090BA2DE9F041002582B098
:101C600002AB43F8085D80460F461846164602212F
:101C70001D4AFDF7BDFC009B04460BB3C3E9028778
:101C80001E61294601A801F07DFAE8B90422019BF2
:101C9000052158729872D8721A72DC60184601F0E9
:101CA00085FAD8B902224FF0FF3311462046FDF7DE
:101CB00035FD054648B9009A136843F400331360B4
:101CC000204602B0BDE8F0810C252046FDF7E4FC7B
:101CD000284608F0B6FE4FF0FF34F1E7019801F016
:101CE00073FA2325F1E700BFB11B0100F0B583B003
:101CF0000646FDF783FD00283DD00D2307680360ED
:101D0000036804469B031FD4002101A801F03AFA9E
:101D100020BB0422019B062158729872D8721A7255
:101D2000DE60184601F042FAD0B90E224FF0FF33C0
:101D300011463046FDF7F2FC0546A8B93046FDF7DE
:101D4000ABFC284603B0F0BD0368002123F4003348
:101D5000036001A801F016FA0028DAD00C2503E090
:101D6000019801F031FA23252760284608F069FE22
:101D70004FF0FF35E5E71625F7E700BF2DE9F04105
:101D800084B0884615461E460746FDF737FD0028F5
:101D900049D00023CDE9008516F002050446CDE9BF
:101DA00002330ED01EE0002D33D14FF48032E369B0
:101DB0001146002B08BF4FF0FF333846FDF7AEFC4D
:101DC00005462368A06923F4803323600368324604
:101DD0009B6869469847B0F10008E4DB404604B0D0
:101DE000BDE8F0810368806923F4803323600368D1
:101DF00032469B6869469847B0F10008EEDAB8F1C0
:101E0000FF3FEBD1232008F01CFE404604B0BDE8A4
:101E1000F081B8F1FF3FE1D1284608F012FE4046BC
:101E200004B0BDE8F081162008F00BFE4FF0FF383B
:101E3000D4E700BFFDF702BD012901D02A20704779
:101E400038B51D461446FDF7D9FC034668B1142C7D
:101E500007D165B1049A042A05D12A680020DA6105
:101E600038BD2A2038BD162038BD092038BD0E20C7
:101E700038BD00BF70B5054684B0C0680E46FDF79A
:101E8000BDFC40B3036804469BB2012B1FD003681E
:101E90009BB20D2B27D003689BB2022B2ED0033EA2
:101EA000012E11D8002329686A68CDE90233CDE9F3
:101EB0000012A069694603685B689847013017D033
:101EC000236843F480332360002004B070BD022EE9
:101ED000E5D10660F8E728680028F5D001F07CF924
:101EE000002004B070BD022ED9D10E230360EBE7B1
:101EF000286801F071F9002004B070BD0368DB02AE
:101F0000CDD5022ECBD1036823F480130360036880
:101F100043F400330360D7E750F8081B090CFDF7C2
:101F2000F5B800BF0148FDF74DBD00BF28BD010059
:101F3000002310B582B0019358B1044601AA0420D1
:101F4000FDF780FF18B9019B0BB10833236002B085
:101F500010BD072002B010BD01F47043B3F5E04F8F
:101F60000BD160B1034630F8082C042042EA01414D
:101F700043F8081D1946FDF74DBF0F207047072095
:101F8000704700BF20B1A0F108010420FDF78EBF0B
:101F90000720704718B101460420FEF737B8072024
:101FA000704700BF2DE9F0410C460B68496923F4E6
:101FB000003323602268002322F40022226047F2CB
:101FC000810227680646FCF7E5F800283BD0054665
:101FD000284B06EBC60103EB81012422143008F0E4
:101FE00022FCAB68DFF890802433AB60236829467D
:101FF00003EA080343F00A03236047F281023B46E9
:102000002046FCF7E7F860B923681B010BD44FF0BA
:10201000FF334FF6FF720B213046FCF7EFF828B183
:102020002760BDE8F0817320BDE8F0814FF00072B9
:10203000304611464FF0FF33FCF7E0F830B173281B
:10204000EFD02760EDE70C20BDE8F081236823F096
:1020500000732360236803EA080848F00C03236038
:10206000236843F400332360236843F40023236090
:10207000BDE8F0818C1B02200000FFFF00207047AC
:1020800038B520F00803022B06D02F2008F0D9FC29
:102090004FF0FF35284638BD14464A1E012A28D87D
:1020A00014BB012906BF01234FF482744FF48774D7
:1020B0001A46FCF7CFF8051E26DB154B05EBC500CD
:1020C00003EB80002422134908F0ADFB2846FDF7FE
:1020D00095FB0368046123F400230360036823F481
:1020E00000330360284638BD012908D0B4F5877F46
:1020F000DED0162008F0A5FC4FF0FF35CAE7B4F596
:10210000827FF6D10B46D3E74FF0FF35C2E700BF21
:102110008C1B022038BD010010B50446FDF76EFB94
:1021200020B12046BDE81040FCF72EB9092008F088
:1021300088FC4FF0FF3010BD2DE9F0470D46DDE97A
:10214000088916461F460446FDF758FB00283BD079
:1021500003689BB20C2B39D003689BB20B2B11D1B7
:10216000204B04EBC40413F82430022B38D0C3688E
:10217000012B14BF39202A2008F063FC4FF0FF30F8
:10218000BDE8F087C368012B0BD0022B01D03920AA
:10219000F2E703689BB2022B07D003689BB2042BC3
:1021A00003D003689BB2052BF1D10E4B04EBC402A4
:1021B00013F82230022BEAD101462046FFF7F2FE47
:1021C000002803D0D8DCD9E70920D5E7CDE9088974
:1021D0003B46324629462046BDE8F047FCF744B965
:1021E0002320C9E78C1B02202DE9F04383B00D4664
:1021F000DDE90A8916461F460446FDF7FFFA002866
:1022000039D003689BB20C2B2AD0C368012B12D0A3
:10221000022B08D04FF0FF34232008F012FC204698
:1022200003B0BDE8F08303689BB2022B07D00368BC
:102230009BB2042B03D003689BB2052BEAD1154B4C
:1022400004EBC40213F82230022BE3D101462046EE
:10225000FFF7A8FE002812D04FF0FF34DDDCDEE7E8
:102260002046CDE900893B4632462946FCF7D0F9A5
:1022700004462320D1E74FF0FF340920CDE73B4649
:10228000324629462046CDE90A8903B0BDE8F0432D
:10229000FCF7BEB98C1B02202DE9F8430C4617460B
:1022A0000646FDF7ABFA00284CD0036805469BB202
:1022B000022B50D121463A463046FCF723FB044618
:1022C00020B1002C3FDC2046BDE8F88306EBC607B2
:1022D000DFF89480BF0018F80730012BF3D10346D4
:1022E00047F2810269693046FBF754FF8146B0B37B
:1022F00008EB07012422143008F095FAD9F80830C9
:1023000049462433C9F808302A680423120C120401
:1023100042F00A022A60284647F28102FBF75AFF80
:10232000F8B92B681B0118D430464FF0FF334FF635
:10233000FF720B21FBF762FF0028C4D00423044680
:102340002B60BEE7092420464FF0FF3408F079FBEC
:102350002046BDE8F8832D24F5E77324F3E70C2429
:10236000F1E70446ADE700BF8C1B0220F8B50E462E
:1023700017460446FDF742FAE8B1134B04EBC402DA
:1023800013F82230022B1CD1036805469BB2022BA6
:1023900003D003689BB2042B13D13A463146204642
:1023A000FCF70AFA10B1002806DCF8BD29462046E1
:1023B000FFF7F8FDF7E7092008F043FB4FF0FF3087
:1023C000F8BD2D20F8E700BF8C1B02202DE9F04757
:1023D0000F460646FDF712FA00286BD0C368044684
:1023E000012B65D103689BB2042B56D023689BB2A6
:1023F0000B2B5DD1F300DFF8C0909A1919F8222059
:10240000012A55D1012233449D0009F80520616954
:10241000002347F281023046D4F80080FBF7BAFE71
:102420008246002842D009EB05012422143008F02E
:10243000FAF9DAF8083051462433CAF8083022682D
:102440004346120C120442F00A022260204647F270
:102450008102FBF7BFFEE0B923681B010ED44FF0E9
:10246000FF334FF6FF720B213046FBF7C7FE60B11A
:102470000028C4F8008002DCBDE8F087732008F073
:10248000E0FA4FF0FF30BDE8F08739463046FCF700
:10249000CFFA0028F3DCBDE8F087F300DFF81890EE
:1024A0009A1919F82220022AA0D1ABE70C20E6E7FE
:1024B0002D20E4E70920E2E78C1B0220F8B50C464A
:1024C00016461F460546FDF799F900283BD00068DF
:1024D00080B2062837D121463B4632462846FCF7D3
:1024E0001DFB044618B1002C2EDC2046F8BD284602
:1024F000FDF784F90368184F23F400330360036881
:1025000005EBC50523F400230646036007EB8501B0
:102510002422384608F087F902233B7033682046AE
:102520001B0C1B0443F00B0333604FF6FF724FF09C
:10253000FF330C21FBF762FE04460028D5D00020B3
:10254000FBF722FFCFE7092420464FF0FF3408F0C5
:1025500078FA2046F8BD00BF8C1B02202DE9F0411F
:10256000B1F58D7F069F1DD11C46C3B1BFB1054695
:102570001646FDF743F9C8B103689BB2022B07D09A
:1025800003689BB2042B03D003689BB2052B0DD1CB
:10259000013E032E51D8DFE806F02532180B0E203D
:1025A000BDE8F081BDE8F041FCF7F0BB0920F7E79A
:1025B000042F39D12368022B36D8214A05EBC505F3
:1025C00002EB8505AB700020EAE7012F2CD12378C0
:1025D000012B29D81A4A05EBC50502EB8502537079
:1025E0000020DDE7042F1FD12068F8B101281BD19E
:1025F000134B05EBC50503F825000020D0E75FEA83
:10260000970C11D017F003060ED105EBC505AD00F0
:102610000B4B281D18442B443A46214683F803C02F
:1026200008F001F93046BBE71620B9E70222044B57
:1026300005EBC50503F82520B2E72A20B0E700BF67
:102640008C1B02202DE9F041B1F58D7F069F12D140
:102650001D466BB167B106461446FDF7CFF800285A
:102660004FD0013C032C52D8DFE804F03921150982
:102670000E20BDE8F081BDE8F041FCF73DBC3B68B1
:10268000042B3CD1234B06EBC60603EB8606B3783E
:1026900000202B60EDE73B68042B30D11D4B06EB8F
:1026A000C60603EB8606737800202B60E1E706EB95
:1026B000C60618493B68B6008A1913F00304D0789F
:1026C00021D19B08834228BF03469A00DBB1043620
:1026D00031443A60284608F0A6F82046C9E73B682E
:1026E000042B0CD10B4B06EBC60613F8263000204A
:1026F000A3F10103B3FA83F35B092B60B9E716205A
:10270000B7E70920B5E70028F9D13860B1E72A20FA
:10271000AFE700BF8C1B022038B548F28105AB4201
:102720000C4653D049F282018B422DD048F202016F
:102730008B4201D0012038BD002CFBD02369B3F5BA
:10274000827F02D0B3F5877FF4D1236823F08053D2
:1027500023605569002D48D123681B0C1B0443F0EE
:102760000503236023681A010CD5254B00EBC0023A
:1027700013F82230022B05D12146FFF713FC08B1D4
:10278000732835D1002038BD002CFBD023689BB2C4
:102790000B2BF7D1106948BB236843F0007323600B
:1027A00023681B01EED5236823F0007323602368A0
:1027B0001B0C1B0443F00C032360236843F4003319
:1027C0002360236843F40023236038BD0029D9D057
:1027D0000B689BB20A2BD5D1506938B90B681B0C1A
:1027E0001B0443F00B030B6038BD2846FBF7C8FC05
:1027F00060602368002043F48023236038BD00BF5D
:102800008C1B022008B5084AC16812880346B2EB47
:10281000114F05D0006810B100F056FD002008BD32
:10282000024A0120136008BDC01C0220B41C022013
:10283000002310B508480949094A0A4C03800B6077
:102840001360236000F00AFD10B90123236010BD5E
:102850004FF0FF3010BD00BFC01C0220B41C02208E
:10286000B01C0220AC1C0220012808B50DD140F29A
:1028700003239A4209D1022907D80A4B1A68012A70
:1028800009D102221A60084808BD162008F0D9F8BC
:102890004FF0FF3008BD0E2008F0D3F84FF0FF30A6
:1028A00008BD00BFAC1C0220325476492DE9F0432C
:1028B0004F4B85B0984240F095804E4C2368012BD9
:1028C00062D02368002B5FD02368072B5CD00723DE
:1028D00025682360052D5DD0062D05D0042D03D07D
:1028E000002005B0BDE8F0830627B8460021424E1F
:1028F000424BC6F81C161B6801A80293029B00F00D
:10290000B3FC0346002848D1019870B34FF0040E81
:10291000DFF8F0C04372BCF800208372013292B23B
:1029200047EA0247C760364FC37203714371837130
:10293000C371414680F808E0ACF800203B6000F02D
:10294000A7FC002832D0019803681BB1184600F09C
:10295000BBFC019800F0B0FC2320256008F071F862
:102960004FF0FF3005B0BDE8F0832320256008F06C
:1029700068F8234B18680028F2D00123236004690B
:1029800000F09AFC002CABD00E2008F05AF84FF063
:10299000FF30A6E72F46A846A8E72320256008F0C9
:1029A00050F84FF0FF3005B0BDE8F0834FF0FF3333
:1029B0000DF1100848F8043DDFF8389008E0D6F82B
:1029C0001C36002BCCD141464846F8F7A3F920B974
:1029D00038680028F3D0C368CFE73C20256008F0B2
:1029E00030F8BDE7092008F02CF84FF0FF3078E709
:1029F00032547649AC1C022000A002401CA60240C2
:102A0000B41C0220C01C02202DE9F047964B84B074
:102A1000984240F01C810F46002900F012811546B3
:102A2000002A00F00E81914C2368022B03D023680A
:102A3000042B40F000812668022E56D000218C4ADB
:102A40008C4BC2F81C161B682946029301A8029BF6
:102A500000F00AFC002840F09980019B93B31868AD
:102A6000002800F09E8039462A4607F0DCFE04214B
:102A70000022814F01983B88456001339BB21E04C0
:102A80000E43C6607D4E017242728272C2723B80FA
:102A9000326000F0FDFB002800F08C800198036894
:102AA0001BB1184600F010FC019800F005FC04234F
:102AB0002320236007F0C5FF4FF0FF35284604B000
:102AC000BDE8F08704232320236007F0BAFF6B4B97
:102AD00018680028F0D0046900F0EEFB002C40F0EC
:102AE000AA80284604B0BDE8F0870021DFF8808185
:102AF000604BC8F81C161B6802A80093009B00F0EE
:102B0000B3FB034600286ED1029878B30421DFF8A6
:102B100068C15B4EBCF800203668013292B2017287
:102B2000110441F003010661544EC1604372837287
:102B3000C372037143718371C3710321ACF8002028
:102B4000336000F0A5FB002857D0029803681BB142
:102B5000184600F0B9FB029800F0AEFB02232320D8
:102B600023604FF0FF3507F06CFFA7E723202660B6
:102B700007F067FF414B186800289DD0066900F0F8
:102B80009BFB002E57D10423236057E704234FF00B
:102B9000FF352320236007F054FF284604B0BDE82A
:102BA000F087184600F088FB04232320236007F0F9
:102BB00048FF5CE74FF0FF3304AFDFF8B48047F81D
:102BC000043DDFF8A89009E0D8F81C36002B7FF40C
:102BD00073AF39464846F8F79DF830BB3068002897
:102BE000F2D0C36877E74FF0FF352320266007F067
:102BF00028FF284604B0BDE8F0874FF0FF330DF101
:102C0000100949F8043DDFF864A009E0D8F81C3643
:102C1000002B7FF451AF49465046F8F77BF8E0B9F6
:102C200030680028F2D0C368A8E704233C20236062
:102C300007F007FF40E70E2007F003FF4FF0FF35D6
:102C40004FE7162007F0FDFE4FF0FF3549E709205A
:102C500007F0F7FE4FF0FF3543E702233C202360E7
:102C600007F0EFFE28E700BF32547649AC1C022083
:102C700000A002401CA60240C01C0220B41C02207E
:102C8000B01C02204FF0FF30704700BF2DE9F04329
:102C90005E4C85B0A04240F0AE8040F203208142FD
:102CA00040F08680111F032900F28280584C216871
:102CB000002900F09A802168012900F0968021689F
:102CC000072900F09280062A66D0072A07D0052A35
:102CD00011D005230020236005B0BDE8F083002B50
:102CE00066D00C9A042A63D100201A68494B1A60F6
:102CF00005B0BDE8F0830725A8460021464E474BA6
:102D00002768C6F81C161B6801A80293029B00F0F6
:102D1000ABFA0346002842D1019868B34FF0040E85
:102D2000DFF800C14372BCF800208372013292B216
:102D300045EA0245C5603A4DC37203714371837120
:102D4000C371414680F808E0ACF800202B6000F029
:102D50009FFA98B3019803681BB1184600F0B4FAC3
:102D6000019800F0A9FA2320276007F06AFE4FF0CF
:102D7000FF3005B0BDE8F0832320276007F061FE37
:102D8000274B18680028F2D0046900F095FA64BB5C
:102D9000204605B0BDE8F0830825A846ADE723200E
:102DA000276007F04EFE4FF0FF3005B0BDE8F0831E
:102DB000162007F046FE4FF0FF308DE74FF0FF334F
:102DC0000DF1100848F8043DDFF8449008E0D6F80B
:102DD0001C36002BCBD141464846F7F79BFF80B904
:102DE00028680028F3D0C368CEE70E2007F029FE3C
:102DF0004FF0FF3070E7092007F023FE4FF0FF305F
:102E00006AE73C20276007F01CFEB0E732547649A1
:102E1000AC1C0220B01C022000A002401CA60240F4
:102E2000B41C0220C01C02202DE9F04F6E4C85B06E
:102E3000A0421E460E9B40F0C88040F20320814213
:102E400040F0B180002E00F0AE80002B00F0AB808F
:102E5000511E082900F2A780644C2168002900F067
:102E6000AE802168012900F0AA802168072900F0BE
:102E7000A680022A1F6878D0072A4ED0012A6FD078
:102E80000025A94600215A4A5A4BD4F80080C2F8BE
:102E90001C161B6801A80293029B00F0E5F90028AC
:102EA00058D1019B002B3DD04FF0040EDFF850C1EC
:102EB000B9F1030FBCF80010587201F1010189B299
:102EC00045EA01429872D872187158719871D87198
:102ED000DA60ACF8001083F808E002D1464A1268C4
:102EE0001A610022454D494618462A6000F0D0F983
:102EF00000283FD0019803681BB1184600F0E4F9A0
:102F0000019800F0D9F92320C4F8008007F099FD5A
:102F10004FF0FF3005B0BDE8F08F042F43D10925F5
:102F2000A946AFE7354D2320C4F8008007F089FD9E
:102F300029680029ECD00C69002C4CD13A46143198
:102F4000304607F070FC286800F0B6F9204605B05E
:102F5000BDE8F08F2320C4F8008007F072FDD7E7AA
:102F6000242F20D1154691468CE7042F1BD1022532
:102F7000A94687E74FF0FF330DF11009DFF870A085
:102F800049F8043DDFF864B008E0DAF81C36002B9D
:102F9000BED149465846F7F7BDFE50B92968002909
:102FA000F3D0CB68C7E7162007F04BFD4FF0FF309A
:102FB000B0E73C20C4F8008007F043FDA8E70E20EE
:102FC00007F03FFD4FF0FF30A4E7092007F039FD7F
:102FD0004FF0FF309EE70E2007F033FD286800F029
:102FE0006BF94FF0FF3095E732547649AC1C022064
:102FF00000A002401CA60240B01C0220B41C02200B
:10300000C01C0220FBF77ABFFCF762B82DE9F04341
:1030100042EAE27283B00092002847D04B1E072B91
:1030200044D880460546002400EBC107AB882868D9
:1030300003F0030301A943F00C06FCF7EDFB019B31
:103040000835334025F8023C03B10134BD42EDD1CF
:1030500094BB69464046F7F75DFE074608B13C2839
:103060001DD1C1460026B9F80430D9F8000003F09C
:10307000030301A943F00C04FCF7CEFB019B09F10B
:103080000809234029F8023C03B101364D45EAD135
:103090000EB9002FDDD0304603B0BDE8F08307F055
:1030A000D0FC4FF0FF3003B0BDE8F083162007F0EE
:1030B000C8FC4FF0FF30EFE72046EDE708B5064BC0
:1030C000834303D0BDE80840FCF7E4BB2D2007F0A4
:1030D000B8FC4FF0FF3008BD3254764950F8081B59
:1030E000090CFDF749B800BF0148FCF76BBC00BFF5
:1030F0005CBD0100002310B582B0019358B10446B5
:1031000001AA0720FCF79EFE18B9019B0BB10833FA
:10311000236002B010BD072002B010BD01F470435F
:10312000B3F5805F0BD160B1034630F8082C07205F
:1031300042EA014143F8081D1946FCF76BBE0F2017
:1031400070470720704700BF20B1A0F10801072099
:10315000FCF7ACBE0720704718B101460720FCF70A
:1031600055BF0720704700BF20B150F8081B090C5D
:10317000FEF780BE704700BF0148FCF723BC00BFCC
:103180006CBD010080B1002310B582B002AA0446D4
:1031900042F8043D0320FCF755FE18B9019B0BB122
:1031A0000833236002B010BD0E20704750B10346B3
:1031B00030F8082C032042EA014143F8081D194663
:1031C000FCF728BE0E20704720B1A0F108010320B3
:1031D000FCF76CBE0E20704718B101460320FCF7C7
:1031E00015BF0E20704700BF28B100230360C0E95F
:1031F0000133184670470720704700BF0268034636
:1032000001320ED000220A6002683AB18268116071
:1032100081601A68002001321A607047C0E901110C
:10322000F7E70420704700BF0346006828B15868DC
:103230001A680168013A59601A60704703680BB157
:1032400040687047184670470068704700687047CC
:1032500050F8081B090CFFF7D5BA00BF0148FCF76E
:10326000B1BB00BF7CBD0100002310B582B001934B
:1032700058B1044601AA0620FCF7E4FD18B9019BE9
:103280000BB10833236002B010BD072002B010BD9F
:1032900011F4704F0BD160B1034630F8082C0620B2
:1032A00042EA014143F8081D1946FCF7B3BD0F205F
:1032B00070470720704700BF20B1A0F10801062029
:1032C000FCF7F4BD0720704718B101460620FCF753
:1032D0009DBE0720704700BF30B403460068B2F5BA
:1032E000803FA0EB010114D2022951DD411E19607B
:1032F00000F8012C19688224481E18600320120A65
:1033000001F8012C1A68511E196002F8014C30BCFA
:103310007047B2F1807F1AD2032939DD8324411E20
:10332000196000F8012C1968100A4D1E1D6001F883
:10333000010C1968120C481E186001F8012C1A685B
:103340000420511E196002F8014C30BC704704295A
:103350001EDD8424411E196000F8012C1968100A32
:103360004D1E1D6001F8010C1968100C4D1E1D60EA
:1033700001F8010C1968120E481E186001F8012CA2
:103380001A680520511E196002F8014C30BC7047C4
:103390006FF06B00BBE700BF30B404687F2A0346C0
:1033A000A4EB010108D800296CDD611E0160012039
:1033B00004F8012C30BC7047FF2A0ED8012961DDCA
:1033C0008121601E186004F8012C1A680220541E26
:1033D0001C6002F8011C30BC7047B2F5803F1CD362
:1033E000B2F1807F2ED203294CDD8325611E01605E
:1033F00004F8012C0168100A4C1E1C6001F8010C35
:103400001968120C481E186001F8012C1A68042073
:10341000511E196002F8015CCCE7022932DD8225D9
:10342000611E016004F8012C0168120A481E186030
:1034300001F8012C1A680320511E196002F8015C82
:1034400030BC704704291DDD8425611E016004F82D
:10345000012C0168100A4C1E1C6001F8010C19684F
:10346000100C4C1E1C6001F8010C1968120E481E4D
:10347000186001F8012C1A680520511E196002F825
:10348000015C97E76FF06B0094E700BF0368591A7F
:10349000002905DD591E0160012003F8012C704749
:1034A0006FF06B00704700BFF8B50568A9423FD8C0
:1034B0000F46691A8B423BD806461C46E81A11464D
:1034C00030601A4607F0AFF9002C204615DB7F2C40
:1034D00014D83368DA1B002A2ADD01205A1E326014
:1034E00003F8014C33680134DF1B002F20DD062276
:1034F000591E3160204403F8012CF8BDFF2C0FD871
:103500003368DA1B012A13DD8122591E316003F86A
:10351000014C33680220591E316003F8012CE1E7A9
:10352000224639463046FFF7D7FE0028DADAF8BDE2
:103530006FF06B00F8BD00BF2DE9F041DDF8188099
:103540000568B8F1000F13D16C1A002C40F3878086
:103550006C1E046005F8018C0468651A002D7EDD80
:1035600005254FF00208661E066004F8015C056838
:10357000A94274D86C1AA34271D806461C46E81AB0
:103580000F46306011461A4607F04DF9002C2046D0
:103590002FDB7F2C41D83368DA1B002A5FDD012046
:1035A0005A1E326003F8014C33680134DA1B002ADA
:1035B00055DD06220444591E002C3160204603F8D4
:1035C000012C16DB44447F2C15D83368DA1B002A03
:1035D00045DD01205A1E326003F8014C3368013486
:1035E000DF1B002F3BDD3022591E3160204403F8E1
:1035F000012CBDE8F081FF2C21D83368DA1B012AA9
:103600002DDD8122591E316003F8014C3368022000
:10361000591E316003F8012CE0E7FF2C17D83368FE
:10362000DA1B012A1BDD8122591E316003F8014C8F
:1036300033680220591E316003F8012CB4E722469A
:1036400039463046FFF748FE0028D2DBC6E722465F
:1036500039463046FFF740FE0028A5DAC9E76FF08B
:103660006B00C6E72DE9F04FDDF824C0BCF1000F78
:1036700065D0424CA4FB0C54640804EB4408C445D8
:1036800018BF0134B4F1804F71D2A40001348C42D0
:1036900069D8002867D0B8F1000F61D086460027AE
:1036A000374EDC1C002514F8031C14F8023C14F8F7
:1036B00001BC4FEAA109090101F0300106EB131A20
:1036C00016F809909B001AF801A003F03C0106EBE4
:1036D0009B13595C69F307050BF03F03F35C6AF336
:1036E0000F2561F31745033763F31F650EF10401DE
:1036F000B845CEF8005023468E4604F10304D1D8D5
:10370000BC4514D91C781E4D0137A61067454FEAF9
:10371000041404F0300415F806E015D33D262B5DA3
:1037200081F800E04B703D238E70CB700431002394
:103730009C46081A10600B706046BDE8F08FC2F816
:1037400000C06046BDE8F08F5B7881F800E005EBD3
:103750001316345D9B0003F03C034C70EE5CE2E713
:1037600047460146CCE714606FF0290CE4E74FF0C0
:10377000FF336FF0290C1360DEE700BFABAAAAAAE3
:103780008CBD01000F282DE9F04F864640F2E08203
:103790004FF00008844601F1400402F1400054F863
:1037A000406C50F8405CA3FB066718EB06082CBF82
:1037B0004FF001094FF0000915EB08054F444FF099
:1037C000000928BF4FF0010940F8405C54F83C6CF8
:1037D000B944A3FB06AB19EB0A092CBF4FF0010853
:1037E0004FF0000850F83C6C08EB0B0516EB09068F
:1037F0004FF0000828BF4FF0010840F83C6C54F827
:10380000386CA844A3FB066718EB06082CBF4FF0E2
:1038100001094FF0000950F8385C4F4415EB0805DA
:103820004FF0000928BF4FF0010940F8385C54F808
:10383000346CB944A3FB06AB19EB0A092CBF4FF05B
:1038400001084FF0000850F8346C08EB0B0516EB3C
:1038500009064FF0000828BF4FF0010840F8346C0B
:1038600054F8306CA844A3FB066718EB06082CBF7D
:103870004FF001094FF0000950F8305C4F4415EB50
:1038800008054FF0000928BF4FF0010940F8305CEF
:1038900054F82C6CB944A3FB06AB19EB0A092CBFF6
:1038A0004FF001084FF0000850F82C6C08EB0B05A6
:1038B00016EB09064FF0000828BF4FF0010840F84A
:1038C0002C6C54F8286CA844A3FB066718EB060878
:1038D0002CBF4FF001094FF0000950F8285C4F440D
:1038E00015EB08054FF0000928BF4FF0010940F81B
:1038F000285C54F8246CB944A3FB06AB19EB0A0905
:103900002CBF4FF001084FF0000850F8246C08EB72
:103910000B0516EB09064FF0000828BF4FF0010811
:1039200040F8246C54F8206CA844A3FB066718EBFD
:1039300006082CBF4FF001094FF0000950F8205C39
:103940004F4415EB08054FF0000928BF4FF001095F
:1039500040F8205C54F81C6CB944A3FB06AB19EB8F
:103960000A092CBF4FF001084FF0000850F81C6CFA
:1039700008EB0B0516EB09064FF0000828BF4FF0C7
:10398000010840F81C6C54F8186CA844A3FB0667A7
:1039900018EB06082CBF4FF001094FF0000950F852
:1039A000185C4F4415EB08054FF0000928BF4FF095
:1039B000010940F8185C54F8146CB944A3FB06AB39
:1039C00019EB0A092CBF4FF001084FF0000850F81E
:1039D000146C08EB0B0516EB09064FF0000828BF26
:1039E0004FF0010840F8146C54F8106CA844A3FB85
:1039F000066718EB06082CBF4FF001094FF00009CD
:103A000050F8105C4F4415EB08054FF0000928BF33
:103A10004FF0010940F8105C54F80C6CB944A3FB5A
:103A200006AB19EB0A092CBF4FF001084FF0000854
:103A300050F80C6C08EB0B0516EB09064FF000086C
:103A400028BF4FF0010840F80C6C54F8086CA844EB
:103A5000A3FB066718EB06082CBF4FF001094FF0D7
:103A6000000950F8085C4F4415EB08054FF00009B9
:103A700028BF4FF0010940F8085C54F8046CB944C1
:103A8000A3FB06AB19EB0A092CBF4FF001084FF05E
:103A9000000850F8046C08EB0B0516EB09064FF014
:103AA000000828BF4FF00108ACF1100CBCF10F0F5B
:103AB00040F8046CA84404F1400400F140003FF6D3
:103AC0006EAEAEF1100000090130800101440244E5
:103AD0000EF00F000728176840F292800C685668B5
:103AE000A3FB049A18EB09082CBF4FF0010C4FF010
:103AF000000C17EB08072CBF0124002417604F6847
:103B00000AEB0C05A3FB07892C4414EB08042CBF1B
:103B100001250025A61905EB09074FF0000528BF70
:103B2000012556608E683D44A3FB0678ED192CBF35
:103B300001240024966808EB0407AD194FF0000437
:103B400028BF01249560CE683C44A3FB0678E419A5
:103B50002CBF01250025D66808EB0507A4194FF0F6
:103B6000000528BF0125D4600E693D44A3FB0678FB
:103B7000ED192CBF01240024166908EB0407AD19C8
:103B80004FF0000428BF012415614E693C44A3FB9B
:103B90000678E4192CBF01250025566908EB0507B6
:103BA000A4194FF0000528BF012554618E693D44DA
:103BB000A3FB0678ED192CBF01240024966908EBBD
:103BC0000407AD194FF0000428BF01249561CE69A8
:103BD0003C44A3FB069A14EB09042CBF4FF00108E8
:103BE0004FF00008D66908EB0A05A4194FF0000849
:103BF00028BF4FF00108D4612031A8440838203292
:103C0000002800F097800C681668A3FB049A19EB53
:103C100008082CBF0124002416EB08064FF000050D
:103C200028BF01255444012805EB040816607FD005
:103C30004C685668A3FB049A19EB08082CBF0124B2
:103C4000002416EB08064FF0000528BF0125544458
:103C5000022805EB040856606AD08C689668A3FBBE
:103C6000049A19EB08082CBF0124002416EB08065F
:103C70004FF0000528BF01255444032805EB040834
:103C8000966055D0CC68D668A3FB049A19EB080857
:103C90002CBF0124002416EB08064FF0000528BFB6
:103CA00001255444042805EB0408D66040D00C6973
:103CB0001669A3FB049A19EB08042CBF4FF0010806
:103CC0004FF00008A6190AEB08054FF0000828BFBE
:103CD0004FF001080528A844166129D04C6956699F
:103CE000A3FB049A18EB09042CBF4FF001084FF016
:103CF0000008A6190AEB08054FF0000828BF4FF08E
:103D000001080628A844566112D08C699169A3FB6A
:103D1000044514EB08082CBF0123002311EB080114
:103D20004FF0000428BF01242B4404EB03089161E9
:103D300002EB80021568002315EB080528BF01235C
:103D400042F8045B4FF00108002BF3D1BDE8F08F7F
:103D50004FF00008BEE600BF4368002B33D030B4FC
:103D600003F180428568013A55F8224005EB820252
:103D70001CB109E052F8044D34B9013BFAD18B680B
:103D80001868D0B930BC70478A68126892B1012BAC
:103D900010D800680B68002801DD002B11DB002B18
:103DA00001DD002816DB2B689342EBD806D330BC2C
:103DB00000207047006830BC70470868404230BC43
:103DC00070470120DEE78B68186800B97047086803
:103DD0004042FBE74FF0FF30D4E700BF20B10023A3
:103DE0000122C0E900238360704700BFB0B110B565
:103DF0000446806860B16268531E3AB10022013BFC
:103E0000591C026000F10400F9D1A068FDF7CAFB5B
:103E100000230122C4E90023A36010BD704700BF46
:103E200070B5426805468A420C4607D842F21073C4
:103E3000994251D88A4235D3002070BD511E10D00E
:103E4000836853F82100002849D102F18042013AE9
:103E500003EB820303E053F8040D18B911464A1E20
:103E6000F9D101218C4238BF0C4604212046FDF7D0
:103E700085FB064680B3A96881B1A20006F0D3FC99
:103E8000D5E90120531E3AB10022013B591C0260C2
:103E900000F10400F9D1A868FDF784FBC5E90146EB
:103EA000002070BD04212046FDF768FB064698B14E
:103EB000A9680029F2D06A68920006F0B4FCD5E93E
:103EC0000120531E002AE7D00022013B591C02604A
:103ED00000F10400F9D1DEE76FF00F0070BD11466C
:103EE000C0E700BF884252D0F8B58A680E46054642
:103EF000002A4ED049684B1E0ED052F823000028ED
:103F00003BD101F18041013902EB810202E052F81C
:103F1000040D90BB013BFAD1012433682B606A6821
:103F2000A2420CD3AF6892000021384606F0A8FCEC
:103F3000A200B168A86806F076FC0020F8BD042154
:103F40002046FDF71BFB0746F0B1A96889B16A68F6
:103F5000920006F068FCD5E90120531E3AB1002218
:103F6000013B591C026000F10400F9D1A868FDF77B
:103F700019FB2246C5E90147D5E742F210723168C4
:103F80005C1C94422960CAD96FF00F00F8BD002074
:103F900070470028D1D0806858B169684B1E31B194
:103FA000013B5C1C026000F10400F9D1A868FDF738
:103FB000F9FA00200123C5E90030A860F8BD00BF70
:103FC000F0B54B680D4685B01446064651687BB186
:103FD000A86803F18042013A50F8227000EB820099
:103FE00027B14FE050F8042D002A4BD1013BF9D105
:103FF00089B101F18040A768013857F82020002AD4
:1040000040F0998007EB800003E050F8042D002A6F
:1040100042D10139F9D100230122B442CDE9012373
:1040200003937FD0B54205D029463046FFF75AFFAB
:104030000746A8B901233360606880B1D4F808C08E
:1040400000F18043013B5CF823200CEB830322B199
:1040500042E053F8042D002A3ED10138F9D100275F
:10406000039860B1029A531E3AB10022013B591CD9
:10407000026000F10400F9D10398FDF793FA384685
:1040800005B0F0BD0029C6D001F18040A768013815
:1040900057F82020002AB5D08B42BCD84BD3002B38
:1040A000B9D0A86803F18041013950F821C057F810
:1040B00021E08900E645084407EB0102ABD33AD87A
:1040C000014606E051F8047D52F8040D8742A2D85B
:1040D00031D3013BF6D19EE700252B46B16851F85C
:1040E000046B0135F21A41F8042C5CF8047B0C4691
:1040F000BA422CBF4FF0000E4FF0010ED21B9E4271
:104100002CBF73460EF10103854241F8042CE6D31F
:104110000BB9A4E701232268D11A9A4244F8041B80
:10412000F8D39CE7214601A8FFF7DCFE07460028EC
:1041300096D101AC76E76FF00907384605B0F0BDBF
:1041400042F210732DE9F0414F68564216439F42E8
:10415000C6F3C0164FD84268044697420D462CD885
:104160002968236801FB06F1C6F1010703FB071369
:1041700023606B688BB10023A168AA6851F8230003
:1041800052F8232000FB07F002FB060241F823202F
:104190006A6801339A42EFD8626893420AD29A0061
:1041A000A0680133815807FB01F181506168043236
:1041B0009942F5D80020BDE8F08104213846FDF78A
:1041C000DDF98046B8B1A16889B16268920006F055
:1041D0002AFBD4E90120531E3AB10022013B591CAD
:1041E000026000F10400F9D1A068FDF7DBF93A465E
:1041F000C4E90178B4E76FF00F00DCE7F8B5456873
:1042000004460E469DB18768AA003846002106F094
:1042100037FB002EACBF01234FF0FF3386EAE67177
:10422000A268A1EBE671116023600020F8BD0421B3
:104230000120FDF7A3F90746B8B1A16881B1626812
:10424000920006F0F0FAD4E90120531E32B1013B8E
:104250005A1C056000F10400F9D1A068FDF7A2F92D
:1042600001230422C4E90137CFE76FF00F00F8BD46
:104270004368B1EB431F09D283684A0953F822000F
:1042800001F01F01C84000F0010070470020704796
:10429000436813B310B48268581E24D052F820101B
:1042A000E9B903F18043013B02EB830302E053F8D9
:1042B000041DA1B90138FAD12024116800224FF061
:1042C000004302E00132202A04D00B424FEA53039C
:1042D000F8D0A01A5DF8044B7047184670474001AB
:1042E00000F12004EAE711682024E7E7436823B3DC
:1042F00010B48268581E26D052F82010F9B903F184
:104300008043013B02EB830302E053F8041DB1B983
:104310000138FAD12024116800224FF0004302E056
:104320000132202A04D00B424FEA5303F8D0A01ADE
:104330000730C0085DF8044B7047184670474001CD
:1043400000F12004E8E711682024E5E72DE9F843AF
:1043500005460F461646002A7ED00C780B4624B13F
:104360007EE013F8012F002A46D10134A642F8D18D
:10437000D5F80480B8F1000F69D104210120FDF7C0
:10438000FDF8814600286DD0A96889B16A6892005D
:1043900006F049FAD5E90120531E3AB14246013BE5
:1043A000591C026000F10400F9D1A868FDF7FAF881
:1043B00001230422C5E901390021484606F060FACC
:1043C00000230122A968A6420B602A6011D907EBDD
:1043D000060C341BAE6823F00301DF001CF8010D4E
:1043E000725807F01807B84001330243A3427250D5
:1043F000F0D10020BDE8F883321B12F0030818BF8B
:104400004FF0010842F2107308EB9208984529D842
:104410006B68984529D904214046FDF7AFF88146DD
:1044200000B3A96889B16A68920006F0FCF9D5E981
:104430000120531E3AB10022013B591C026000F1D9
:104440000400F9D1A868FDF7ADF8C5E901894FEA84
:104450008802D5F80890AFE7D0F80480144689E7C1
:104460000024CAE76FF00F00C4E7984682E700BF58
:104470002DE9F04144688846002C3ED01546621E66
:104480000746806840D050F8221099BB04F1804361
:10449000013B00EB830302E053F8041D51BB013ADA
:1044A000FAD12726016800224FF0004302E00132D2
:1044B000202A03D00B424FEA5303F8D0B61AF6086D
:1044C000B54224D32A460021404606F0D9F976B1F8
:1044D0000023A844B96823F003028C58DD0005F0DE
:1044E00018050133EC40B34208F8014DF2D1002029
:1044F000BDE8F08156012736D5E70846214606F08B
:10450000BFF92046BDE8F08101682726CBE76FF0B0
:104510000700EDE72DE9F041436804464D0901F03D
:104520001F0643B35A1ED0F808E000F099805EF8E9
:1045300022C0BCF1000F40F09C8003F180400138A4
:104540000EEB800003E050F8047D002F5ED1013AAD
:10455000F9D14FF02008DEF8007000204FF0004243
:1045600002E00130202805D03A424FEA5202F8D04A
:10457000A8EB000C6144B1EB431F0BD911F01F02F3
:1045800018BF012242F2107002EB511787426DD81A
:104590009F4240D8F5B19D425DD26FF040477F1BEE
:1045A000DA19C7EB87779200BF00A068013BC119F9
:1045B000805811449D4241F8040CA2F10402F4D148
:1045C000002103F18043013B9B00A268D150043BD2
:1045D0001A1DFAD1BEB163689D4214D20027C6F1FC
:1045E000200CAB00A0680135C15801FA06F2C25098
:1045F000A068C2583A43C250626821FA0CF7AA4236
:1046000003F10403EED80020BDE8F0814FEA421C1C
:104610000CF12008A1E704213846FCF7AFFF8046E3
:1046200020B3A16889B16268920006F0FCF8D4E971
:104630000120531E3AB10022013B591C026000F1D7
:104640000400F9D1A068FCF7ADFF3B46C4E901784E
:10465000002DBFD09FE7002BB2D1002EBBD1D2E7F7
:10466000DEF8007094464FF0200876E76FF00F00F8
:10467000CAE75201674602F1200894466DE700BF81
:10468000F8B544684D09AC423AD301F01F0132D06D
:10469000B5B10023AA008468A658043244F8236008
:1046A00044680133661B9E42F5D89C4208D9002518
:1046B0009A0084680133A550446804329C42F8D8BB
:1046C000B9B1B4B1002704F18043013B9B00C1F1B3
:1046D000200C8668013CF55825FA01F2F2508668F4
:1046E000F25842EA0702F25005FA0CF7A3F104036C
:1046F000EFD10020F8BD19B9002CFAD00B46D6E74F
:10470000054664B18668A2003046002106F0B8F87C
:1047100000230122A96818460B602A60F8BD042115
:104720000120FCF72BFF0646B8B1A96881B16A6881
:10473000920006F078F8D5E90120531E32B1013B12
:104740005A1C046000F10400F9D1A868FCF72AFFA4
:1047500001230422C5E90136D6E76FF00F00F8BD4A
:1047600070B443684A6873B1846803F18045013DC1
:1047700054F8256004EB85041EB11AE054F8045D7A
:10478000BDB9013BFAD18AB102F180448E68013C87
:1047900056F82450CDB906EB840402E054F8045DC9
:1047A0008DB9013AFAD1002B37D00268104670BC9F
:1047B0007047002AF9D002F180448E68013C56F817
:1047C0002450002DE7D09342EFD89342096803D2DA
:1047D00070BC4A42104670470268002A01DD002979
:1047E00024DB002901DD002A1DDBB3B1846803F15D
:1047F0008041013954F8215056F821008900854242
:104800000C443144D2D80CD3013B06D054F8045D9B
:1048100051F8040D8542F6D9C8E71A4670BC104617
:1048200070475242C2E74FF0FF32BFE70122BDE7B7
:10483000F0B400290546436832DB002B42D086687D
:1048400003F18042013A56F8220006EB820268B971
:104850004FF0FF30012702E052F8044D3CB9013B14
:10486000FAD1002908BF0020F0BC70470127A1B190
:10487000012B12D82868002801DD7B1C1ED0012FD7
:1048800001D1002824DB00293368B8BF494299428E
:10489000EAD315D8F0BC002070472868F0BC7047F8
:1048A00063B1866803F18042013A56F8220006EBB4
:1048B000820250B901204FF0FF37D0E70120D3E743
:1048C0004042D1E74FF0FF30CBE74FF0FF37CFE763
:1048D0004FF0FF30C8E700BF90422DE9F047074690
:1048E0000C4606D08842154602D0FFF7FBFAA0B965
:1048F0002C4601233B60656875B1A36805F18042D1
:10490000013A53F8221003EB820219B107E052F882
:10491000041D21B9013DFAD10020BDE8F08742F223
:104920001072954275D87A68AA4276D20421284638
:10493000FCF724FE064600286BD0B96889B17A6876
:10494000920005F070FFD7E90120531E3AB1002212
:10495000013B591C026000F10400F9D1B868FCF772
:1049600021FEC7E90156A36800244FEA850AA3F196
:10497000040C06EB0A00002233680CF1040CDCF88E
:1049800000101B19144628BF01225B1828BF012400
:1049900046F8043B86421444EDD1002CBCD042F2D0
:1049A00010784FF000090FE0BD6805EB0A000368BE
:1049B00000221C1928BF012240F8044B0AF1040A06
:1049C00035460124002AA7D07B686E1CAB42EED886
:1049D00046451ED8B342E7D204213046FCF7CEFD4F
:1049E0000546B0B1B96889B17A68920005F01BFF3D
:1049F000D7E90120531E3AB1013B5A1CC0F8009080
:104A000000F10400F8D1B868FCF7CCFDC7E90165F6
:104A1000CBE76FF00F00BDE8F087BE68A4E700BFEA
:104A2000F0B54B680D4685B01446064651687BB11B
:104A3000A86803F18042013A50F8227000EB82002E
:104A400027B14FE050F8042D002A4BD1013BF9D19A
:104A500089B101F18040A768013857F82020002A69
:104A600040F0998007EB800003E050F8042D002A05
:104A700042D10139F9D100230122B442CDE9012309
:104A800003937FD0B54205D029463046FFF72AFA76
:104A90000746A8B901233360606880B1D4F808C024
:104AA00000F18043013B5CF823200CEB830322B12F
:104AB00042E053F8042D002A3ED10138F9D10027F5
:104AC000039860B1029A531E3AB10022013B591C6F
:104AD000026000F10400F9D10398FCF763FD384649
:104AE00005B0F0BD0029C6D001F18040A7680138AB
:104AF00057F82020002AB5D08B42BCD84BD3002BCE
:104B0000B9D0A86803F18041013950F821C057F8A5
:104B100021E08900E645084407EB0102ABD33AD80F
:104B2000014606E051F8047D52F8040D8742A2D8F0
:104B300031D3013BF6D19EE700252B46B16851F8F1
:104B4000046B0135F21A41F8042C5CF8047B0C4626
:104B5000BA422CBF4FF0000E4FF0010ED21B9E4206
:104B60002CBF73460EF10103854241F8042CE6D3B5
:104B70000BB9A4E701232268D11A9A4244F8041B16
:104B8000F8D39CE7214601A8FFF7ACF907460028B7
:104B900096D101AC76E76FF00907384605B0F0BD55
:104BA0002DE9F0410C681368054603FB04F3002B64
:104BB00039DA4B6817460E46526883B1896803F1AB
:104BC0008040013851F820C001EB8001BCF1000F9A
:104BD00003D02EE051F8040D58BB013BFAD17AB155
:104BE00002F18041D7F808C001395CF8210078B99A
:104BF0000CEB810102E051F8040D28BB013AFAD117
:104C00003A4631462846FFF70BFF48B1BDE8F08130
:104C1000324639462846FFF703FF0028F6D16442A2
:104C20002C60BDE8F081FFF757FE0028EED12C6024
:104C3000F7E7002AE4D002F18041D7F808C0013933
:104C40005CF821000028D3D09342D9D8E0D3002BC0
:104C5000D6D0B06803F18041013950F821805CF86A
:104C600021E08900F04508440CEB0102C8D8CFD3FD
:104C7000014606E051F804CD52F8040D8445BFD832
:104C8000C6D3013BF6D1BBE72DE9F0410C681368B0
:104C9000054603FB04F3002B64DD4B6817460E4604
:104CA000526883B1896803F18040013851F820C00F
:104CB00001EB8001BCF1000F03D01FE051F8040D9F
:104CC000E0B9013BFAD182B102F18041D7F808C0C6
:104CD00001395CF8210000283BD10CEB810102E096
:104CE00051F8040DA8B9013AFAD13A46314628469E
:104CF000FFF796FE00B92C60BDE8F081002AF4D0E1
:104D000002F18041D7F808C001395CF82100002881
:104D1000E3D09342E9D81CD3002BE6D0B06803F16E
:104D20008041013950F821805CF821E08900F0458C
:104D300008440CEB0102D8D80BD3014606E051F829
:104D400004CD52F8040D8445CFD802D3013BF6D1EF
:104D5000CBE7324639462846FFF762FE0028CBD122
:104D60006442C8E7FFF7B8FD0028C4D0BDE8F08171
:104D7000002AACBF01234FF0FF33F0B501260D68C8
:104D800082EAE27C05FB03F785B0ACEBE27C002F06
:104D90000296CDE900C3CDF80CD006462CDD4B6859
:104DA0000C4673B1A76803F18041013957F821001F
:104DB00007EB810118B10EE051F8040D58B9013B21
:104DC000FAD182B9214601AA3046FFF7F9F800B9B5
:104DD000356005B0F0BD002AF4D0012BF2D83B6855
:104DE0009C45EFD3EED9224601A93046FFF718FEC5
:104DF0000028EED16D42EBE701AAFFF76DFD002818
:104E0000E6D005B0F0BD00BF2DE9F047064600230F
:104E1000012086B08E42904600900390CDE9013388
:104E2000CDE9043300F0D1800F46464500F0D5802F
:104E30007D6885B1BB6805F18042013A53F82210C4
:104E400003EB820329B1BAE053F8042D002A40F0A5
:104E5000B680013DF8D1D8F804400025002C3DD0A3
:104E6000D8F8083004F18042013A53F8221003EBDD
:104E7000820319B104E053F8042D0AB9013CFAD1B8
:104E800042F2107304EB0509994500F2B080D6F8A0
:104E900004A0D14525D904214846FCF76FFB824682
:104EA000002800F0A480B16889B17268920005F012
:104EB000BAFCD6E90120531E3AB10022013B591C2D
:104EC000026000F10400F9D1B068FCF76BFBC6E9A1
:104ED000019A4FEA8902D6F8089025E02546D6F8CF
:104EE00004A0BAF1000F40F0858004210120FCF7F6
:104EF00045FB814600287AD0B16889B1726892007A
:104F000005F091FCD6E90120531E3AB15246013B0F
:104F1000591C026000F10400F9D1B068FCF742FBB3
:104F200001230422C6E901390021484605F0A8FC06
:104F300000210123B268116033609CB104F1804903
:104F400009F1FF394FEA8909D8F80830B26853F8F7
:104F500009304A44B9682846FEF714FC013CA9F11F
:104F60000409F1D100243A68D8F8003003FB02F3B9
:104F70003360059860B1049A531E3AB10022013B98
:104F80005D1C026000F10400F9D10598FCF70AFBF2
:104F9000002201230298CDE90332059258B101990C
:104FA0004B1E31B1013B591C026000F10400F9D1E4
:104FB0000298FCF7F7FA204606B0BDE8F087D8F86B
:104FC0000440002C7FF44CAF5AE76846FEF78AFF96
:104FD00004460028CDD16F4627E703A83146FEF7E7
:104FE00081FF04460028C4D10DF10C0820E76FF0C2
:104FF0000F04BEE7D1466CE7012300B585B00092EF
:1050000001AACDE90133CDF80CD0FFF7FDFE05B0C4
:105010005DF804FB2DE9F04F5E68A3B096B1D3F8BC
:10502000088006F1804909F1FF3958F8295008EB4A
:10503000890E6DB9F446374602E05CF8044D3CB980
:10504000013FFAD16FF00B06304623B0BDE8F08F78
:105050001D68002DF6D014468A46002201219B4689
:105060006368054610911391169119911C91CDE931
:105070001122CDE91422CDE91722CDE91A22CDE97A
:105080001D22002B00F01A82A26803F18041013931
:1050900052F8210002EB810220B17BE052F8041D9E
:1050A000002977D1013BF9D158F82920002A77D17E
:1050B000724603E052F8041D00296FD1013EF9D178
:1050C00010A82146FEF70EFF0646002800F0928049
:1050D0000027129860B1119A531E3AB10022013B89
:1050E0005C1C026000F10400F9D11298FCF75AFA36
:1050F000002201231598CDE91032129258B114996B
:105100004B1E31B1013B591C026000F10400F9D182
:105110001598FCF747FA002201231898CDE91332BD
:10512000159258B117994B1E31B1013B5D1C0260BD
:1051300000F10400F9D11898FCF734FA0022012399
:105140001B98CDE91632189258B11A994B1E31B1FD
:10515000013B5C1C026000F10400F9D11B98FCF7D4
:1051600021FA002101231B91CDE91931002F3FF4D1
:105170006BAF1D9A531E32B13A46013B581C116069
:1051800002F10402F9D13846FCF70CFA304623B09C
:10519000BDE8F08F58F82920002A89D09E428FD38D
:1051A0009E4200F29081002B8AD0A16803F18042D8
:1051B000013A51F8220058F82260920086421144C8
:1051C0009044FFF47DAF00F27E810A4608E052F879
:1051D000040D58F8041D88423FF672AFC0F0738189
:1051E000013BF4D110A82146FEF77CFE06460028BC
:1051F0007FF46EAF13A85946FEF774FE06460028EA
:105200007FF466AF42F2107201236768139302378E
:105210009742109300F29381DDF85C8047451DD9D9
:1052200004213846FCF7AAF98146002800F087815E
:10523000189981B1179A920005F0F5FADDE9172067
:10524000531E32B1013B5A1C066000F10400F9D133
:105250001898FCF7A7F9B846CDE91779B8F1000F0F
:1052600000F07181189E4FEA8802002730463946C7
:1052700005F006FB0122189B1F601A9B16929342B1
:1052800040F2B28104210320FCF778F90746002898
:1052900000F055810323149ACDE91D300392002AB2
:1052A00000F07181B2F10109159900F0CF8151F838
:1052B0002900002840F0C58102F18042013A4B46A6
:1052C00001EB820204E052F8040D002840F0AE81A8
:1052D000013BF8D12026086800224FF0004102E08F
:1052E0000132202A04D001424FEA5101F8D0B31A0A
:1052F00003F01F031F2B40F09F8100230293119B9B
:1053000013A80493013BA3EB090801934FEA481348
:1053100019460593FFF7FEF8064600287FF4D9AE3C
:105320004FEA88080DE0189810A950F8083013AA21
:10533000013340F808300846FFF7A6FC002840F08B
:10534000798113A910A8FFF70BFA0028EBDA059969
:1053500013A8FFF795F9064600287FF4BAAE6FF060
:105360000303039ACDE908B502F18047049A03FBD1
:1053700009F302F18042023A9200154605934FEA82
:1053800089030393C9EBC963023FCDE90630CDE938
:105390000AA4B9000491019B4B4540F27381039824
:1053A0001299159A05F1040A125851F80A30059815
:1053B000934200EB0504189EC0F04C814FF0FF3380
:1053C00033510126189A1E9F1359A5F1040B33443B
:1053D00013514BE0DDF86C8092004046002105F04F
:1053E0004FFA00221B9B1A601996B9F1000F00F0CA
:1053F000F980159B049A9B581B9A03991360159A80
:105400001B9B525819A95A60189B0DF13C081B5957
:105410001FAA08460F93CDE91F66CDF88480FFF7D9
:10542000F3FC002840F006811D9A002A00F0C2809B
:1054300092000021384605F023FA00233B60019BCF
:105440001C96012B1CA9129B00F0ED8053F80B3029
:1054500019A83B60129B5B597B60129B53F80A3082
:10546000BB60FFF77DF9002840F31C81189A13599F
:10547000013B13511A9A002AACD104210120FCF7F8
:105480007DF88046002800F040811B9991B11A9A5E
:10549000920005F0C8F9DDE91A1002464B1E39B139
:1054A0000021013B1160591C02F10402F8D11B9844
:1054B000FCF778F80422CDE91A688EE758F829201D
:1054C000002A3FF4F5AD55B36E68EEB90421012012
:1054D000FCF754F8074690B3A96881B16A68920056
:1054E00005F0A1F9D5E90120531E32B1013B591C49
:1054F000066000F10400F9D1A868FCF753F8012315
:105500000422C5E9013701E0AF68B2000021384646
:1055100005F0B6F900210123AA6811602B60BAF1E9
:10552000000F07D021465046FEF7DCFC0646002857
:105530007FF4CEAD0026304623B0BDE8F08F0027C3
:105540006FF00F06C5E504210120FCF717F80646A9
:105550000028F4D0189989B1179A920005F063F9E0
:10556000DDE917305A1E3BB14346013A571C036030
:1055700000F10400F9D11898FCF714F80123042273
:10558000CDE9173671E61F231946029310A8FEF7DE
:10559000C1FF064600287FF49CAD029913A8FEF7D0
:1055A000B9FF064600287FF494AD149B039303F1E2
:1055B000FF39A4E6042101200D92FBF7DFFF03462B
:1055C000002800F0A28047B10D9A39460C9005F0F2
:1055D0002AF93846FBF7E6FF0C9B1F460422CDE96B
:1055E0001D6326E74B4607E704210220FBF7C6FFB1
:1055F00006460028A3D01B9989B11A9A920005F09B
:1056000012F9DDE91A1318464A1E31B1013A501C4D
:105610001F6003F10403F9D11B98FBF7C3FF0223BA
:10562000CDE91A362EE65B5919A815E75B0103F19F
:10563000200651E606464CE5C3F11F0302931946C6
:10564000A4E74FEA491303F1200645E6086820263F
:105650004B4641E64F5992B19C464FF0000B6146D4
:105660005B464BEA0700F2F7BDFD00234FF0FF3227
:105670008B4208BF824200D210463051A1E64FF063
:10568000FF30FAE7DDE9076BDDE9095A0B9C002DD5
:105690005FD016A92846FEF725FC002853D0064601
:1056A0001E9F16E50125189B1FAA1B5913A919A8AF
:1056B0000F93CDF88480CDE91F55FFF7A5FB002897
:1056C000B8D1069B019A03F10063013B13445E01CC
:1056D000314619A8FEF71EFF0028ABD110A919AA60
:1056E0000846FFF7D1FA034658BB1FA910A80F932D
:1056F000CDE91F55CDF88480FEF72EFB002807DB8F
:10570000019B5D46013B019345E66FF00F06E0E427
:1057100013A919A8FEF7E6FB00288BD1314619A87A
:10572000FEF7F8FE002885D110A919AA0846FFF750
:1057300037FA00287FF47EAF189A1359013B1351B2
:10574000DEE70646C5E4DBF80030226803FB02F31F
:105750002B60BAF1000F05D0029910A8FEF790FF58
:10576000064608B11E9FB4E4236810A95046109362
:10577000FEF7B8FB06460028F4D101240FAB1FA9A1
:1057800050460F96CDE91F442193FEF7E5FA002815
:10579000E8D1CAF80040E5E72DE9F0415368174623
:1057A00083B1946803F18045013D54F8252004EB52
:1057B00085042AB11AE154F8045D002D40F01681E9
:1057C000013BF8D10A46064601463B460020FFF75A
:1057D00021FC002851D16FF04048716891B1B06848
:1057E00001EB080350F823C000EB8302BCF1000F6B
:1057F00056D114460B4603E054F8045D002D4FD1FA
:10580000013BF9D16FF0404439463046FEF7A8FF1E
:10581000002842DB35683B6803FB05F3002B2EDDD7
:1058200073687A6883B1B168181951F820C001EB28
:105830008001BCF1000F05D090E051F8040D002864
:1058400040F08C80013BF8D18AB1D7F808C011191B
:105850005CF82100002840F0BE800CEB810104E0E0
:1058600051F8040D002840F08380013AF8D13A46FF
:1058700031463046FFF7D4F840B1BDE8F0813A46F2
:1058800031463046FFF728F80028F6D13560394612
:105890003046FEF765FF0028BCDA0020BDE8F08145
:1058A0003468002CAEDA3B6803FB04F3002B23DAE8
:1058B000BCF1000F29D1134602E053F8042D22BB9E
:1058C0000139FAD17B6873B1D7F808C003EB08023D
:1058D0005CF822500CEB82021DB171E052F8045DBD
:1058E00005BB013BFAD13A4631463046FFF798F8FE
:1058F0000028C2D1346070E73A4631463046FEF7A0
:10590000EBFF0028F6D0BDE8F0817B68002BEAD0E1
:10591000D7F808C003EB08025CF822500CEB8202B7
:10592000002DDED09942DED84AD30029DBD001EB2E
:10593000080350F823205CF823509B00954218443C
:105940006344D0D307D93BE050F8045D53F8042DED
:105950009542C8D834D30139F6D1C4E7002A86D09D
:10596000D7F808C011195CF8210000283FF475AF82
:1059700093423FF67CAF2ED3002B3FF478AFB16853
:105980001A1951F822005CF822E092008645114471
:105990006244FFF46CAF08D91DE051F804CD52F811
:1059A000040D84453FF663AF15D3013BF5D13A466C
:1059B00031463046FFF734F800287FF45EAF65E7E4
:1059C000324639463046FFF72BF800287FF455AFB2
:1059D0006442346001E7324639463046FFF720F82A
:1059E00000287FF44AAF6D4235600DE73B68002B1D
:1059F000BFF6E8AE6FF009003FE700BF2DE9F041C8
:105A00000F4601250021BB6886B004461646009566
:105A10000395CDE90111CDE90411002B40D079683F
:105A20004A1E11D053F82200002840F0C48001F132
:105A30008041013903EB810304E053F8041D002980
:105A400040F0B980013AF8D101253B680093042168
:105A50002846FBF793FD8046002800F03C81029920
:105A600089B1019A920004F0DEFEDDE90120531EA7
:105A70003AB10022013B591C026000F10400F9D147
:105A80000298FBF78FFDCDE90158AD002A460021B1
:105A9000404604F0F5FE2A46B968029804F0C3FEB9
:105AA000314603A8FEF71EFA074600285DD1019E85
:105AB000002E00F00E810146029D043D002255F8A3
:105AC000040F04E0202A01F1010100F0818020FA96
:105AD00002F313F0010302F10102F3D0049DB5B10A
:105AE00000208446059F043F002257F8046F03E01E
:105AF000202A00F1010071D026FA02F313F001030D
:105B000002F10102F4D0814228BF01460D466846E9
:105B10002946FEF7B5FD074638BB294603A8FEF720
:105B2000AFFD074608BB01236FF040460393009387
:105B3000019F7FB10298BA1950F8223000EB82021F
:105B4000002B51D13B4603E052F8041D00294BD1F4
:105B5000013BF9D1294603A8FEF7DCFC074620B932
:105B600003A92046FEF7BEF90746029860B1019AE4
:105B7000531E3AB10022013B5C1C026000F104009C
:105B8000F9D10298FBF70EFD002201230598CDE91B
:105B90000032029258B104994B1E31B1013B591C9D
:105BA000026000F10400F9D10598FBF7FBFC3846D0
:105BB00006B0BDE8F08142F210733968551C9D4271
:105BC000009100F28380002D7FF441AFA8465DE78D
:105BD0000137BE427FF472AF19467FE70CF1010C2A
:105BE000AC4581D11D4692E7009B002BB2D000212D
:105BF0008E46A0F1040C00225CF8040F03E0202A7A
:105C000001F1010142D020FA02F313F0010302F185
:105C10000102F4D06846FEF733FD07460028A4D100
:105C2000DDF810C0BCF1000F4ED001468646059F3E
:105C3000043F002257F8040F03E0202A01F101017C
:105C40002AD020FA02F313F0010302F10102F4D08A
:105C500003A8FEF715FD0746002886D103A968466C
:105C6000FEF77EFD00281DDB03AA69466846FEF7A5
:105C7000D7FE074600287FF478AF01216846FEF77B
:105C8000FFFC074600283FF453AF6EE70EF1010E0C
:105C9000BE45B0D11946BDE70EF1010EE645C8D1AB
:105CA0001946D5E703A96A460846FEF7B9FE074636
:105CB00000287FF45AAF012103A8FEF7E1FC074654
:105CC00000283FF435AF50E76146C1E76FF00F079A
:105CD0005AE7314602E702986FF00F0746E700BF28
:105CE0002DE9F043B1F5806FADF2044D00F2A580CF
:105CF0000D4617460646694618462A46B8470746DF
:105D000020B138460DF2044DBDE8F083002D00F0BF
:105D10008A809DF80030002B40F089806B46044655
:105D200003E013F8012F002A4DD10134A542F8D128
:105D3000D6F80480B8F1000F70D104210120FBF7E0
:105D40001DFC8146002875D0B16889B17268920047
:105D500004F069FDD6E90120531E3AB14246013BE9
:105D6000591C026000F10400F9D1B068FBF71AFC7D
:105D700001230422C6E901390021484604F080FDD0
:105D800000230122B168A5420B603260B9D90DEB46
:105D900005022C1BB16823F003084FEAC30E12F86A
:105DA00001CD51F808000EF0180E0CFA0EFC01336C
:105DB00040EA0C00A34241F80800EBD138460DF24E
:105DC000044DBDE8F0832A1B12F0030818BF4FF002
:105DD000010842F2107308EB920898452AD87368BC
:105DE00098452DD904214046FBF7C8FB814608B3EE
:105DF000B16889B17268920004F015FDD6E90120FE
:105E0000531E3AB10022013B591C026000F104000C
:105E1000F9D1B068FBF7C6FBC6E901894FEA8802F1
:105E2000D6F80890A8E7D6F804802C4682E72A46E0
:105E30000446C9E76FF00F0763E76FF0030760E7F9
:105E4000984677E72DE9F0435368A1B07BB1946899
:105E500003F1804C0CF1FF3C54F82C5004EB8C0403
:105E60001DB10AE054F8045D3DB9013BFAD16FF071
:105E70000304204621B0BDE8F0831368002BF6DD53
:105E800001240023064602A8059408940B940E945E
:105E900002941194149417941A940F461546CDE960
:105EA0000633CDE90933CDE90C33CDE90F33CDE924
:105EB0000333CDE91233CDE91533CDE91833CDE9FC
:105EC0001B33FFF79BFD0446A0B9039B83B10499E4
:105ED00003F18044013C51F8242001EB84042AB1F1
:105EE000B5E054F8042D002A40F0B180013BF8D110
:105EF0006FF00D04079860B1069A531E3AB1002264
:105F0000013B591C026000F10400F9D10798FBF72E
:105F100049FB002201230A98CDE90532079258B1C6
:105F200009994B1E31B1013B5F1C026000F1040076
:105F3000F9D10A98FBF736FB002201230D98CDE931
:105F400008320A9258B10C994B1E31B1013B5E1CCC
:105F5000026000F10400F9D10D98FBF723FB002249
:105F600001231098CDE90B320D9258B10F994B1EB9
:105F700031B1013B5D1C026000F10400F9D11098C1
:105F8000FBF710FB002201230498CDE90E3210929A
:105F900058B103994B1E31B1013B591C026000F10D
:105FA0000400F9D10498FBF7FDFA002201231398AD
:105FB000CDE90232049258B112994B1E31B1013B26
:105FC0005F1C026000F10400F9D11398FBF7EAFAB4
:105FD000002201231698CDE91132139258B1159978
:105FE0004B1E31B1013B5E1C026000F10400F9D18F
:105FF0001698FBF7D7FA002201231998CDE914323D
:10600000169258B118994B1E31B1013B5D1C0260CC
:1060100000F10400F9D11998FBF7C4FA002201231A
